:100000000C94360E0C945E0E0C945E0E0C945E0EE8
:100010000C945E0E0C945E0E0C945E0E0C945E0EB0
:100020000C945E0E0C945E0E0C945E0E0C943A656D
:100030000C94BC680C9467650C945E0E0C94FE16D0
:100040000C94EC160C945E0E0C945E0E0C945E0EEA
:100050000C945E0E0C945E0E0C945E0E0C945E0E70
:100060000C947C680C945A170C94D2650C949F667F
:100070000C945E0E0C945E0E0C945E0E0C945E0E50
:100080000C945E0E0C945E0E0C945E0E7C6A806A7C
:10009000886A926AA96AC36AD86AE76AFC6A136BBB
:1000A0001D6B3B6B416B466B4C6B526BAC6BB66B19
:1000B0005B6B616B676B706B746B796B816B936B54
:1000C000996B9F6BA46B846A846B896B8E6B537086
:1000D0006C617368008040000000000000000000B8
:1000E0000000000000000000000000000000000010
:1000F0000000000000000000000000000000000000
:1001000000000000000000000000000000000000EF
:1001100000000000000000000000000000000000DF
:10012000000080C0E0E0F0F8F8FCFCFCF8F8F8F023
:1001300040000000000080808000000000000000FF
:1001400000000000000000000000000080C0C0E0CF
:10015000E0E0F0F0F0E0C00000000000C0F8FFFFB9
:100160009F8783838383838383838383838383833F
:1001700083838383838383830383808383838383D2
:10018000838383838383838383838383838383833F
:100190008383C3E3733F1F0000000080E0F0F8FC9E
:1001A000FEFFFFFFFF7F3F1F1F0F0783C3E1E1E05B
:1001B000E0C0000E1F3F7F7FFFF3E0E08000000003
:1001C0000000000000000080F0FCFEFFFFFFFF7F4A
:1001D0003F0F0301010100000080F0FEFFFFC7C1D7
:1001E000C1C1C1C1C1C1C1C1C1C1C1C1C1C1C1C1FF
:1001F000C1C1C1C1C101C1F0FEFF3F0F070F0D0D0D
:100200000D1D191919193131313171616161E1C166
:10021000C1C18100000080E0F8FCFFFFFFFF2F1745
:100220000F038180C0E0F0F8FCFEFFFFFFFFFFFF3F
:100230007F010000000000000001010307070E1EFF
:100240001C3870E0F0F8FEFFFF7F1F0F0300010075
:10025000000000000000000000000000000000009E
:10026000000000000000000000000000000000008E
:10027000000000000000000000000000000000007E
:10028000000000000000000000000000000000006E
:1002900000000000007EFFFFFFFFFFFFFBF8FCFCFB
:1002A000FEFF7F3F1F0F07C3FFFFFFFFFFFF7F071B
:1002B0000000000000000000000000000000C0E09E
:1002C000F8FEFFFF7F1F0F1F3D7CF8F8F0E0800075
:1002D000000000000000000000000000000000001E
:1002E000000000000000000000000000000000000E
:1002F00000000000000000000000000000000000FE
:1003000000000000000000000000000000000000ED
:1003100000000000000000010101010103070707C0
:100320000301000000E0FCFFFFFFFFFF1F030000D0
:10033000000000000000000000C0F078DE27130974
:100340000E0703000000000000000001030F7FFF04
:10035000FC7878F800000000000000000000008039
:10036000808080808080808000808000808000008D
:1003700000000000008080808080808080808080FD
:1003800080808080808080000000000000000000ED
:10039000000000000000000000000000000000005D
:1003A000000080F0FEFFFFFFFF3F0F010000000094
:1003B00000000000C0E0381E0F0300010000000034
:1003C000000000000000000000000000000000002D
:1003D0000000030301000000000000000000000E08
:1003E0000E02020202020303000F0F000F0F0808A3
:1003F00008080808080F0F08080808080F0F000071
:1004000000000F0F000000000000000000000000CE
:1004100000000000000000000000000000000000DC
:10042000C0F8BFFFFFFF1F7F0100000000000000B9
:1004300000F0FCFF7F7830000000000000000000AA
:1004400000000000000000000000000000000000AC
:10045000000000000000000000000000000000009C
:10046000000000000000000000000000000000008C
:10047000000000000000000000000000000000007C
:10048000000000000000000000000000000000006C
:100490000000000000000000000000000000301C10
:1004A000070E0F0701000000000000000000000020
:1004B000000000000000000000000000000000003C
:1004C000000000000000000000000000000000002C
:1004D00000000000000000001B1E272D36394B4E87
:1004E000636C7278878D939CB1B4C6C9D2D8E1E4AD
:1004F0004F4646004F4E2000010203040103020450
:1005000004020301040302010301020004050607BB
:100510006D656E75537461636B206F766572666C82
:100520006F77006D656E75537461636B20756E64D3
:100530006572666C6F7700707265737320616E7997
:10054000204B657900414C455254004D4553534171
:100550004745004C4F4144494E4700202020202071
:10056000202020202020202020202020202020208B
:100570002000506C6561736520526573657420536B
:10058000776974636865730053776974636820578B
:1005900061726E696E6700204F6C642056657273DD
:1005A000696F6E20454550524F4D202020434845ED
:1005B000434B2053455454494E47532F43414C49D4
:1005C0004200416C61726D732044697361626C65B5
:1005D00064005265736574207468726F74746C651E
:1005E000005468726F74746C65206E6F7420696457
:1005F0006C6500507265737320616E79206B65794C
:1006000020746F20736B697000414C455254004553
:100610004550524F4D206C6F77206D656D004F46F1
:1006200046414253525573525525454C73454C250E
:10063000544873544825414C73414C255031205047
:10064000312550322050322550332050332500546C
:100650004852525544454C45494430494431494437
:100660003241494C47454154524E5357315357320A
:1006700053573353573453573553573653573753CC
:100680005738535739535741535742535743004FE5
:100690004646004F4E20002D2D2D004348002D2DA5
:1006A0002D200052554420454C45205448522041AD
:1006B000494C20005031202050322020503320203F
:1006C00048414C4646554C4C4359433143594332BB
:1006D0004359433350504D3150504D3250504D33AB
:1006E00050504D3450504D3550504D3650504D3780
:1006F00050504D384348312043483220434833203E
:100700004348342043483520434836204348372067
:100710004348382043483920434831304348313139
:10072000434831324348313343483134434831350B
:1007300043483136002D2D2D2D00564552533A2079
:1007400056312E353630342D6572657A0044415469
:10075000453A2031332E30332E3230313200544975
:100760004D453A2031383A30363A3231002053562E
:100770004E3A20657239782D7237343500204D4F4E
:10078000443A202020200012081200081C08080803
:100790001C08000008220049002208000000000098
:1007A000227F2200000008220049002208000008E1
:1007B000220049002208000000227F2200000000E1
:1007C00000082200490022080000081C0808081C34
:1007D0000800A22FC641AA40262A0E236652584F6F
:1007E000D6465348804EF6484B1CF81D2E1ECE1E92
:1007F000EA1F54546D0003457870457846466E658F
:100800004D656443727300544F540053544B11535D
:10081000542500544D45115453570053544154002E
:100820005B4D454E555D20746F2072656672657331
:100830006800537461636B0F6200746D61696E0FC1
:100840006D7300746D7231204A69747465720F752E
:100850007300746D72314C6174206D696E0F757325
:1008600000746D72314C6174206D61780F75730086
:100870005354415432005452453031324147004DB7
:100880006F64650042616E6447617000506F74531D
:1008900063726F6C6C00416C61726D205761726E97
:1008A000696E67004D656D6F7279205761726E6970
:1008B0006E670044656661756C74205377005377EA
:1008C00069746368205761726E696E67005468725C
:1008D0006F74746C65205761726E696E6700537037
:1008E0006C617368204E616D650053706C61736854
:1008F0002073637265656E004C69676874206F6E63
:100900002053746B204D76004C69676874206F66C5
:1009100066206166746572004C696768742073773D
:100920006974636800466C617368206F6E2062654D
:100930006570004265657020636F756E74646F77D3
:100940006E004D696E75746520626565700054684F
:10095000726F74746C6520726576657273650004DD
:1009600053494E474F534D5046494C540046696CCD
:100970007465722041444300496E6163746976690D
:10098000747920616C61726D004261747465727972
:10099000207761726E696E6700436F6E7472617367
:1009A000740048617074696320537472656E677473
:1009B0006800537065616B657220506974636800EC
:1009C00006426565706572506953706B7200536FB3
:1009D000756E64204D6F64650006517569657420FD
:1009E0004E6F4B6579207853686F727453686F72DD
:1009F00074204E6F726D20204C6F6E672020784CF3
:100A00006F6E672000426565706572004F776E6596
:100A100072204E616D6500524144494F2053455448
:100A200055500043616C004D756C7469706C69655C
:100A3000720003636831636832636833636834004B
:100A4000036F6666202B3D203A3D006D6F64650A9A
:100A500025207372632020737700536C61766500E4
:100A6000545241494E4552000003030303005645CA
:100A70005253494F4E005472696D2D202B00204D6A
:100A8000656E75204578697420446F776E2020204C
:100A900055705269676874204C656674004449411A
:100AA0004700424700414E41005B4D454E555D2099
:100AB0005748454E20444F4E45004D4F5645205314
:100AC0005449434B532F504F545300534554204DDA
:100AD0004944504F494E54005B4D454E555D20549E
:100AE0004F205354415254005354415254204341D7
:100AF0004C4942524154494F4E0043414C494252A5
:100B00004154494F4E0066726565004D4F44454C57
:100B100053454C00434F4C20446972656374696FC0
:100B20006E0041494C20446972656374696F6E00C0
:100B3000454C4520446972656374696F6E00537754
:100B40006173682052696E6700436F6C6C656374F3
:100B5000697665002D2D2D20202031323020202077
:100B600031323058202031343020202039302020BC
:100B700020200053776173682054797065004845E0
:100B80004C49205345545550000044454C4554456C
:100B9000204D4F44454C0F5B4D454E555D00543242
:100BA00054685472696700547261696E65720045D9
:100BB0002E204C696D69747300504F534E454700A9
:100BC00053686966742053656C004C50342F4C5048
:100BD00035202044534D326F6E6C792044534D3292
:100BE0002F44534D580044534D20547970650053A1
:100BF000656E64205278204E756D626572205B4D83
:100C0000454E555D0050504D2046724C656E0D6D41
:100C1000536563002052784E756D000434434820BC
:100C20003643482038434820313043483132434826
:100C3000313443483136434800755300755365637A
:100C40000050504D20202050585820202044534D13
:100C500032202050504D3136200050726F746F009A
:100C600052455441313233004265657020436E7401
:100C7000005472696D20537700064578702020205B
:100C8000457846696E6546696E6520204D656469E4
:100C9000756D436F61727365005472696D20496EA2
:100CA0006300542D4578706F00542D5472696D00A7
:100CB0000A436F756E7420446F776E436F756E7460
:100CC00020557020200054696D65722000547269AF
:100CD000676765720054696D6572004E616D6500ED
:100CE0005345545550000009010000000000000663
:100CF00002004475706C69636174696E67206D6F82
:100D000064656C005B4D454E555D20205B45584940
:100D1000545D005945530B4E4F0044454C455445D6
:100D2000204D4F44454C004455504C494341544597
:100D3000204D4F44454C00204142434445464748DE
:100D4000494A4B4C4D4E4F5051525354555657589B
:100D5000595A6162636465666768696A6B6C6D6E37
:100D60006F707172737475767778797A3031323347
:100D70003435363738395F2D2E00657870202025C0
:100D8000202073773120737732004558504F2F441D
:100D90005200000344522048696768004452204CC6
:100DA0006F77004452204D696400447253773200DB
:100DB00044725377310057656967687400457870ED
:100DC0006F004558504F2F445200002B2A52004DBF
:100DD00049584552005B4D454E555D20205B4558B6
:100DE00049545D005945530B4E4F0044454C455402
:100DF00045204D49583F005072657373205B45583C
:100E000049545D20746F2061626F7274004D617887
:100E1000206D69786572732072656163683A20009D
:100E200044454C455445204D4958205B4D454E5551
:100E30005D00536C6F772020557000536C6F7720E6
:100E400020446F776E0044656C61792055700044D2
:100E5000656C617920446F776E00084164642020DE
:100E60002020204D756C7469706C795265706C61CE
:100E7000636520004D756C747078005761726E69FF
:100E80006E670053776974636800437572766573A3
:100E9000005472696D00466C4D6F64657472696DC3
:100EA000004F666673657400466D5472696D5661D5
:100EB0006C0057656967687400536F7572636500ED
:100EC00045444954204D49582000494E53455254F9
:100ED000204D495820002D2D2D2D202020763E6FAD
:100EE00066732020763C6F667320207C767C3E6F94
:100EF00066737C767C3C6F6673414E4420202020D4
:100F00004F522020202020584F5220202020763180
:100F10003D3D7632207631213D76322076313E7667
:100F200032202076313C7632202076313E3D7632BA
:100F30002076313C3D7632200053570043555354C0
:100F40004F4D2053574954434845530000025341E5
:100F500046455459205357495443484553000002CD
:100F6000434C454152204D49584553205B4D454E19
:100F7000555D002052455441004368616E6E656CBA
:100F8000204F726465720054454D504C4154455396
:100F900000434F5059205452494D205B4D454E550A
:100FA0005D002D2D2D494E56004C494D495453009E
:100FB0000003030303030303030303030303030304
:100FC0000300435600435552564553005052455373
:100FD000455400454449542D3E0043555256450062
:100FE0000900032D2D2D494E56002D2D2D783E3014
:100FF000783C307C787C663E30663C307C667C6336
:10100000312063322063332063342063352063361C
:1010100020633720633820633920633130633131F6
:1010200063313263313363313463313563313600D8
:10103000454550524F4D206F766572666C6F770054
:10104000454550524F4D206F766572666C6F770044
:1010500067656E7772697465206572726F7200459C
:101060004550524F4D20466F726D617474696E67C2
:101070000042616420454570726F6D204461746167
:10108000004D4F44454C2020202020004D4520207D
:1010900020202020202000500850000000000000E8
:1010A00000006F000007000700147F147F14242A3B
:1010B0007F2A122313086462364955225000050323
:1010C0000000001C2241000041221C0014083E08C0
:1010D0001408083E080800503000000808080808F6
:1010E00000606000002010080402003E49453E00F8
:1010F00000427F400062514946004149493600188C
:1011000014127F0027454539003E494932000179D4
:1011100005030036494936000649291E00003636C7
:101120000000005636000008142241141414141450
:101130004122140800020151090600060909067E31
:101140000909097E7F494949363E414141227F4193
:1011500041221C7F494949417F090909013E414912
:10116000497A7F0808087F00417F41002040413FC5
:10117000017F081422417F404040407F020C027FE3
:101180007F0408107F3E4141413E7F090909063E28
:101190004151215E7F0919294626494949320101F9
:1011A0007F01013F4040403F1F2040201F3F403013
:1011B000403F6314081463070870080761514945EC
:1011C00043007F41410002040810200041417F009C
:1011D000040201020440404040400001020400209B
:1011E000545454787F484444383844444420384464
:1011F00044487F3854545418087E0901020C525256
:10120000523E7F0804047800447D40002040443D65
:10121000007F1028440000417F40007C04180478BF
:101220007C0804047838444444387C1414140808B6
:101230001414187C7C080404084854545420043FB7
:101240004440203C4040207C1C2040201C3C40204E
:10125000403C44281028440C5050503C4464544CAA
:1012600044000836410000007F00000041360800BD
:101270000808221C08081C220808A0608000000042
:101280000000000000000000000000FFFF00000060
:101290000000001F3F00003F1F00003030FFFF3004
:1012A00030FFFF30303078CCCCFFFFCCCC8C0C063C
:1012B0000F0F86C0E070381C0C3CFEC7E3F33B1EEA
:1012C0000C00000000333B1F0F000000000000F086
:1012D000F81C0E07030000000003070E1CF8F000C6
:1012E000003030E0C0FCFCC0E03030C0C0C0C0FC0A
:1012F000FCC0C0C0C000000000000000000000C032
:10130000C0C0C0C0C0C0C0C0C0000000000000001D
:1013100000000000000080C0E070381C0C000000DD
:10132000000000000000000000000038380000004D
:10133000000000000000000000000003033F3F0326
:10134000033F3F03030C0C0C0C3F3F0C0C07030C3A
:101350000E07030100183C3C180F1F383133331EB1
:101360001E333300000000000000000000000003F6
:10137000070E1C38300000000030381C0E07030038
:1013800000030301000F0F00010303000000000F22
:101390000F000000000000333B1F0F0000000000A2
:1013A0000000000000000000000000183C3C180095
:1013B0000000000C0E07030100000000000000FC0C
:1013C000FE87C3E377FEFC00000C0EFFFF00000069
:1013D0000000000C0E0783C3E77E3C00000303C33C
:1013E000C3C3E7FE3C0000C0E070381C0EFFFF00E6
:1013F000003F3F33333373E3C30000FCFEC7C3C376
:10140000C78E0C00000303C3E3733B1F0F00003CB7
:10141000FEE7C3C3E7FE3C00003C7EE7C3C3E7FE34
:10142000FC0000183C3C18000000000000183C3C88
:1014300018000000000000C0E0F0381C0E07033068
:1014400030303030303030303003070E1C38F0E0B0
:10145000C000000C0E07030383C3E77E3C00000FAF
:101460001F3B3130381F0F000030303F3F3030001D
:101470000000003C3E373331303030000030303037
:101480003030391F0F00000303030303033F3F0005
:10149000000C1C383030381F0F00000F1F38303060
:1014A000391F0F000000003F3F0000000000000F48
:1014B0001F393030391F0F0000000030381C0E0774
:1014C000030000060F0F06000000000000333B1F62
:1014D0000F000000000000000103070E1C3830035D
:1014E00003030303030303030330381C0E07030144
:1014F0000000000000000033330100000000003C49
:101500007EE7C3C3E77E3CF0F8DCCEC7C7CEDCF88D
:10151000F0FFFFC3C3C3C3C3E7FE3CFCFE070303E6
:101520000303070E0CFFFF030303070E1CF8F0FF75
:10153000FFC3C3C3C3C3C30303FFFFC3C3C3C3C347
:10154000C30303FCFE0703C3C3C3C7CECCFFFFC066
:10155000C0C0C0C0C0FFFF00000303FFFF030300C3
:1015600000000000000303FFFF0303FFFFC0E0F0E3
:10157000381C0E0703FFFF0000000000000000FF02
:10158000FF0E1CF8F81C0EFFFFFFFF3870E0C08054
:1015900000FFFFFCFE070303030307FEFC0000003F
:1015A000000000000000003F3F0000000000003F7E
:1015B0003F3F3F3030303030391F0F0F1F38303051
:1015C0003030381C0C3F3F303030381C0E07033FA2
:1015D0003F30303030303030303F3F0000000000CE
:1015E0000000000F1F3830303030303F3F3F3F00A9
:1015F00000000000003F3F000030303F3F3030002F
:10160000000C1C383030381F0F00003F3F00010332
:10161000070E1C38303F3F30303030303030303FF4
:101620003F0000000000003F3F3F3F00000001037B
:10163000033F3F0F1F3830303030381F0FFFFFC3DC
:10164000C3C3C3C3E77E3CFCFE070303030307FEDB
:10165000FCFFFFC3C3C3C3C3E77E3C3C7EE7C3C3F9
:10166000C3C3C78E0C03030303FFFF03030303FF7E
:10167000FF000000000000FFFFFFFF00000000006F
:1016800000FFFFFFFF000000000000FFFF0F1F38FA
:10169000F0E0E0F0381F0F3F7FE0C08080C0E07FC7
:1016A0003F03030383C3E3733B1F0F0000FFFF03EC
:1016B00003030300000C1C3870E0C0800000000031
:1016C0000003030303FFFF000030381C0E07070E62
:1016D0001C3830000000000000000000003F3F0008
:1016E000000000000000000F1F383033371E1C3F81
:1016F000333F3F000003070E1C38300C1C383030DD
:101700003030391F0F000000003F3F000000000F85
:101710001F3830303030381F0F03070E1C38381C8C
:101720000E07030F1F38381F1F38381F0F3C3E07A6
:1017300003010103073E3C000000013F3F010000A0
:10174000003C3E373331303030303000003F3F30E6
:10175000303030000000000000000103070E0C00D4
:1017600000303030303F3F0000000000000000003B
:101770000000003030303030303030303000000386
:10178000070E1C383000000000303030303070E080
:10179000C0FFFFC0E070303070E0C0C0E07030309B
:1017A0003030300000C0E070303070E0C0FFFFC06B
:1017B000E0703030303070E0C0C0C0FCFEC7C30302
:1017C000070E0CF0F89C0C0C0C0C0CFCFCFFFFC082
:1017D000E070303070E0C000003030F3F300000003
:1017E00000000000003030F3F30000FFFF0080C075
:1017F000E07030000000000303FFFF00000000F075
:10180000F03070E0E07070E0C0F0F0C0E0703030B8
:1018100070E0C0C0E0703030303070E0C0000000D8
:10182000000000000000000C1E3F33333333333F11
:101830003F3F3F3030303030381F0F0F1F383030CF
:101840003030381C0C0F1F3830303030303F3F0FF5
:101850001F3B3333333333030300003F3F000000AB
:10186000000000000133333333333B1F0F3F3F0091
:1018700000000000003F3F000030303F3F303000AC
:10188000000C1C383030381F0F00003F3F03070F9B
:101890001C38300000000030303F3F303000003F47
:1018A0003F0000030300003F3F3F3F0000000000F7
:1018B000003F3F0F1F3830303030381F0FF0F0300E
:1018C00030303030F0E0C0C0E0F0303030E0C0F018
:1018D000F0F0F0C0E070303070E0C0C0E0F03030C8
:1018E00030303000003030FFFF303000000000F0BA
:1018F000F0000000000000F0F0F0F0000000000038
:1019000000F0F0F0F0000000000000F0F03070E0B7
:10191000C08080C0E07030F0F0800000000000F077
:10192000F03030303030B0F0F070300000C0E03CCB
:101930003E0703000000000000FFFF000000000061
:101940000003073E3CE0C00000C0C0C0C00C1CF853
:10195000F0E0C0C0E0F0F81C0CC0C0C0C03F3F03C6
:101960000303030303010000010303030303033F15
:101970003F3F3F00000000000000003031333333B0
:1019800033333F1E0C00000F1F383030381C0C0F53
:101990001F383030381C0C3F3F03070E1C38381CF2
:1019A0000E07030F1F38381C1C38381F0F30381C27
:1019B0000F07070F1C3830000133333333333B1F1D
:1019C0000F30383C3E373331303030000000010FEB
:1019D0001F38300000000000003F3F000000000002
:1019E0000030381F0F01000000000000000C0E073F
:1019F000030100000103070E0C00000000408008F6
:101A00000420100201151A211A271A341A3B1A4809
:101A10001A531A5E1A53696D706C6520342D434851
:101A200000542D43757400537469636B7920542DF1
:101A300043757400562D5461696C00456C65766F72
:101A40006E5C44656C74610048656C692053657414
:101A50007570004779726F20536574757000536517
:101A600072766F2054657374000000891112239BF5
:101A7000322446AD573665BF74488CC19D5AAFD3EA
:101A8000BE6CCAE5DB7EE9F7F88110080193331AD2
:101A900022A5562C47B7753E64C99C408DDBBF52CA
:101AA000AEEDDA64CBFFF976E802218B30100299B3
:101AB000132667AF763444BD554AADC3BC588ED1AA
:101AC0009F6EEBE7FA7CC8F5D983310A2091121892
:101AD00003A7772E66B5543C45CBBD42ACD99E508A
:101AE0008FEFFB66EAFDD874C904428D5316619FDF
:101AF000702004A9153227BB364CCEC5DF5EEDD76A
:101B0000FC6888E1997AABF3BA85520C4397711E51
:101B100060A1142805B3373A26CDDE44CFDFFD5649
:101B2000ECE9986089FBBB72AA06638F7214409D32
:101B3000512225AB343006B9174EEFC7FE5CCCD529
:101B4000DD6AA9E3B8788AF19B87730E6295501C11
:101B500041A3352A24B1163807CFFF46EEDDDC5409
:101B6000CDEBB962A8F99A708B088481951AA79376
:101B7000B62CC2A5D33EE1B7F04008C919522BDB01
:101B80003A644EED5F766DFF7C899400859BB712B9
:101B9000A6ADD224C3BFF136E0C1184809D33B5AE1
:101BA0002AE55E6C4FF77D7E6C0AA583B41886919A
:101BB000972EE3A7F23CC0B5D14229CB38500AD9C1
:101BC0001B666FEF7E744CFD5D8BB502A499961079
:101BD00087AFF326E2BDD034C1C3394A28D11A58A1
:101BE0000BE77F6E6EF55C7C4D0CC685D71EE597C6
:101BF000F42880A1913AA3B3B2444ACD5B5669DF81
:101C000078600CE91D722FFB3E8DD604C79FF51638
:101C1000E4A9902081BBB332A2C55A4C4BD7795E60
:101C200068E11C680DF33F7A2E0EE787F61CC49519
:101C3000D52AA1A3B03882B193466BCF7A5448DD40
:101C400059622DEB3C700EF91F8FF706E69DD414F8
:101C5000C5ABB122A0B9923083C77B4E6AD5585C20
:101C600049E33D6A2CF11E780F00941811241FBE21
:101C7000CFEFD0E1DEBFCDBF11E0A0E0B1E0EEE5F7
:101C8000F9ED02C005900D92A234B107D9F71EE01C
:101C9000A2E4B1E001C01D92A437B107E1F71CE155
:101CA000CCE6DCE104C02297FE010E94686CCA36D3
:101CB000D107C9F70E9415180C94AD6C0C94000064
:101CC0003091B50422B78091B5043817C9F7932F26
:101CD00080E030E0282B392BC901089529E28202E7
:101CE00090011124359527953595279587FD815CC1
:101CF00086FB880F880B80F9992787FD9095281B14
:101D0000390BC9010895F8942091D10D3091D20D6D
:101D10007894C9010895482F50E09A01220F331F8B
:101D200063E0440F551F6A95E1F7240F351F2454D3
:101D30003E4FC901089590E09C01220F331F220FEE
:101D4000331F280F391F24503D4FC9010895AF920A
:101D5000BF92CF92DF92EF92FF920F931F93CF9398
:101D6000DF93C82E162FEA01F22ED02E57FF10C097
:101D700022FF02C08CE101C08FE09C2D981B892FAF
:101D8000612F4DE22F2D0E94B85AD095C195DF4F9B
:101D90002D2D2F218C2D612F4AE30E94B85A8F2DB3
:101DA00090E0B4E0AB2EB12CA822B922F2FE02C022
:101DB000E2E001C0E0E0CE016CE370E00E94166C4E
:101DC0009B01442737FD4095542F0F2D00618E2F26
:101DD0008C0D612FA2E0EA2E0E94265DA114B104B1
:101DE00011F0ECE101C0E1E1CE016CE370E00E9492
:101DF000166C9C01442737FD4095542F0D2D006132
:101E00008E2F8C0D612FF2E0EF2E0E94265DDF9168
:101E1000CF911F910F91FF90EF90DF90CF90BF90E7
:101E2000AF9008950F931F93062F122F206250E05A
:101E30000E945C5E17FD07C08091A30D602F46E7EE
:101E4000212F0E94B85A1F910F910895242F40917D
:101E500008010E94120F08950F93022F442319F4D2
:101E600045E357E020C04530A8F4E0918601F0E05A
:101E7000EE0FFF1FEE0FFF1F3197E40FF11DE8502B
:101E8000FB4F449150E0440F551F440F551F4156DE
:101E9000594F09C0453250F450E0440F551F440FCC
:101EA000551F4056594F24E00E947B5B0F910895C7
:101EB000FF920F931F93182FF62E022F442321F425
:101EC0004EE956E024E00EC08A5E4A3008F48550A0
:101ED0006F2D50E0202F0E945C5E812F6F2D4BE90B
:101EE00056E022E00E947B5B1F910F91FF900895C6
:101EF0000F931F93DF93CF9300D0CDB7DEB7382F6A
:101F0000162F942F022F442329F0463139F04A3EF0
:101F100081F408C08A5F47E956E007C08A5F43E959
:101F200056E003C08A5F4FE856E0202F0E94BA5B5C
:101F300028C04095441F4427441F81E2841B482F3A
:101F4000832F39839A830E94B85A3981832F8A5FFD
:101F50009A81E92FFF27E7FDF095F7FF03C0F09581
:101F6000E195FF4FFF27E7FDF0953197AF01440F53
:101F7000551F4E0F5F1F415B594F612F23E00E9499
:101F80007B5B0F900F90CF91DF911F910F91089580
:101F90008FE496E00895DF92EF92FF920F931F93E4
:101FA000D82EE62EF42E1091AD01E12FFF27E7FD8C
:101FB000F095F7FF03C0F095E195FF4FE031A4F4F1
:101FC00083E0E802F0011124E25EF94F8D2D6E2DC1
:101FD000AF0123E00F2D0E947B5B1F3F3CF58D2D51
:101FE00086506E2D41E21FC08D2D8650E53264F47F
:101FF00011161CF4412F4F5002C0412F415F6E2D2E
:102000002F2D0E94780F12C011161CF4412F44523C
:1020100002C0412F4C5D6E2D2F2D0E94780F8D2D0B
:102020008E5E6E2D4DE62F2D0E94B85A1F910F9196
:10203000FF90EF90DF9008958C3038F4E82FF0E0B7
:10204000EE0FFF1FE651FB4F2AC0803198F4E82FB6
:10205000F0E0DF01AA0FBB1FA457BB4FEE0FFF1F1D
:10206000E45AFE4F2D913C91119780819181281B5C
:10207000390B0AC0843158F4E82FF0E0EE0FFF1F4F
:10208000E457FB4F20813181220F331F0DC0843272
:1020900048F4E82FF0E0EE0FFF1FE053FB4F2081E4
:1020A000318102C020E030E0C9010895AF92BF92B3
:1020B000DF92EF92FF920F931F93DF93CF9300D0A5
:1020C000CDB7DEB7F82E463008F0DEC0882309F41D
:1020D000DEC0863119F08A3E19F4D6C061E0D7C05F
:1020E000992787FD90959C0197FF04C022273327ED
:1020F000281B390B2A307CF41F144CF02DE030E003
:10210000A901481B590BCA010E94C65FBAC00D96AF
:102110000E94C65FBBC02A50A22EBB249501220F8D
:10212000331F2A0D3B1D2E553E4FF901E85AFD4F36
:102130005081552309F4A8C0453029F4F501E05831
:10214000FB4F80819CC0F901EA5AFD4FD080295A8B
:102150003D4FF901E080553008F4A6C0583060F0DA
:102160008D2D81504A8359830E941C108C018E2D25
:1021700081500E941C10A2C020E030E000E010E07E
:10218000583088F4553088F5523009F462C0533025
:1021900020F4513009F06EC057C05330D1F05430A4
:1021A00009F068C01CC05A3009F44EC05B3038F4E6
:1021B000583009F43FC0593009F05CC040C05C3071
:1021C00009F44CC05C3008F444C05D3009F052C0E2
:1021D0004AC017FF39C0109501951F4F35C017FF32
:1021E00038C0109501951F4F34C0142F1F5F8D2DDF
:1021F00060E0412F0E945610082F8E2D60E0412F85
:102200000E945610F501EE0FFF1FEA0DFB1DE65070
:10221000FC4F9081953029F4002361F1882341F52A
:102220002AC0963029F4002319F5882319F120C01B
:10223000802721C081E002171307E1F41CC081E070
:1022400002171307C1F416C081E0201731079CF074
:1022500011C081E00217130774F00CC081E002176F
:1022600013074CF407C081E02017310724F402C0A3
:1022700081E001C080E0F501E058FB4F80831F142E
:102280002CF061E0682703C060E001C0682F862F52
:102290000F900F90CF91DF911F910F91FF90EF90D2
:1022A000DF90BF90AF9008958D2D81504A83598360
:1022B0000E941C108C018E2D0E946E0E9C014A8182
:1022C00059815ECF86B380958E7708950E94621102
:1022D0008823E1F70E94355F08958091730160E0E3
:1022E00040E00E945610882331F480919D04909123
:1022F0009E04009711F0C79A0895C79808950F9308
:102300001F93CF93DF93EC018B010E944E5A82E220
:1023100060E049E056E024E00E94BA5B80E2BE0142
:102320000E94E15B88E2B8010E94E15B80E363EF19
:1023300075E00E94E15B0E94C65E809170010E9480
:10234000BC5E0E946611DF91CF911F910F9108959D
:102350000F93AB0160E123E000E00E947B5B0F91F3
:102360000895DF92EF92FF920F931F93CF93DF9325
:102370008091850181FD83C088E895E062E775E082
:102380000E947F1190919D01892F887341F08831BF
:1023900031F0883221F0803311F0883329F4892F0D
:1023A000877C886080939D0100E010E065E1E62E67
:1023B000F12C08C0C701801B91090E94C65F110F54
:1023C000182B0F5F0830B0F3D0909D01D12680E02C
:1023D00060E14BE555E026E100E00E947B5BCD2DFE
:1023E000D0E0CE0180FF05C082E06FE476E00E947D
:1023F000A811C1FF05C087E162E576E00E94A8113F
:10240000C2FF05C08CE265E576E00E94A811CE010E
:10241000887390700097B1F0012F13FF05C081E41D
:1024200068E576E00E94A81104FF05C081E46BE531
:1024300076E00E94A81105FF05C081E46EE576E014
:102440000E94A811C6FF05C086E561E676E00E94FD
:10245000A811D7FE05C08BE664E676E00E94A811BD
:102460000E94C65E80919D01181749F00E9462117A
:10247000882329F40E946D1100E010E09BCFDF91CA
:10248000CF911F910F91FF90EF90DF9008951F93D0
:10249000CF93DF930E94621120E030E011E0482FDB
:1024A00050E02F5F3F4FBA01022E02C0759567952D
:1024B0000A94E2F760FD03C01F5F183091F71150D6
:1024C000163030F5812F0E94CC54882309F11093E7
:1024D0006F01812F0E94D05481E00E949C550E9480
:1024E0004E5A86E160E043E555E024E00E94BA5B85
:1024F000C2EAD1E01AE04991812F68E124E00E940C
:10250000B85A155F1837B9F70E94C65E0E94661167
:10251000DF91CF911F910895CF93DF93EC010E943B
:102520004E5A82E260E04BE455E024E00E94BA5B40
:1025300088E1BE010E94E15B0E94C65E809170014D
:102540000E94BC5EDF91CF9108951F93CF93DF93DC
:10255000EC01162F0E944E5A82E260E045E455E0FD
:1025600024E00E94BA5B88E1BE010E94E15B8CE13D
:1025700068E347E355E00E94E95B0E94C65E1123D1
:1025800019F48091700101C089E10E94BC5E82E172
:102590000E94D06B0E9466110E9462118823C9F4C8
:1025A0008091650E833019F4A8951092650E809184
:1025B000730160E040E00E945610882331F480915E
:1025C0008A01882311F4112311F0C79AE5CFC79827
:1025D000E3CFDF91CF911F91089580917F048823ED
:1025E00051F087E995E060E00E94A51280917F0498
:1025F0008E7F80937F0408958091850187FD07C0B9
:10260000887329F482EC95E060E00E94A512089599
:102610008091850182FD0AC00E94BD56883C9105CB
:1026200028F48FE096E060E00E94A5120895EF92F2
:10263000FF92CF93DF93A82FAF70A6509091B40173
:10264000923074F0292F332727FD309521503040E8
:10265000C1E0D0E002C0CC0FDD1F2A95E2F79C2F2D
:10266000A83008F09CC06A2F659570E0FB01EE0F62
:10267000FF1FE050FF4F0190F081E02DB0819923C2
:1026800079F4CB2FDD27C7FDD095D7FF03C0D095B8
:10269000C195DF4F9C2FC7FD9D5F959595959F5FD9
:1026A0004091860150E04170507022E030E0241BE0
:1026B000350B2617370769F42091B3012F7009F401
:1026C00073C021E094E03091880130FF03C0919500
:1026D00001C020E04B2F552747FD5095C92FDD271E
:1026E000C7FDD095A0FF03C0C40FD51F04C0BA0119
:1026F0006C1B7D0BEB01209729F07E019F2D9B2702
:1027000097FF0BC0222349F4BB2339F010820E94AB
:10271000256086E10E94D06B41C0CE0184589F4F56
:10272000893F9105B8F4C08386E00E949C55CE0194
:1027300083589F4F8B3F910588F5D7FF03C0D095F5
:10274000C195DF4FD595C795D595C795BE01645CFA
:10275000462F1FC01C161D0614F48DE701C083E828
:10276000808386E00E949C55CE0183589F4F8B3F0B
:102770009105A0F4CE01D7FF03C0909581959F4F9E
:1027800064E070E00E94166C709561957F4F462F53
:10279000445C87E494E065E10E945D6A80E0DF913B
:1027A000CF91FF90EF90089520E08DCF8F929F9270
:1027B000AF92BF92CF92DF92EF92FF920F931F934F
:1027C000CF93DF93182FEB015A016901802E84FF0C
:1027D00006C01F70106694E0992E05E003C085E0E6
:1027E000982E04E0802F8066181761F0802F806497
:1027F000181741F080911905882369F0133611F0FC
:10280000133449F47E010894E11CF11C83E10E9419
:10281000D06B892D18C0992D9066191761F0992DEC
:102820009064191741F0882309F474C0123619F026
:10283000123409F06FC07E010894E108F10884E1C8
:102840000E94D06B802F90E00E94C65F882351F0D9
:10285000EE24FF24EC1AFD0A892D0E942560802FAA
:102860000E942560A114B10491F481E0C816D1043E
:1028700071F4103661F41092190501E0E02EF12C8C
:10288000209711F0EE24FF2480E60E94256020911D
:102890009A0430919B04E21AF30ACE14DF0444F444
:1028A000812F0E94256083E10E94D06B76010AC0CF
:1028B000EA14FB043CF4812F0E94256084E10E940D
:1028C000D06B7501EC16FD06A9F0E114F10451F48A
:1028D000812F0E941660D7FF02C083E101C084E10E
:1028E0000E94D06B882D83700E949C5581E080935C
:1028F000970402C010929704C701DF91CF911F91F6
:102900000F91FF90EF90DF90CF90BF90AF909F908E
:102910008F9008957E01A6CF0F93772767FD70955E
:10292000552747FD5095332727FD30950E94D61334
:102930000F9108950F93772767FD7095552747FDF1
:102940005095332727FD309502E00E94D6130F9152
:1029500008950F93772767FD7095552747FD50958C
:10296000332727FD309501E00E94D6130F9108957B
:10297000E0919604F0E0EE0FFF1FE257FB4F8081DD
:102980009181089590919604992319F4882331F444
:1029900018C0882319F4892F815001C080E08093EA
:1029A000960487E10E94D06BE0919604F0E0EE0F70
:1029B000FF1FE457FB4F0190F081E02D8EEB09954E
:1029C000089583E295E060E00E94A5120895FC015D
:1029D000A0919604B0E0AA0FBB1FA457BB4F8D93E4
:1029E0009C938FEB099587E10E94D06B0895CF935C
:1029F000DF93EC0180919604982F9F5F909396044B
:102A0000953040F08093960480E195E060E00E946C
:102A1000A5120FC087E10E94D06BE0919604F0E010
:102A2000EE0FFF1FE457FB4FD183C0838FEBFE01F6
:102A30000995DF91CF9108951092A1041092A304FB
:102A40001092A2041092A004089520919D04309148
:102A50009E042115310531F02150304030939E0401
:102A600020939D04882369F040918A0150E084EF0F
:102A700091E0489F9001499F300D589F300D1124DF
:102A800002C020E030E080919F04882369F06091CB
:102A9000920170E044EF51E0649FC001659F900D8A
:102AA000749F900D112402C080E090E040919D043D
:102AB00050919E044217530720F430939E042093B4
:102AC0009D0420919D0430919E042817390720F41D
:102AD00090939E0480939D040E946D1108950E941E
:102AE000830E41E02091E8043091E90482179307B6
:102AF00009F440E040939C040E94830E9093E90403
:102B00008093E8048EE195E060E00E94E4338091D8
:102B10009C04882371F080E00E94AA550E944E5ABE
:102B200010929B0410929A0480E00E94CE1E0E9494
:102B3000C65E0895E82FF0E0E85FFA4FE491F0E018
:102B4000EE0FFF1FE854FB4F20813181C90108952A
:102B5000CF92DF92EF92FF920F931F93DF93CF9369
:102B60000F92CDB7DEB720E0CC24DD24822F29835D
:102B70000E949A15092F10E0C00ED11E29812F5FE7
:102B80002430A1F7C6010F90CF91DF911F910F91D3
:102B9000FF90EF90DF90CF900895A8EBB4E0E8ECC1
:102BA000F4E060E0862F806487B9369A40895189C5
:102BB0008D919C91119796958795840F951F8E7F87
:102BC00011969C938E9320813181C901840F951FAA
:102BD00096958795918B808B349BFECF349A84B1E8
:102BE00095B1820F931F96958795819391936F5F0F
:102BF00012966830B9F60895EF92FF920F931F93E3
:102C0000CF93DF938091880184FD44C00E946D11B1
:102C10000E944E5A80E060E045ED50E020E000E088
:102C20000E94595A80918E0184FD08C080E068E3BB
:102C300043E951E02AE000E10E947B5B0E94C65E0E
:102C4000809170010E94BC5E0E94661100E20E94A9
:102C5000CD150150E1F70E94A8158C010E94830E4A
:102C6000EC01C057DE4F0DC00E94CD150E94A81583
:102C70007C010E946211882369F4E016F10651F488
:102C800006C00E94830EC817D90771F703C00E94BF
:102C90006D11F7CFDF91CF911F910F91FF90EF90C2
:102CA0000895E8EBF4E040E012C067B9369A349B2F
:102CB000FECF349A24B135B1820F931F5150A9F73A
:102CC00096958795819391934F5F483031F054E00A
:102CD00080E090E0642F6064E8CF0895E8EBF4E0D2
:102CE00020E0822F806487B9369A349BFECF349AD5
:102CF00084B195B1880F991F819391932F5F2830EC
:102D000081F70895FF920F931F93CF93DF938091E4
:102D1000850180FD3AC08091860190E081709070BD
:102D200002E010E0081B190BF801EE0FFF1FEE5B2D
:102D3000FE4FC181D281609687859089C81BD90BCF
:102D40000E946E16F02E802F0E949A15C817D90780
:102D5000E4F40E9462118823C1F40DC00E946E1633
:102D60008F2D0E949A15C817D9077CF40E94621112
:102D7000882341F00AC081EE95E062ED75E00E9483
:102D80007F11ECCF0E946D11E9CFDF91CF911F91A0
:102D90000F91FF9008958EE587B9369A349BFECF48
:102DA000349A84B195B104964091090150910A0179
:102DB0009A0163E0220F331F6A95E1F7241B350B5C
:102DC000820F931F23E0969587952A95E1F79093BC
:102DD0000A0180930901089578941F920F920FB60B
:102DE0000F9211248F938091B5048F5F8093B50467
:102DF0008F910F900FBE0F901F90189578941F928F
:102E00000F920FB60F9211242F933F934F935F931E
:102E10006F937F938F939F93AF93BF93EF93FF93A2
:102E2000F89487B78D7F87BF789481B78E5F81BF15
:102E30009091490480914B04882379F0809191010D
:102E4000882349F0813051F48091730E890F80936B
:102E5000730E87FF02C01B9A01C01B9880910B0163
:102E6000982F915090930B01882371F48DE48093F7
:102E70000B0187E494E00E9470690E9436608091A3
:102E8000650E82608093650EF89487B7826087BF75
:102E90007894FF91EF91BF91AF919F918F917F9126
:102EA0006F915F914F913F912F910F900FBE0F90B7
:102EB0001F90189578941F920F920FB60F921124BD
:102EC0001F932F933F934F935F936F937F938F93B2
:102ED0009F93AF93BF93EF93FF9320918000309126
:102EE0008100F89480917D008F7D80937D0078949F
:102EF0008091B6049091B704A901481B590BCA01EF
:102F0000969587953093B7042093B6041091B40436
:102F1000212F2150283058F59C012152334055E093
:102F20002737350708F5E12FF0E0EE0FFF1FEE55CC
:102F3000FB4FAC014C5D554020918C01332727FDA0
:102F40003095265F3F4F429FC001439F900D529F97
:102F5000900D11246AE070E00E94166C718360830A
:102F60001F5F1093B4040CC01092B40409C0815ABE
:102F70009F402EE28F3D920718F481E08093B404C5
:102F8000F89480917D00806280937D007894FF9119
:102F9000EF91BF91AF919F918F917F916F915F91D1
:102FA0004F913F912F911F910F900FBE0F901F9047
:102FB0001895E5E7FEE09F0181918535E1F32457FF
:102FC0003E40C9010895CF93DF930E94600EEC014B
:102FD00080918901813019F40E94CD1507C082309B
:102FE00019F40E94511602C00E946E168EE587B930
:102FF0000E946F150E94CB168091650E833019F4E4
:10300000A8951092650E0E94600E8C1B9D0B20915E
:10301000C1063091C2062817390720F49093C206E2
:103020008093C106DF91CF9108958FEF8ABB1BBAC1
:1030300091E897BB9EE798BB9EE394BB91EC95BB50
:1030400011BA82BB88E082B987EF83B91092610020
:103050001092620084E1809364008BEF809365009E
:103060000E94865E80E487B985E886B987E083BFE1
:103070008CE981BF87B7836087BF1FBC8AE08EBDA4
:1030800010928B0082E880938A0080917D0080629C
:1030900080937D00EDB7FEB7329785E502C080834F
:1030A00031979EE0E437F90709F0C8F7789482EC8D
:1030B0009DE390938D0480938C048EE29EE10E94A8
:1030C000F71489E10E94BC5E0E9455558091700101
:1030D0000E94BC5EC79A80E00E94355F80EF90E05E
:1030E00090930A01809309010E94C7672DE088E14F
:1030F00090E00FB6F894A89581BD0FBE21BD8EE17A
:1031000095E060E00E94E433809170010E94BC5E13
:1031100080ED97E09BBD8ABD80E186BF87B7806167
:1031200087BF0E94E317FDCF87E494E00E945969AE
:10313000089529E28202900111243595279535954D
:10314000279587FD815C86FB880F880B80F999277E
:1031500087FD9095281B390BC90108959C01E5E076
:1031600035952795EA95E1F7AC01440F452F441FAB
:10317000550B280F391F892F990F990B8595280F0B
:10318000391F241B350BC9010895F8942091D10DE6
:103190003091D20D7894C9010895CF92DF92EF92C9
:1031A000FF920F931F93D82EC62E142F042F06952F
:1031B000E82EE01AF62EF01A8E2D6F2D0E946B5C11
:1031C000602F6C0D8E2D412F0E94675C802F8D0D1E
:1031D0006F2D412F0E946B5C8E2D6F2D412F0E9411
:1031E000675C1F910F91FF90EF90DF90CF90089553
:1031F000AC0180E060E021E00E94BA5B08950F938B
:103200001F93CF93DF93182F8BE198E00E94F8185B
:10321000113658F0133628F0133639F48AE999E15B
:1032200002C082EC9DE30E94E71486E068E043E17F
:1032300058E00E94E95B4091390650913A068AE2D3
:1032400068E020E000E00E94A70E40913B0650910C
:103250003C068EE468E020E00E94A70E86E060E174
:103260004BE058E00E94E95B40913D0650913E06DC
:103270008AE260E120E00E94A70E40913F06509153
:103280004006F4E056954795FA95E1F78EE460E143
:1032900020E00E94A70E86E660E047E058E00E942A
:1032A000E95B40913706509138068EE460E020E0FB
:1032B0000E94A70E8091BD069091BE0689379105A8
:1032C00028F08091BC06C82FD0E002C0C0E0D0E05A
:1032D00082E06CE34EE70E94675C85E06CE143E2CC
:1032E0000E946B5C1BE0812F6BE343E00E946B5CF0
:1032F0001A5F1338C1F716E00CE3FE01EC5BF94FDF
:103300004081602F641B812F0E946B5C2196C8371F
:10331000D10510F0C0E0D0E02091BC0630E0C2172B
:10332000D30719F01F5F1E3741F7DF91CF911F912F
:103330000F9108951F93182F80E798E00E94F818C6
:103340001236E1F0133628F4103631F01136E9F474
:1033500018C01336D1F415C08FEF97E090930D018C
:1033600080930C011092C0061092BF061092C20604
:103370001092C10687E10E94D06B07C08FEF98E1E1
:1033800002C082EC9DE30E94E71488E061E678E0E9
:103390000E94E15B4091BF065091C006569547954B
:1033A00084E568E00E946C5E80E162E578E00E945E
:1033B000E15B40910C0150910D015695479584E5D4
:1033C00060E10E946C5E88E163E478E00E94E15B6A
:1033D0004091BF065091C00680910C0190910D0163
:1033E000481B590B5695479584E568E10E946C5E31
:1033F00080E26AE378E00E94E15B2091C1063091AF
:10340000C20684E690E0289FA001299F500D389FB6
:10341000500D1124A4E056954795AA95E1F784E54F
:1034200060E220E30E945C5E88E262E378E00E9452
:10343000E15B0E94D917AC018FE368E20E94ED5B6B
:1034400082E168E340E258E00E94E95B1F91089541
:103450008AEE9FE00895442319F044EF54E002C03F
:1034600040EF54E091E0222309F490E0292F0E94DC
:10347000BA5B08950F93942F01E0222309F400E032
:1034800042EE5FE0292F0E94A55B0F910895FF9205
:103490000F931F93F82E062F142F80E860E0402F23
:1034A00050E0212F0E945C5E0A3010F00FE601C050
:1034B00005E7802F60E04FE2212F0E94B85A4F2D80
:1034C00050E04F5F5F4F802F60E0212F0E945C5ED5
:1034D0001F910F91FF9008956F927F928F929F920C
:1034E000AF92CF92DF92EF92FF920F931F93CF9301
:1034F000DF93EC01162FD42E4901E091F204F091F4
:10350000F3046090F4047090F5048091C2089091E7
:10351000C3088E1B9F0B20E430E0B9010E94166C9B
:10352000462F60931C058091C0089091C1088619B0
:103530009709B9010E94166C862F60931D054423DC
:1035400021F0F093C308E093C208882321F0709221
:10355000C1086092C00880911B05882321F48091E6
:10356000880185FF06C010921C0510921D0510925F
:103570001B0560911C05662351F480911D0588236D
:1035800031F480919A0490919B04009781F04091CE
:103590008A0150E024EF31E0429FC001439F900D2B
:1035A000529F900D112490939E0480939D0481144A
:1035B000910409F456C08881882309F04BC0662322
:1035C00031F180911905882311F5ED2DE61BE7FDFA
:1035D000E0E0202F30E08E2F992787FD909582170D
:1035E000930714F0E02FE150FF27E7FDF0958D2DB4
:1035F00090E0E817F90749F0EE0FFF1FE80DF91DFD
:1036000025913491C9010E94E71410921C051536CA
:1036100041F4DD2011F0ED2D01C0E02FF0E03197F5
:103620000FC01436C9F42D2D30E0802F90E00197A3
:10363000281739071CF4ED2DEF5F01C0E0E0F0E042
:10364000EE0FFF1FE80DF91D25913491C9010E946D
:10365000E71402C040E001C041E08D2D602F0E94C0
:10366000471AE114F10451F098818C2D9C1508F44F
:10367000892FF701E80FF11D549101C050E08091AE
:103680001905882309F04FC080911D05882329F171
:103690004881481B47FD40E0242F332727FD309504
:1036A0008A2D90E0281739070CF04A2D488389812C
:1036B000E114F10459F0C41608F44C2DF701E40F9D
:1036C000F11DE4918E1718F4E82F01C0E0E0E983C2
:1036D00080E68093D30D10921D058881882319F10F
:1036E00090911C059923F9F04981E114F104B1F09E
:1036F000491B47FD40E09C2D8C1508F4982FF701DD
:10370000E90FF11DE491242F332727FD30958E2FEB
:1037100090E0281739071CF04E2F01C040E0498384
:1037200080E68093D30D103651F1113690F41334A6
:1037300009F480C0143430F4113279F1123409F0F4
:103740009CC06AC0143409F43FC0153409F095C018
:103750004FC01436E9F1153638F4123609F45FC05B
:10376000133609F08AC069C01138A1F01F3B21F05F
:10377000153609F082C040C01982188212C0552344
:1037800009F47BC081E090911905911180E080934C
:10379000190573C0109219050DC080911905882371
:1037A00019F01092190569C08881882319F08114D5
:1037B000910421F480E00E94C2145FC087E10E945E
:1037C000D06B1982188256C08981851709F455C0BB
:1037D000E114F10409F451C080911905882309F01E
:1037E0004CC08981851710F48F5F12C0198242C0C6
:1037F0008981882309F441C0E114F10409F43DC032
:10380000809119058823C9F58981882319F0815091
:10381000898330C059832EC088818A1571F18091C7
:103820001905882351F588818A1510F48F5F0DC022
:1038300018820EC08881882301F1809119058823A0
:10384000E1F48881882319F08150888301C0A8821F
:103850008981E114F10461F098819C1508F4C92E66
:10386000EC0CF11CF7019491891718F4982F01C002
:1038700090E0998380E68093D30DDF91CF911F91E3
:103880000F91FF90EF90DF90CF90AF909F908F902F
:103890007F906F9008954F925F926F927F928F9278
:1038A0009F92AF92BF92CF92DF92EF92FF920F93CF
:1038B0001F93DF93CF930F92CDB7DEB7D82E80E65C
:1038C0009AE00E94F81884E498E06D2D41E026EE1D
:1038D00037E006E0A8E6EA2EAAE0FA2EF5E0CF2EC1
:1038E000E6E0AE2E0E946C1A809044089090450845
:1038F0008091630081FF07C08AE268E14AE55AE0EF
:103900000E94E95B52C182E168E04BE45AE00E9408
:10391000E95B8A9480911905882319F072E0C72E1B
:1039200002C0CC24C394EE24FF2410E1A82CBB24B5
:10393000A7FCB09464E0662E712C2701440C551C42
:103940008CE791E0480E591E4E2D4F5F80E0612FAD
:1039500020E00E942C0FAE14BF0411F491E09110EE
:1039600090E0F201218122952695269523709923D6
:1039700011F400E001C00C2D88E1612F40E45AE011
:1039800099830E94A55B99819923C1F080911905C3
:103990008823A1F0F2016181629566956695637056
:1039A0008D2D40E022E00E94A9148295880F880F97
:1039B000807CF20191819F73982B9183AE14BF0498
:1039C00021F401E0F92DF13009F000E0F2018181EC
:1039D000880F880F85958595FDE08F02C001112421
:1039E000B3010E94166CAB01002311F420E001C06A
:1039F0002C2D82E4612F0E945C5E0023A9F080914F
:103A00001905882389F0F2016181660F660F6595BB
:103A100065958D2D41EE2FE10E94A9148F73F2015F
:103A20009181907C982B9183AE14BF0421F491E096
:103A3000F92DF23009F090E0F201208127709923EE
:103A400011F400E001C00C2D88E4612F42E35AE03C
:103A500099830E94A55B9981992391F08091190522
:103A6000882371F0F201608167708D2D40E023E0C2
:103A70000E94A9148770F2019081987F982B9083FF
:103A8000AE14BF0421F401E0F92DF33009F000E099
:103A9000F2014081459545954595002311F420E0BC
:103AA00001C02C2D8AE5612F0E94780F0023B1F010
:103AB00080911905882391F0F201608165956595E3
:103AC00065958D2D4AEE26E10E94A914880F880F76
:103AD000880FF20190819770982B9083185F08945B
:103AE000E11CF11C103309F028CF80E367E27AE093
:103AF0000E94E15B40918C01552747FD5095465F40
:103B00005F4FF82DF43011F421E201C020E28EE481
:103B100060E30E945C5E282D243049F48D2D609175
:103B20008C0146EF28E20E94A91480938C01EE24B8
:103B3000E394882D853009F0EE2480E068E343E2C9
:103B40005AE02E2D0E94BA5B44EAA42E44E0B42E23
:103B500004E711E090E3F501419151915F01F80113
:103B6000219131918F01421B530B440F551F892F17
:103B700068E320E299830E945C5E9981985E9039A7
:103B800051F7EE2091F0FD2DF03679F4A4E7B1E085
:103B9000E4EAF4E088E001900D928150E1F781E0E1
:103BA0000E949C5587E10E94D06B0F90CF91DF91CE
:103BB0001F910F91FF90EF90DF90CF90BF90AF904B
:103BC0009F908F907F906F905F904F900895AF92ED
:103BD000CF92EF92FF920F93AE2CEE24FF24CC24D1
:103BE0000E946C1A0F91FF90EF90CF90AF900895C4
:103BF000EF920F93DF93CF930F92CDB7DEB7682F7D
:103C00008EE69AE069830E94F81886E498E069815C
:103C100042E026EE37E006E0EE240E94E71D80E158
:103C20006DE677E00E94E15B88E16AE377E00E945D
:103C3000E15B80E26DE477E00E94E15B88E26EE5A3
:103C400077E00E94E15B80E36DE777E00E94E15B53
:103C50000F90CF91DF910F91EF900895CF92DF9267
:103C6000EF92FF920F931F93DF93CF9300D0CDB7C6
:103C7000DEB7682F8DE99AE069830E94F81888E41E
:103C800098E0698143E026EE37E006E0EE240E94EA
:103C9000E71D9EE0C92ED12C00E010E0143020F08A
:103CA00088EFF82EF00E01C0F02EC6010E94C65F0C
:103CB000E82E1F5F8AE26F2D412F20E00E94780FCF
:103CC0004E2D405D84E46F2D2E2D0E94B85A085F62
:103CD0000894C11CD11C193009F708E3CC24DD2459
:103CE00010E0812F90E00E94C65FF82EA601425896
:103CF000554F80E0602F25E00E94B45B4F2D405D62
:103D000080E2602F2F2D0E94B85A1F5F85E090E05F
:103D1000C80ED91E0850163021F784E568E146E741
:103D20005AE027E00E94B45BB6E0EB2EF12C10E2E3
:103D300030E084E5612F47E857E0232F00E03A8325
:103D40000E94595AC7010E94C65F282FC7010196D9
:103D500029830E94C65F082F2981422F405D8CE68F
:103D6000612F0E94B85A402F405D88E7612F202FB5
:103D70000E94B85A3A813F5F185FE2E0F0E0EE0E31
:103D8000FF1E3430B1F60F900F90CF91DF911F914D
:103D90000F91FF90EF90DF90CF9008958F929F92B8
:103DA000AF92BF92DF92EF92FF920F931F93CF9348
:103DB000DF93D82E85EA9AE00E94F8188AE498E00A
:103DC0006D2D44E026EE37E006E0EE24E3940E94F9
:103DD000E71DF0904A08CAEED4E010E000E0812C24
:103DE00024E0922EA12CB12C88E1612F41E40E94A5
:103DF000775B402F4F5C8EE1612F0E94775B802FB5
:103E00000E949A15AC018AE2612F0E94ED5B073097
:103E1000B1F068817981882777FD8095982F24E615
:103E200030E040E050E00E94D76BA50194010E9471
:103E30004B6C8AE5612FA9010E946C5E0AC08F2D30
:103E4000813011F040E201C041E28AE5612F0E9419
:103E5000260F0F5F185F2296083031F68CE668E275
:103E600042EA5AE022E00E94B45B4091090150917D
:103E70000A0188E760E320E00E945C5E8F2D8130BC
:103E800059F4F0921B058D2D6091720141E82FE7E6
:103E90000E94A91480937201DF91CF911F910F911D
:103EA000FF90EF90DF90BF90AF909F908F9008951C
:103EB000EF920F93E42E40E020E030E000E00E941B
:103EC000E71D0F91EF900895CF92DF92EF92FF924E
:103ED0000F931F93CF93DF938AE26CE247E10E9436
:103EE000CD1886E56CE247E10E94CD188AE26BE2CC
:103EF00043E00E946B5C89E26CE243E00E94675CF5
:103F000086E56BE243E00E946B5C85E56CE243E092
:103F10000E94675C8091EA049091EB04C1E7D0E0D5
:103F2000BE010E94166C262F8091EC049091ED0446
:103F30000FE81FEFB8010E94166C645D822F865D4A
:103F400045E00E94CD188091F0049091F104BE01EB
:103F50000E94166C262F8091EE049091EF04B80118
:103F60000E94166C645D822F8A5A45E00E94CD182B
:103F7000C2EFD4E04AE3F42E0DE510E038E3E32E7F
:103F80008991999180509C4FB8010E94166CD62E51
:103F9000D394CE2CCD188F2D6C2D4D2D0E946B5CA3
:103FA0008F2D8F5F6C2D4D2D0E946B5C8F2D8E5F42
:103FB0006C2D4D2D0E946B5C85E0F80E8F2D8934A1
:103FC000F9F6DF91CF911F910F91FF90EF90DF9065
:103FD000CF9008954F925F926F927F928F929F92AF
:103FE000AF92BF92CF92DF92EF92FF920F931F9307
:103FF000DF93CF930F92CDB7DEB7B82E8AEF9AE05A
:104000000E94F81887E798E06B2D45E026EE37E030
:1040100006E0EE24E3940E94E71D10927708BBE5CA
:10402000EB2EB8E0FB2EADE4CA2EA8E0DA2E860116
:10403000470160E0862F69830E949A15D4014D9153
:104040005C911197282F392F6981421753070CF47F
:104050009A01F401219331934F01D8014D915C9164
:104060001197282F392F241735070CF49A01F801DE
:10407000219331938F016F5F6730E1F680914C0897
:1040800080931B05FB2DF03219F0FF3B71F40BC040
:104090008F5F80934C08833041F487E10E94D06B9E
:1040A00081E00E949C5510924C0880914C08813010
:1040B000B1F0813020F0823009F0A4C03FC08CE024
:1040C00060E148EE5AE021E100E00E947B5B82E182
:1040D00068E148ED5AE02FE00E947B5B93C08EE1DF
:1040E00060E14BEC5AE02CE000E00E947B5B82E157
:1040F00068E149EA5AE020E10E947B5BF9E68F2EF5
:10410000F8E09F2E20E008E91AE3E8E6AE2EE5ECA1
:10411000BE2ED7010D931D937D01F601A192B192A0
:104120006F01822F29830E949A15D4018D939D934C
:104130004D0129812F5F273061F764C082E160E182
:104140004AEB5AE020E100E00E947B5B82E168E1FB
:1041500049EA5AE020E10E947B5B79E6A72E78E0ED
:10416000B72E63E4462E61E0562EF20150E4852E10
:10417000912CD7018D919D917D01D6016D907D90FF
:104180006D019C012619370937FF03C03095219531
:104190003F4F23333105DCF0D5012D913C91318324
:1041A00020838901081B190BC801B4010E94166CF9
:1041B000061B170B17870687C301821B930B9C01F5
:1041C000B4010E94166C261B370B358F248FA2E09A
:1041D000B0E0AA0EBB1E3296B9E6EB16B8E0FB06BD
:1041E00041F680E090E0F201219131912F01820FA0
:1041F000931FFBE54F16F1E05F06A9F790936E0160
:1042000080936D010E94641F0F90CF91DF911F91E9
:104210000F91FF90EF90DF90CF90BF90AF909F9065
:104220008F907F906F905F904F900895282F30E08F
:10423000C901880F991FA90163E0440F551F6A95B2
:10424000E1F7840F951FA9014F5F5F4FBA01660F19
:10425000771FA3E0440F551FAA95E1F7640F751F60
:1042600064547E4F20953095205E3F4FA901440F46
:10427000551FE3E0220F331FEA95E1F7420F531F6A
:1042800084549E4F0E947B6C8AE0E2EFF2E0DF01F3
:104290001D928A95E9F782E00E949C550E9438564B
:1042A00008950F931F93CF93DF93282F30E0E901F8
:1042B000CC0FDD1FC90113E0880F991F1A95E1F794
:1042C000C80FD91F8E0104541E4FA9014F5F5F4FC5
:1042D000CA01880F991FA3E0440F551FAA95E1F763
:1042E000840F951F20953095205E3F4FA901440F04
:1042F000551FE3E0220F331FEA95E1F7420F531FEA
:1043000084549E4FB8010E947B6C8AE0D8011D92B4
:104310008A95E9F780919B08CE55DE4F8A8F8B8F67
:1043200084E68C8F82E00E949C550E943856DF9173
:10433000CF911F910F910895FF920F931F9385EFD7
:10434000EEE3F5E0DF011D928A95E9F780913306EF
:10435000ACEBB1E050E021E030E060E07C9177230D
:1043600011F0472F01C040E1641738F5F22E032FFA
:10437000162F1F5F802F90E0FC01EE0FFF1FEE0F46
:10438000FF1FE80FF91FE25CFA4F912F9F738081A6
:10439000807C892B80648083F182F39453830F5F48
:1043A000141738F3962F9095642F822F8F5F890F03
:1043B000390F340F290F240F840F772359F1832FDE
:1043C00090E0FC01EE0FFF1FEE0FFF1FE80FF91F3B
:1043D000E25CFA4F4F738081807C5483842B806829
:1043E000808322832F5F1A968C911A97781719F47D
:1043F0001182138205C021832F5F852F8F5F8383F6
:10440000822F5F5F1A96503219F42093330604C04E
:104410003F5FA4CF809333061F910F91FF900895C3
:104420001F93182F88E06BEE7DE00E94E15B82E134
:1044300068E244EE5DE00E94E95B82E160E345ED05
:104440005DE00E94E95B113679F01F3B19F01036F0
:10445000A9F404C080E00E94D06B10C080913406A3
:104460000E9416210E949C21812F0E94256081E0DC
:104470000E94C2148EE093E20E94F7141F910895E7
:10448000ECEBF1E080E090819150903108F48F5F87
:104490003A9692E0EC3FF907B1F708951F93182F71
:1044A00080E16DE07EE00E94E15B0E944022482FA7
:1044B00088E760E150E020E00E945C5E80E267EF08
:1044C0007DE00E94E15B113651F481E60E94256097
:1044D00081E00E94C2148EE093E20E94F7141F91C3
:1044E00008950E944022803230F08EE492E20E94D1
:1044F000F71481E0089580E00895EF92FF920F9302
:104500001F93DF93CF9300D0CDB7DEB7182F813242
:1045100008F07BC0882319F4442341F476C080322C
:1045200019F4442331F071C0442319F0012F0F5FB7
:1045300002C0012F0150812F4A8369830E948B0E94
:104540007C01802F0E948B0EFC01D7018C91982F4B
:1045500091504A816981903108F057C02081213102
:1045600008F053C06623A1F10E947122882309F04C
:104570004CC0212F30E0A9014F5F5F4FCA01880F67
:10458000991F13E0440F551F1A95E1F7840F951FEB
:10459000B901660F771FA901A3E0440F551FAA9523
:1045A000E1F7640F751F64547E4F20953095205EAF
:1045B0003F4FA901440F551FE3E0220F331FEA9537
:1045C000E1F7420F531F84549E4F0E947B6C1DC025
:1045D000281759F0442331F08031B8F48F5FF70188
:1045E000808313C0D7019C9310C0D701CF010A96D6
:1045F00004C020813C9131932D93E817F907C9F746
:1046000082E00E949C550E9438560F900F90CF91E7
:10461000DF911F910F91FF90EF9008956F927F921D
:104620008F929F92AF92BF92CF92DF92EF92FF92C2
:104630000F931F93CF93DF93182F8FEC9DE00E9471
:10464000F818E0903306EA948EE998E0612F44E090
:1046500022ED37E00AE00E94E71DC0909E08CC20C2
:1046600011F410929D081236D9F1133670F41334F8
:10467000A9F1143420F4123409F070C031C010369E
:10468000C1F0113609F06AC045C0103809F452C0B3
:10469000113820F4133609F061C020C01E3BB9F177
:1046A0001F3B09F05BC081E080939C0810929D083D
:1046B0002EC01C143CF481E090919D08911180E083
:1046C00080939D0880919D0880939C088091990813
:1046D000882309F443C010929D0840C010929C08A2
:1046E00080919D088823D1F141E0123609F040E025
:1046F00080919A0860919C080E947D2280919C087C
:10470000882319F0133609F4CA9410929C080E9469
:104710009C2124C080919D08882301F180919A08F2
:104720008093340610929D0881E60E94256080E106
:1047300092E212C01C1494F480919908882341F0ED
:104740000E947122882321F480919A080E945121AD
:1047500010929D088FE290E50E94F71438E0D32E66
:1047600077247A9423E6822E9924BB24BA94662473
:104770006394E0901805E90CFF24F701EE0FFF1F8A
:10478000EE0FFF1FEE0DFF1DE25CFA4F4081842FFC
:10479000807C09F462C146FF06C04F7380E06D2D36
:1047A00020E00E94580F1C14E4F4E701CC0FDD1F39
:1047B000CC0FDD1FCE0DDF1DC25CDA4F8981C8161C
:1047C00081F46D2D695F80E048E10E94675C8B8118
:1047D00080939A0888818F7380939B0860929908D0
:1047E000B92CF701EE0FFF1FEE0FFF1FEE0DFF1D9F
:1047F000E25CFA4F808187FF05C19481C92FDD27D4
:10480000C7FDD095AA24A3949281C912AA2486FD3B
:104810001FC0FE01EE0FFF1FCE01A3E0880F991FFE
:10482000AA95E1F7E80FF91FED53FE4F4081469539
:10483000477050E04553524F80919D08882311F4F2
:1048400000E001C00A2D82E16D2D21E00E947B5B1A
:10485000FE01EE0FFF1FCE0163E0880F991F6A95DE
:10486000E1F7E80FF91FEE55FE4F448D552747FD40
:1048700050958DE26D2D2A2D0E945C5E80919D08E1
:10488000882311F420E001C02A2D8DE26D2D45E230
:104890000E94B85AFE01EE0FFF1FCE0143E0880FC1
:1048A000991F4A95E1F7E80FF91FEE55FE4F438D2A
:1048B00080919D08882311F420E001C02A2D86E311
:1048C0006D2D0E942C0FFE01EE0FFF1FCE0123E085
:1048D000880F991F2A95E1F7E80FF91FEE55FE4F53
:1048E000458D442359F080919D08882311F420E0E0
:1048F00001C02A2D8EE46D2D0E94780FFE01EE0F6F
:10490000FF1FCE01B3E0880F991FBA95E1F7E80FBA
:10491000F91FEE55FE4F468D442391F023E0429F50
:10492000A00111244651504F80919D08882311F415
:1049300000E001C00A2D86E66D2D23E00E947B5B1E
:10494000FE01EE0FFF1FCE0173E0880F991F7A95CD
:10495000E1F7E80FF91FE454FE4F21E08581882339
:1049600009F420E0FE01EE0FFF1FCE0153E0880F97
:10497000991F5A95E1F7E80FF91FE454FE4F86811D
:10498000882329F0222309F498C04AE203C0222395
:1049900061F044E480911905882311F420E001C0FE
:1049A0002A2D89E76D2D0E94B85A8A2D813051F544
:1049B0005E01AA0CBB1C33E0CC0FDD1F3A95E1F77A
:1049C000AC0EBD1EE2EAF1E0AE0EBF1E812FF50176
:1049D000648D43E82DE70E949A14F501848FF70156
:1049E000EE0FFF1FEE0FFF1FEE0DFF1DE25CFA4FF3
:1049F000848180939A0880818F7380939B081092A2
:104A00009908B92CF701EE0FFF1FEE0FFF1FEE0DF7
:104A1000FF1DE25CFA4F8181882331F088150CF488
:104A2000882E87150CF0782EF701EE0FFF1FEE0F82
:104A3000FF1FEE0DFF1DE25CFA4F8281882331F0EB
:104A400088150CF4882E87150CF0782E9394F8E0D6
:104A5000DF0E292D273009F08CCECC20A1F08B2D34
:104A60008F3FF9F4C81464F48091180590E0019721
:104A7000EFEF8F3F9E0711F480E090E080931805E0
:104A80007C14ECF414C0FB2DFF3F59F48091180501
:104A900090E001972FEF8F3F920761F480E090E064
:104AA00009C08B2D86305CF0992D983040F08091B4
:104AB00018058F5F8093180502C043E56BCFDF9127
:104AC000CF911F910F91FF90EF90DF90CF90BF900B
:104AD000AF909F908F907F906F9008952F923F920C
:104AE0004F925F926F927F928F929F92AF92BF92FE
:104AF000CF92DF92EF92FF920F931F935C01CC2431
:104B0000DD243B018824992464E6262E312C412C97
:104B1000512CC201B1016619770988099909A601CA
:104B200095010E94D76B7B018C0182E390E0A0E0AD
:104B3000B0E0E80EF91E0A1F1B1FC601B5010E9456
:104B4000D76B0E94D76BBC0188279927A4019301DA
:104B50000E94D76B44E096958795779567954A951F
:104B6000D1F7E60EF71E081F191FC801B701A201F1
:104B700091010E94296CC9011F910F91FF90EF9044
:104B8000DF90CF90BF90AF909F908F907F906F906D
:104B90005F904F903F902F9008951F93CF93DF9396
:104BA0009C016115710511F1132F111F1127111FA0
:104BB00019F0309521953F4F77FF0EC0C0E0D4E04B
:104BC000709561957F4FCE01821B930B0E946E25DD
:104BD0009E01281B390B05C0C9010E946E25282F94
:104BE000392F112319F0309521953F4FC901DF91DD
:104BF000CF911F9108956F927F928F929F92AF9263
:104C0000BF92CF92DF92EF92FF920F931F93DF93A9
:104C1000CF93CDB7DEB7982E962F322F802F6E2DE3
:104C2000222359F0442361F440919A0450919B044B
:104C30004115510539F421E001C020E0FF2405C0F1
:104C400022E001C021E0FF24F394332311F09111FD
:104C500021E04A2D433679F44C2D50E0440F551F86
:104C60008A0173E0000F111F7A95E1F7041B150B01
:104C7000085A1C4F11C0FA2DF236D9F44C2D50E0D1
:104C8000440F551F8A0193E0000F111F9A95E1F719
:104C9000041B150B075A1C4FF80140810E94780F26
:104CA000FF2009F463C0F8016081892D4AEE26E1F6
:104CB00059C069887724BB24882051F54C2D50E0D9
:104CC000440F551F6A01B3E0CC0CDD1CBA95E1F727
:104CD000C41AD50AAA0CBB1CAA0CBB1CCA0CDB1C30
:104CE000C60CD71C4CE453E0C40ED51EF60140811F
:104CF000552747FD50950E945C5EFF20B9F1F601F3
:104D00006081892D4CE924E60E949A14F6012DC099
:104D1000DD24AA0CBB1CA601E3E0440F551FEA9555
:104D2000E1F74C195D09A40EB51EA80CB11CAA0C24
:104D3000BB1CF301EA0DFB1DE45BFC4F40815527D2
:104D400047FD50954C595F4F0E945C5EFF2071F00B
:104D50008501060D171D045B1C4F892DF80160812C
:104D60004CE920E00E949A14F8018083CF91DF91F2
:104D70001F910F91FF90EF90DF90CF90BF90AF9079
:104D80009F908F907F906F9008952F923F924F92B7
:104D90005F926F927F928F929F92AF92BF92CF92CB
:104DA000DF92EF92FF920F931F93DF93CF93CDB7D4
:104DB000DEB72A970FB6F894DEBF0FBECDBFD82E50
:104DC00082EC9DE00E94F81887E998E06D2D40E0A4
:104DD00020E030E000E07AECE72E7DE0F72ECC24F6
:104DE00053E0A52E0E946C1A40918F084F5F80E31C
:104DF00060E020E00E942C0FF090970880918F08CF
:104E000090E0880F991FFC0123E0EE0FFF1F2A9509
:104E1000E1F7E81BF90BE85AFC4F808160E040E0C5
:104E20000E9456108823C1F080918F0890E0880F6F
:104E3000991FFC0113E0EE0FFF1F1A95E1F7E81B25
:104E4000F90BE75AFC4F808160E040E00E94561069
:104E5000882321F411E003C010E001C012E060914A
:104E60008F08462F50E0FA01EE0FFF1FE651FB4F6F
:104E7000808191818A3191051CF01092960807C0BB
:104E80002FEF873E92071CF481E0809396082091D3
:104E9000860130E02170307082E090E0821B930B3D
:104EA0008417950741F4643030F48091B301807F1A
:104EB00011F01092960880E16DEB7DE00E94E15BBD
:104EC0000F92EDB7FEB7319621E0F11020E080910E
:104ED000960880838D2D61E041E006E3A0E1EA2E93
:104EE000C0908F08A12E88240E94FB250F9088E196
:104EF00066EB7DE00E94E15B0F92EDB7FEB7319665
:104F000021E03F2D313009F020E080919608808328
:104F10008D2D61E041E006E3F8E1EF2EC0908F08AF
:104F2000A12E882483940E94FB250F9080E260EBE1
:104F30007DE00E94E15B0F92EDB7FEB7319621E074
:104F40008F2D823009F020E010828D2D61E041E04C
:104F50000EE1E0E2EE2EC0908F0873E6A72E8824C3
:104F60000E94FB250F9088E26AEA7DE00E94E15BE7
:104F70000F92EDB7FEB7319621E09F2D933009F0E7
:104F800020E010828D2D61E041E00EE158E2E52E37
:104F9000C0908F0832E6A32E88240E94FB250F9034
:104FA000113019F0123049F404C080E363EA7DE067
:104FB00007C080E36CE97DE003C080E364E97DE045
:104FC0000E94E15B00918F08402F50E0812F90E01C
:104FD000880F991F880F991FBA01660F771F9B01D1
:104FE000B3E0220F331FBA95E1F7261B370B820F70
:104FF000931F8E559E4FFC01E655FE4FA081A9835D
:10500000FC01E555FE4FB081BA83FC01E455FE4F2B
:105010009080E4E69E0E83559E4FDC018C908E0EB0
:105020002091860130E02170307082E090E0821B98
:10503000930B8417950709F062C0043008F05FC035
:105040008091B301807F09F45AC0EE24FF248701C8
:1050500020E030E0B9816B2E772467FC7094A1E2E8
:105060004A2E512C292C332427FC3094F0E4CF2EE7
:10507000D22ED801C701B595A79597958795B3010D
:1050800029873A870E94CD25880F991FB2010E9477
:10509000166C629DC001639D900D729D900D112450
:1050A0006FE3A62EAD0C64E670E00E94026CEC2D5E
:1050B000E61B6E2F8A2D0E941B5C29853A85C9014B
:1050C00083709070009761F48A2D6FE30E941B5CDF
:1050D0006D2D6695605E8FE30E941B5C3A85298585
:1050E0002F5F3F4F81E290E0A0E0B0E0E80EF91EB4
:1050F0000A1F1B1F2E33310509F0BACF7CC0DD24F7
:105100009981492E552447FC509401E210E0A92DC5
:10511000BB27A7FDB095BC83AB8354E6652E712CED
:1051200040E2A42EBA812B2E332427FC3094E82DA4
:10513000FF27E7FDF095FE83ED83FD2D21E2F29F31
:1051400070011124C701B2010E94CD25B8010E944F
:10515000166CAB81BC816A9FC0016B9F900D7A9FDA
:10516000900D11243EE5C32ECD0CB3010E94026CBC
:10517000BA2DB61B6B2F8C2D0E941B5CED2DF0E021
:10518000E370F070F887EF83309749F48C2D60E27C
:105190000E941B5C6D2D605E8EE50E941B5CC7014A
:1051A000B1010E94CD25B8010E94166C2D813E816F
:1051B000629FC001639F900D729F900D11242EE598
:1051C000F22EFD18B3010E94026C605E8F2D0E94CA
:1051D0001B5C8F819885009749F48F2D60E20E94B7
:1051E0001B5C6A2D6D198EE50E941B5CD3949D2D6E
:1051F0009F3109F0A2CFE0918F08F0E0EE0FFF1F82
:10520000E651FB4F408051805201CC24B7FCC09442
:10521000DC2CC601B50121E230E040E050E00E9404
:105220004B6C822F825A61E04EE30E946B5C40918E
:105230008F082091860130E02170307082E090E08C
:10524000821B930B242F30E08217930709F050C084
:10525000443008F04DC08091B301807F09F448C00C
:10526000C601B50160507C4F8F4F9F4F22E030E068
:1052700040E050E00E944B6CA9816A2F772767FDC0
:105280007095C9010E94CD25BC01660F771F882744
:1052900077FD8095982F292D97FC2D5F25952595D5
:1052A000332727FD3095432F532F0E94D76B29E1D9
:1052B00030E040E050E00E944B6C79018A01CA0165
:1052C000B9012FED3FEF4FEF5FEF0E944B6C622F64
:1052D000605C8FE34EE30E94675CC801B70122E087
:1052E00030E040E050E00E944B6C79018A013CC004
:1052F0001A141B041C041D0414F4698101C06A8182
:10530000772767FD7095C2010E94CD259C01442737
:1053100037FD4095542F1A141B041C041D0414F46B
:10532000692D01C0682D67FD6D5F659565957727CF
:1053300067FD7095872F972F0E94D76B29E130E08A
:1053400040E050E00E944B6C79018A01CA01B9012A
:105350002FED3FEF4FEF5FEF0E944B6C622F605ECF
:105360008FE34EE30E94675CC601B50129E130E09E
:1053700040E050E00E94D76B612CB1E07B2E812C85
:10538000912CA40193010E944B6C82E760E3A90178
:1053900020E00E945C5EC801B70129E130E040E0F6
:1053A00050E00E94D76BA40193010E944B6C84E5EE
:1053B00068E0A90120E00E945C5E1A141B041C0432
:1053C0001D0474F4B9816B2F772767FD7095C201B6
:1053D00044970E94CD25F701E81BF90BCF010BC0C4
:1053E000FA816F2F772767FD7095C20144960E945E
:1053F000CD258E199F099C01220F331F220F331FC9
:10540000280F391F442737FD4095542F84E560E16C
:1054100000E3F3E0EF2E0E94265D2A960FB6F89483
:10542000DEBF0FBECDBFCF91DF911F910F91FF90D7
:10543000EF90DF90CF90BF90AF909F908F907F9034
:105440006F905F904F903F902F9008952F923F92D2
:105450004F925F926F927F928F929F92AF92BF9284
:10546000CF92DF92EF92FF920F931F93DF93CF9330
:10547000CDB7DEB72F970FB6F894DEBF0FBECDBF06
:10548000982E8AE89DE00E94F81884E998E0692D3A
:1054900043E022ED37E00AE0F2E9EF2EFDE0FF2ED7
:1054A000CC24C394E4E0AE2E0E946C1AF0909408D1
:1054B000FA9430909508292D203841F4F7FC06C065
:1054C000F0928F0885EC96E20E94F71485E168E07F
:1054D0004AE75DE00E94E95B88E593E09C838B836B
:1054E00070E9472E78E0572EEAEEF4E0FB87EA8772
:1054F00010E1662477242F2D332727FD30953A833A
:105500002983C901880F991FFC0153E0EE0FFF1F8B
:105510005A95E1F7E81BF90BFE83ED83F62CEB813E
:10552000FC81808160E040E00E945610882361F099
:10553000EB81FC81818160E040E00E94561088236D
:1055400029F4BB24B39404C0BB2402C042E0B42EAF
:105550002B2D30E038872F83C901880F991F880FC2
:10556000991FA301440F551F9A0103E0220F331F17
:105570000A95E1F7241B350B820F931F8E559E4F22
:10558000DC01A355BE4FFC01E455FE4F3C91208148
:10559000321751F4FC01E555FE4F86559E4F41E010
:1055A0002081FC018081281340E0EA85FB85819100
:1055B0009191FB87EA879C0197FF04C0222733273C
:1055C000281B390B2A3131050CF040E0242E8A319A
:1055D00091051CF0F201108207C0FFEF873E9F0784
:1055E0001CF421E0F20120838091860190E081701B
:1055F0009070E2E0F0E0E81BF90BE615F70551F4D6
:105600008091B301807F31F0F301E057F74F1082B2
:10561000222423944F2D4F5F80E0612F20E00E94D1
:105620002C0F5D864C86F2013081F1E0F987311153
:10563000198680911905882351F4DD24D394809133
:105640009A0490919B04009721F4DD2402C0DD248C
:10565000D39489819A818615970511F421E0311040
:1056600020E00F92EDB7FEB73183892D60E04D2D1C
:1056700007E2E12ECF2CAB2C88240E94FB250F9053
:1056800029813A812615370509F0D2C0332009F067
:10569000CBC0DD2009F4CCC0222009F4C9C08F8121
:1056A0009885880F991F880F991FED81FE818E0FB5
:1056B0009F1F8E559E4FF9858F0F911D86559E4FCA
:1056C0009F878E87892DEE85FF8560814CE924E6D2
:1056D0000E949A14EE85FF858083AAC021E00F9274
:1056E000F2018081EDB7FEB78183892D60E04D2DF9
:1056F00009E3E12ECF2CAB2C882483940E94FB2558
:105700000F9029813A812615370509F097C0332D6E
:10571000313009F08FC0DD2009F490C0222009F457
:105720008DC08F819885880F991F880F991FED81F3
:10573000FE818E0F9F1F8E559E4FF9858F0F911DF5
:1057400084559E4F98878F83892DEF81F8856081DE
:105750004CE920E00E949A14EF81F88580836EC0A6
:1057600021E00F92EDB7FEB71182892D60E04D2D3B
:105770000FE3E12ECF2CF3E6AF2E88240E94FB2509
:105780000F9029813A812615370521F421E0332D28
:10579000333009F020E00F92EDB7FEB71182892D6A
:1057A00060E04D2D07E5E12ECF2CE2E6AE2E8824F9
:1057B0000E94FB250894411C511C0F90EC85FD852F
:1057C0008081882319F4222031F008C0222031F48E
:1057D0008AE34FE705C08BE34EE702C08AE34DE260
:1057E000612F0E94775BFB2DF13019F0F23049F404
:1057F00004C085E7612F4DE407C085E7612F4CE4C5
:1058000003C085E7612F48E40E94775B0894611C20
:10581000711C2B813C81225F3F4F3C832B83185F9F
:10582000103309F07BCE0CC0332D313009F456CF44
:1058300020E055CF832D823009F492CF20E091CF24
:105840002F960FB6F894DEBF0FBECDBFCF91DF917C
:105850001F910F91FF90EF90DF90CF90BF90AF908E
:105860009F908F907F906F905F904F903F902F9080
:10587000089520E030E0F901E95CF24FE491E81787
:1058800011F4822F08952F5F3F4FEE23A1F780E0A0
:105890000895823430F4E82FF0E0E95CF24F84910F
:1058A000089580E20895EF92FF920F931F93182FAF
:1058B000F62EE22E862FBA010E94E15B86E66F2D5E
:1058C000412F2E2D0E942B1AEE2039F0802F612FB0
:1058D00040E021E00E94A914182F812F1F910F9101
:1058E000FF90EF900895FF920F931F93F82E109161
:1058F000AD01212F332727FD309537FF03C03095A9
:1059000021953F4F022F25320CF43DC020913E08D7
:1059100030913F0880913C0890913D08282B392B0D
:105920008091400890914108282B392B80913B08A9
:1059300090E0282B392B4091380850E0242B352B50
:105940002115310531F4812F881F8827881F809306
:10595000380811161CF4812F845202C0812F8C5DEF
:1059600060E040E00E945610882359F0909138087A
:10597000992339F491E020913B08211190E0909314
:105980003B088093380820913E0830913F082F5FF4
:105990003F4F30933F0820933E0820913C083091C0
:1059A0003D082F0D311D30933D0820933C080E9487
:1059B000830E2091400830914108821B930B84365E
:1059C000910508F471C12C593F4F30934108209341
:1059D000400820913C0830913D08E0913E08F0914C
:1059E0003F08C901BF010E94026CF62E462F50E00D
:1059F0004E9FC0014F9F900D5E9F900D1124281B5C
:105A0000390B30933D0820933C0810923F081092C8
:105A10003E0800311CF410923B080FC005326CF4B4
:105A200011161CF4812F8F5002C0812F815F60E01E
:105A300040E00E94561080933B0880913706909179
:105A400038060196909338068093370640913906C0
:105A500050913A064F5F5F4F50933A064093390694
:105A6000FF2049F080913D0690913E06019690936B
:105A70003E0680933D0680913B08882349F0809143
:105A80003B0690913C06019690933C0680933B0622
:105A9000F69420913F06309140062F0D311D309332
:105AA000400620933F068091AF019091B001909302
:105AB0004306809342066091AD01772767FD70959C
:105AC00077FF03C0709561957F4F662319F410929C
:105AD00041061EC0613019F4841B950B15C060315E
:105AE00068F460FF06C0A4E036952795AA95E1F713
:105AF00009C020913D0630913E0604C020913B062E
:105B000030913C06821B930B909343068093420690
:105B100080914106813051F0813018F0823049F592
:105B200014C08091AD01882321F120C080914206EC
:105B30009091430618161906E4F08091AF019091F8
:105B4000B0010097B1F082E012C0809142069091BE
:105B500043062FEF853C92071CF483E080934106B7
:105B60008091AF019091B001009719F481E080938A
:105B70004106809142069091430620913908309168
:105B80003A082817390709F479C0209141062130D5
:105B900009F065C02091880122FF45C02091AF0126
:105BA0003091B00121153105F1F18E31910519F4D3
:105BB00089E10E94D06B8091420690914306843126
:105BC000910519F48AE10E94D06B80914206909170
:105BD00043068A30910519F48BE10E94D06B8091C5
:105BE000420690914306843091051CF48CE10E949A
:105BF000D06B8091880183FF16C0809142069091FE
:105C000043068E31910549F08431910531F08A3097
:105C1000910519F08430910534F482E390E090937B
:105C20009E0480939D048091880181FF27C080910C
:105C3000AE01209142063091430680FF07C080915B
:105C4000AF019091B001821B930B01C0C9016CE3BD
:105C500070E00E94026C009789F480E003C022305B
:105C600069F48CE10E94D06B8091880183FF06C0AB
:105C700082E390E090939E0480939D0420914206DD
:105C80003091430630933A08209339088091AE0151
:105C900080FF0AC08091AF019091B001821B930BED
:105CA00090934306809342061F910F91FF900895B1
:105CB0008091AD01992787FD909597FF03C090953E
:105CC00081959F4F982F823034F1803124F585954E
:105CD0009A3024F40E94496190E003C0992787FD1F
:105CE00090950197FC01EE0FFF1FE651FB4F2081BD
:105CF00031818091AD0187FF05C080E094E0821B77
:105D0000930B03C0C90180509C4F26E09695879560
:105D10002A95E1F702C080E090E00E94732C83E0B6
:105D20000E944961E82FF0E0EE0FFF1FE851FB4FA2
:105D30008081918180509C4FB6E096958795BA9569
:105D4000E1F72091AE0122FF0AC08530910538F0BD
:105D50002091A004222319F423E02093A004209191
:105D60003408309135082F5F3F4F3093350820932A
:105D700034082091320830913308280F391F3093AE
:105D80003308209332080E94830E20913608309108
:105D90003708821B930B23E0883E9207E8F10E94AC
:105DA000830E90933708809336088091B10182303A
:105DB00051F485E160E040E00E945610882319F01C
:105DC00087E00E94D06B80913208909133086091F7
:105DD0003408709135080E94026C109233081092BA
:105DE000320810923508109234088091BD069091C7
:105DF000BE0601969093BE068093BD068091BC06B8
:105E0000E82FF0E0EC5BF94F60838F5F8093BC0676
:105E1000883710F01092BC06089510924106109237
:105E20003A061092390610923E0610923D061092E4
:105E30003C0610923B061092400610923F060895D1
:105E40000F931F93182F80913506882319F067E26E
:105E50007DE002C06AE17DE088E00E94E15B81E0D4
:105E600060E142EA51E02AE000E10E947B5B82E4CB
:105E700060E14FE30E94775B82E168E243E15DE02D
:105E80000E94E95B82E160E344E05DE00E94E95B3F
:105E9000113609F44AC01F3B21F0103609F04FC0FB
:105EA00004C080E00E94D06B4AC0809135068823F0
:105EB000A9F082EF9CE00E948C12809136060E942D
:105EC0000455882339F087E10E94D06B82E08093EB
:105ED000350629C080E00E94D06B25C080916F01FB
:105EE0008F5F0E94C85710916F0108C01150113187
:105EF00008F01FE080916F01181739F0812F8F5F34
:105F00000E947B57882391F301C010E010936F012A
:105F100081E00E949C550E94385680916F010E943A
:105F2000D0540E940D2F80E601C081E60E942560BA
:105F300081E00E94C21482EA9FE20E94F7141F913E
:105F40000F910895AF92BF92DF92EF92FF920F935D
:105F50001F93CF93DF93182F8BE09BE00E94F818DC
:105F6000809119058823A1F4E0911C05E7FF10C07A
:105F7000E195EA3008F0E9E0F0E0EE0FFF1FEE52A5
:105F8000F84F25913491C9010E94E71410921C0525
:105F9000F090890889E898E0612F4FE00E94581F2F
:105FA00086E360E046E05BE00E94E95B0E94BD564C
:105FB000AC0186E660E020E00E945C5E80E06AE082
:105FC00041E00E94471AD0908908809135068230BE
:105FD00021F41092880810923506163648F41436CB
:105FE00090F5103609F456C0113609F075C00AC094
:105FF000113809F456C01F3B09F465C0103809F088
:106000006BC053C0809188088823E9F010928808FB
:1060100087E10E94D06B81E60E9425600E9438567D
:106020008091890880936F010E94D0540E940D2FA7
:1060300081E00E949C550E94385682E00E949C5547
:106040000E94385649C080916F018D15B9F0812F9B
:106050000E9425608091890880936F010E943856C4
:1060600080916F010E94D0540E940D2F81E00E9408
:106070009C550E94385681E00E94D06B153619F469
:1060800080E89EE404C0143639F586EC91E40E9461
:10609000E71422C081E08093880887E10E94D06BDA
:1060A0001BC081E00E94C21417C080918808882319
:1060B00099F081E080933506D092360680E29FE227
:1060C0000E94F71409C01092880880916F01809394
:1060D000890881E00E94AA5580918808882341F0B0
:1060E000FD1431F06D2D6F5F8F2D8F5F0E948957EA
:1060F000CD2DDD27C7FDD095809118059E01281B69
:106100003109C901181619065CF0CE01019797FFF5
:1061100002C080E090E08093180510E1DD240BC000
:1061200025303105D4F3CE0104978B3091059CF3D3
:106130008AE090E0F0CFF0901805FD0CAF2CBB2466
:1061400095012F5F3F4F442737FD4095542FCA15C7
:10615000DB0511F401E101C000E182E1612F72E091
:10616000E72E0E94265D80916F01F81629F481E0E8
:10617000612F4AE20E94775B8F2D69E778E04FE05C
:106180000E948854CA15DB0531F480918808882361
:1061900011F001E101C000E188E1612F49E758E019
:1061A0002FE00E947B5BD394185F3D2D363019F6AB
:1061B000DF91CF911F910F91FF90EF90DF90BF90F3
:1061C000AF900895AF92BF92CF92DF92EF92FF927D
:1061D0000F931F93CF93DF935B016C0110E1E12ECE
:1061E000F12CC0E0D0E800E010E89E0140E050E073
:1061F000CA01B9010E94D76BA616B706C806D90610
:1062000010F4C027D127169507950894E108F108E6
:10621000E114F10461F4CE01DF91CF911F910F9150
:10622000FF90EF90DF90CF90BF90AF900895C02B7C
:10623000D12BDBCFE1E0683068F4E0E070E09B0157
:10624000220F331F220F331F260F371FA901485774
:106250005C4F0EC070E0685070409B0153E0220F0D
:10626000331F5A95E1F7260F371FA90140555C4FA0
:10627000DA012C9180509C4F97FD0FC0B8E0803020
:106280009B078CF0EE2319F028E030E002C024E0F8
:1062900030E0240F351FF9012081332727FD309589
:1062A000322F222730C0EE2329F0692F9070880FFB
:1062B000991F03C0692F66959170262F30E0FA016F
:1062C000E20FF31F6181772767FD7095AC0155954B
:1062D0004795649F9001659F300D749F300D112488
:1062E0006081772767FD709540E052E0481B590BAD
:1062F00055954795649FC001659F900D749F900DC3
:106300001124280F391FC90169E170E00E94166C41
:10631000CB0108952F923F924F925F926F927F929E
:106320009F92AF92BF92CF92DF92EF92FF920F9324
:106330001F93DF93CF9300D00F92CDB7DEB7182F06
:10634000992493948091A008883008F499248AEDC8
:106350009FE00E94F818992011F05AE001C056E021
:106360008EEB98E0612F40E020E030E000E070EE3E
:10637000E72E7FE0F72ECC24C394A52E0E946C1A42
:106380004091A00850E04F5F5F4F84E260E021E061
:106390000E945C5E8091A008992079F090E00897B7
:1063A0007C0103E0EE0CFF1C0A95E1F7E80EF91EF4
:1063B00020EB33E0E20EF31E0CC090E07C01EE0C0B
:1063C000FF1CEE0CFF1CE80EF91E88E893E0E80EB7
:1063D000F91E0091BE080150D090BF08113661F03F
:1063E000123628F41434D1F0153471F50EC0143679
:1063F000A9F0153649F509C0DD2031F11092BF082A
:1064000081E60E942560DD241FC080911905882344
:10641000D9F01D14CCF48D2D815014C08091190534
:10642000882391F02D2D332727FD3095992019F0E1
:1064300089E090E002C085E090E02817390724F455
:106440008D2D8F5F8093BF088091BF0880931905C1
:10645000CE2C4F2C6E2C7F2C90E122243324A02EA6
:10646000BB24A7FCB094F30141913F01552747FDA0
:10647000509521E0A214B30409F020E088E1692FCF
:1064800099830E945C5E0894211C311C9981985F5D
:10649000983349F7992001F1A5E06A2E712C6E0C12
:1064A0007F1C90E1F5E02F2E312CF30141913F014B
:1064B000552747FD509521E0A214B30409F020E0D0
:1064C00080E3692F99830E945C5E0894211C311C33
:1064D0009981985F903349F70F3F11F421E0D11073
:1064E00020E08CE068E043ED5FE00E94BA5B992019
:1064F00019F089E090E002C085E090E021E0A81664
:10650000B90609F020E08CE068E34CEC5FE00E9403
:10651000BA5B992019F089E090E002C085E090E034
:10652000A816B90694F407FD4EC0A02EBB24A7FC04
:10653000B094AE0CBF1C812FF50160814CE924E6BC
:106540000E949A14F50180833EC01016E4F5812F55
:106550006091BD084CEF24E000E00E948C14809311
:10656000BD0890919704992371F1992021F050E191
:1065700094E049E003C058E092E045E024E682025E
:1065800030011124892F90E0909581959F4F869D31
:106590009001879D300D969D300D1124EC2DF42D2A
:1065A000A52E00E0C9016A2D702F0E94166C619320
:1065B000260D371D8E2F8C198417A0F382E00E94C0
:1065C0009C550E94385680911905882351F0AA24C1
:1065D000ECE92E2EEFEF3E2E4D2C552447FC509427
:1065E000A5C000E01CEFAA24BB2470E2D72EACC0EB
:1065F000C90165E0880F991F6A95E1F7992019F0A4
:1066000064E070E002C062E070E00E94166C462F09
:10661000062F055C37016A0C711CF30180819927F4
:1066200087FD909555E0880F991F5A95E1F7B101C4
:106630000E94166C562F90E2D92ED60E2F5F3F4F38
:106640008D2D90E09B838A834216530609F050C03B
:1066500082349105ACF48AE3C82EC40E625E8C2DA0
:1066600045E059830E94675C5981EA81FB81E134EE
:10667000F10531F0652F615E8C2D45E00E94675C6D
:10668000FD2DF03430F4802F81506D2D45E00E94B7
:10669000675C2A813B812F33310594F401506D2DC5
:1066A0006F5F802F45E00E94675C8A819B818E33FB
:1066B000910531F06D2D6E5F802F45E00E94675C83
:1066C00080919A0490919B04009741F4123631F026
:1066D000133621F0123411F0133439F5812FF30100
:1066E00060814CE924E60E949A14F30180831DC066
:1066F0002A813B81213431052CF4615E802F43E0F7
:106700000E94675C3D2D303428F4802F6D2D43E0CE
:106710000E94675C8A819B818F33910534F46D2DD3
:106720006F5F802F43E00E94675CA3942A2D30E0C6
:10673000992019F089E090E002C085E090E02817E8
:1067400039070CF455CF4DCFC8016091A0080E94C5
:106750001A31BCE3EB2EEA0C9C01A5E03695279597
:10676000AA95E1F76D2D621B8E2D0E941B5C950191
:10677000237030702115310521F48E2D60E20E94C6
:106780001B5C0894A11CB11C005E1F4F90E4A9166D
:10679000B104D1F68CE560E040E40E946B5C0F90A0
:1067A0000F900F90CF91DF911F910F91FF90EF907D
:1067B000DF90CF90BF90AF909F907F906F905F9051
:1067C0004F903F902F9008952F923F924F925F925B
:1067D0006F927F928F929F92AF92BF92CF92DF92F1
:1067E000EF92FF920F931F93DF93CF93CDB7DEB756
:1067F000A2970FB6F894DEBF0FBECDBF8F8F98A3C0
:106800006A8B80919C04882309F474C080911A05D6
:10681000882319F0815080931A058091C5069091C4
:10682000C6062091C3063091C406820F931F2091A3
:10683000C7063091C806820F931F2091C906309178
:10684000CA06820F931F20914E0730914F072C01EB
:10685000421A530A920157FE03C0309521953F4FCB
:1068600041E0213034073CF090934F0780934E076E
:1068700081E080939F0480918701863FD9F19091B8
:1068800008019233B8F190914B079F5F90934B07AB
:10689000903160F020914C0730914D072F5F3F4FB2
:1068A00030934D0720934C0710924B0790919F0413
:1068B000992321F010924D0710924C0720914C071C
:1068C00030914D07992787FD90950A9667E771E00B
:1068D000869FA001879F500D969F500D112442174F
:1068E000530740F4237030702130310519F480E1F2
:1068F0000E94D06B80918601582F51705F5F59873D
:1069000081FF02C01D8602C063E06D876090BA01FE
:10691000662009F44AC08985E82FF0E0EE0FFF1FDA
:10692000E651FB4FA080B180CC24B7FCC094DC2C96
:106930009D85E92FF0E0EE0FFF1FE651FB4F208110
:106940003181442737FD4095542FCA01B9010E9477
:10695000D76B7B018C01C601B501A60195010E9490
:10696000D76BE60EF71E081F191F662D70E080E03A
:1069700090E0EAE0660F771F881F991FEA95D1F72C
:1069800024E630E040E050E00E944B6CB901CA01BF
:106990000E94D76B6E157F058007910730F4C80100
:1069A000B7010E94E2304C0102C088249924B4014E
:1069B00080E090E024E630E040E050E00E94D76BB9
:1069C0006B8F7C8F8D8F9E8F62E4662E61E0762EBA
:1069D000A3ECB6E0BE8BAD8BFE013196F88FEF8B4A
:1069E00050E0252E51E0352E22EA31E03F872E87F8
:1069F0004AEE54E05A8F498F2901F98BE88BBC8B02
:106A0000AB8BEE24FF241B865A89517059A3AE2C00
:106A10008E2D0E949A159C01D30111968D919C9107
:106A20001297281B390BB901882777FD8095982F7D
:106A30004AE0660F771F881F991F4A95D1F71216F3
:106A400013062CF45D962D913C915E9703C0F301E3
:106A5000278530892436310514F424E630E04427B4
:106A600037FD4095542F0E944B6C8901FCEF21307B
:106A70003F072CF024E00030120724F405C000E0AA
:106A80001CEF02C000E014E08091880180FF0FC07D
:106A90008091860190E08170907042E050E0481B48
:106AA000590BE416F50619F4109501951F4FA98DA1
:106AB000BA8D0D931D93BA8FA98FC8010F968F3190
:106AC0009105F0F4B4E0EB16F1047CF48A2D8F5FAD
:106AD0000E94496190E00197E1E0F0E002C0EE0F12
:106AE000FF1F8A95E2F7CF0108C081E090E00E2CED
:106AF00002C0880F991F0A94E2F7FB85F82BFB87E9
:106B00002A2D243008F07AC139A1332309F05FC05F
:106B10008091AE0181FF5BC06701CC0CDD1C4CE7AE
:106B200051E0C40ED51ED60111968C911197807C30
:106B300009F44DC08C9185958595859561E040E07F
:106B40000E945610882309F442C0D601EC91E770E8
:106B5000F0E0DF01AA0FBB1FAC55BB4FEE0FFF1FCC
:106B6000EC58FE4F8D919C91119720813181821BB1
:106B7000930B62E070E00E94166CF701EE0FFF1FAE
:106B8000E358FE4F2081422F440F440F4595459511
:106B9000552747FD5095649FC001659F900D749FD8
:106BA000900D11246FE170E00E94166C660F771F44
:106BB000660F771F2295269526952370213019F0B0
:106BC000223029F403C0060F171F01C08B01811466
:106BD000910409F1B985AB1619F0ED85AE16D9F41B
:106BE0006091BA0170E080E090E04AE0660F771FA4
:106BF000881F991F4A95D1F79801442737FD409582
:106C0000542F0E94D76B2B8D3C8D4D8D5E8D0E9435
:106C10004B6C022F132FF201EA54FE4F808160E08B
:106C200040E00E945610882369F0F201E954FE4FBB
:106C3000808160E040E00E945610882329F4CC2433
:106C4000C39404C0CC2402C032E0C32E80918601DC
:106C500090E08170907022E0A22EB12CA81AB90A9F
:106C6000AE14BF0469F58091B301807F49F1C8017A
:106C700080509C4F62E070E00E94166C9B01EC2DEE
:106C8000F0E0EE0FFF1FEE0FFF1FA701440F551F8F
:106C9000CA01A3E0880F991FAA95E1F7841B950B01
:106CA000E80FF91FE45BFC4F6081772767FD709563
:106CB000C9010E94CD25AC01440F551F30E028C00A
:106CC00031E0101611060CF430E08C2D90E0A70195
:106CD000440F551FFA0163E0EE0FFF1F6A95E1F7BD
:106CE000E41BF50B880F991F880F991FE80FF91FF8
:106CF000EE55FE4FE30FF11DE655FE4F60817727FD
:106D000067FD7095C8013AA30E94CD25AC013AA158
:106D1000EC2DF0E0EE0FFF1FEE0FFF1FB701660F27
:106D2000771FCB0113E0880F991F1A95E1F7861B97
:106D3000970BE80FF91FEE55FE4FE30FF11DE455D9
:106D4000FE4F6081772767FD70956C597F4F8827CC
:106D500077FD8095982FDA019D01442737FD4095F6
:106D6000542F0E94D76B24E630E040E050E00E94B0
:106D70004B6C022F132FAE14BF0499F58091B30111
:106D8000982F907F09F466C60050144063C6D10165
:106D9000ED91FC91119760818091880180FD619552
:106DA000772767FD7095872F972F63587F4F8F4FF9
:106DB0009F4F20E034E0201B310B442737FD4095E6
:106DC000542F0E94D76B20E038E040E050E00E9452
:106DD0004B6C2030B8E03B07B0E04B07B0E05B07FE
:106DE00039F4D101ED91FC912081332727FD3095B5
:106DF000220F331FE889F98931832083AB89BC894D
:106E00000D931D93BC8BAB8B0894E11CF11CE2E04D
:106E1000F0E06E0E7F1E288939892E5F3F4F398B37
:106E2000288B2E0E3F1E4EE050E0440E551E57E0BC
:106E3000E516F10409F0EBCD0091B7016B8506234F
:106E4000809150078095802319F088E10E94D06BD3
:106E50000093500780E094E09093D2068093D1068F
:106E60009093D4068093D306E4EAF4E024E731E07B
:106E7000ABEDB6E0BD0181919191D9014D915D914C
:106E80009D01841B950B880F991FDB018D939D93AA
:106E9000BD01B4E0EC3AFB0771F78091AC0490912E
:106EA000AD04880F991F9093E4068093E3068091C8
:106EB000AE049091AF04880F991F9093E6068093DB
:106EC000E5068091B0049091B104880F991F9093CA
:106ED000E8068093E7068091B2049091B304880F8E
:106EE000991F9093EA068093E906EBE0F7E0FC87B0
:106EF000EB872BEE36E04191519161917191D9016F
:106F00004D935D939D01B7E0EB34FB07A1F7C09073
:106F1000BA01CC2009F47AC0E985AE2EBB24AA0CB4
:106F2000BB1C23EC422E26E0522EA40CB51CD5012E
:106F30002D903C90442437FC4094542CBD850B2F5D
:106F400010E0000F111F0D53194FF80120813181FE
:106F5000442737FD4095542FCA01B9010E94D76BD1
:106F60003B014C01C201B101A20191010E94D76B0A
:106F7000660E771E881E991EDD24EE24FF248AE00B
:106F8000CC0CDD1CEE1CFF1C8A95D1F7C701B601A5
:106F900024E630E040E050E00E944B6CB901CA01A9
:106FA0000E94D76B661577058805990578F5C401A9
:106FB000B3010E94E230BC0180E090E024E630E0C2
:106FC00040E050E00E94D76B3B014C01C201B1018F
:106FD000A70196010E94D76BA40193010E944B6CFC
:106FE000D5012D933C93F80160817181882777FD4D
:106FF0008095982FA70196010E94D76BA401930159
:107000000E944B6CD80111963C932E93E090B801EE
:107010008E2D807E09F4DEC0B9852B2F30E0220F43
:10702000331FF901ED53F94F40815181CE01019693
:10703000280F391FD901ED91FC91BD856B2F70E0B0
:10704000660F771FDB01AD53B94F2D913C91860F31
:10705000971FDC018D919C91BA89B1FD05C0E40FA9
:10706000F51F280F391F04C020E030E0E0E0F0E019
:10707000A091B901AA2349F0B0E0AA0FBB1FAF53FA
:10708000B94F0D911C91119702C000E010E0E2FE93
:1070900003C0F095E195FF4FE3FE03C030952195C5
:1070A0003F4FE4FE03C0109501951F4F8091B8013A
:1070B000829586958770823071F1833020F481301B
:1070C00009F088C007C0833009F459C0843009F042
:1070D00081C06CC0C90168E070E00E94166C7B0141
:1070E000C90160E870E00E94166C29014E185F0823
:1070F0007201E61AF70AC90160E072E00E94166C9C
:10710000E61AF70AC8018E1B9F0B9093D606809350
:10711000D506CF0120C0CF0168E070E00E94166C58
:107120007B01CF0160E870E00E94166C3F016E1891
:107130007F087301E61AF70ACF0160E072E00E944F
:10714000166CE61AF70AC801821B930B9093D606B9
:107150008093D506C90162E070E00E94166C600F52
:10716000711FCB018E0D9F1D9093D8068093D7067B
:107170006E197F097093DA066093D9062BC0C80197
:107180008E1B9F0B9093D6068093D506E00FF11FC0
:10719000CF01820F931F9093D8068093D706E21BEE
:1071A000F30BF093DA06E093D90614C0C8018E1BE6
:1071B0009F0B9093D6068093D506C801820F931F2C
:1071C0009093D8068093D706021B130B1093DA0610
:1071D0000093D90680919C04882311F00E94582EB8
:1071E00080E4EBE0F7E0DF011D928A95E9F7BA89C8
:1071F000B1FF2DC08091860190E08170907022E0F7
:1072000030E0281B390B80E090E0ED89FE89AF89E2
:10721000B88D2817390729F01182108211961C9217
:107220001E920196329612968430910591F7109233
:10723000DC061092DB061092DE061092DD0610923C
:10724000E0061092DF061092E2061092E10684E852
:1072500093E090930101809300019C012F5F3F4FC9
:1072600030930301209302019C012E5F3F4F309326
:107270000501209304010396909307018093060172
:1072800021E1422E28E0522E91E9692E97E0792ED5
:1072900081E5282E87E0382E19861D8689850E9473
:1072A0008B0E7C01FC0180818150803108F0ADC2E1
:1072B000838161E040E00E945610D2019C918823B6
:1072C000A1F4292F1C92F7019181892F88508230D7
:1072D00008F08AC287818E70843009F485C29930A3
:1072E00009F04BC000E01CEF4AC021E0911120E002
:1072F00081E0D2018C93D7011196EC913E2F315051
:10730000832F90E0DC01AA0FBB1FAD53B94F0D9145
:107310001C911197343160F0B9853B1748F4DC01BA
:10732000AA0FBB1FAA0FBB1FA55FB84F0D911C91E1
:10733000D70117963C911797832F807381F0832F85
:107340008295837090E0019741E050E002C0440FC5
:10735000551F8A95E2F7CA015D85582B5D8736FF78
:107360000EC0E53060F4F0E0EE0FFF1FE250FF4F7B
:10737000C70108969183808302C000E010E0D70126
:107380001796CC901797C6FC0BC018968C9118973F
:10739000882331F02AA30E946E0E080F191F2AA11C
:1073A000F7018681882321F48581882309F458C157
:1073B000D3016D917D918D919C911397222389F436
:1073C00020E031E040E050E00E944B6C5095409549
:1073D000309521953F4F4F4F5F4F4801820E931ECE
:1073E0005AC08C2D8E70843051F5D701EC91F0E0AD
:1073F000EE0FFF1FE751F94F60817181882777FDFC
:107400008095982F20E034E640E050E00E94D76B52
:10741000F3016083718382839383D70112962C9149
:107420001297222361F0332727FD3095432F532FE6
:107430000E944B6CF3012083318342835383D30139
:107440006D917D918D919C91139720E031E040E00A
:1074500050E00E944B6C50954095309521953F4FE0
:107460004F4F5F4F4801820E931E8114910499F093
:10747000F701258197FE22952F7030E044E650E019
:10748000249FC001259F900D349F900D1124D101A0
:1074900011969C938E93F10180819181009799F0D0
:1074A00020919C04222319F0019791838083D101BC
:1074B0008D919C911197009731F0F301608171815A
:1074C00082819381B7C08114910409F4C9C0D701A6
:1074D00016968C911697882309F4B4C080919C0469
:1074E000882309F476C012962C9112972223B1F0CA
:1074F000332727FD309537FF03C0309521953F4F47
:10750000332727FD3095432F532F60E070E080E252
:1075100093E00E944B6C59016A0106C0A12CB12C6A
:10752000F0E2CF2EF3E0DF2EF70186811814190464
:10753000FCF48F7090E00097F1F144E650E0849FF6
:107540009001859F300D949F300D1124442737FD05
:107550004095542FC601B5010E944B6CF301808108
:107560009181A281B381280F391F4A1F5B1F2CC054
:1075700082958F7090E00097F1F044E650E0849F90
:107580009001859F300D949F300D1124442737FDC5
:107590004095542FC601B5010E944B6C59016A01F8
:1075A000D3012D913D914D915C9113972A193B097F
:1075B0004C095D0909C09801442737FD4095542FB7
:1075C000542F432F322F2227F3012083318342830C
:1075D0005383D3016D917D918D919C9120E031E099
:1075E00040E050E00E944B6CC801AA2797FDA0958F
:1075F000BA2F1814190434F482179307A407B50797
:1076000034F012C0281739074A075B076CF42227A9
:1076100017FD2095322F322F212F102F0027F30135
:107620000083118322833383D3016D917D918D91EA
:107630009C91139720E031E040E050E00E944B6CB9
:1076400089010EC0C801AA2797FDA095BA2FBA2FAD
:10765000A92F982F8827F30180839183A283B38376
:10766000D70114966C911497633061F1643028F45B
:10767000613051F06230A0F444C0653069F165308A
:1076800038F1663081F52BC0F7018181893029F40A
:1076900017FD35C0005012400EC017FF32C02CC07D
:1076A000D70111968C911197893041F4101611066B
:1076B00004F100501E4F000F111F23C010161106B9
:1076C000DCF01FC017FF1DC0109501951F4F19C09A
:1076D0001016110674F010C017FF0EC010C010165F
:1076E00011063CF00CC06750C8010E941A318C0191
:1076F00008C000E014E005C000E010E002C000E0B7
:107700001CEFF701878180FD13C0E181EE2381F03A
:10771000E53070F4F0E03197EE0FFF1F21E030E02C
:107720002C0F3D1FE20FF31F80819181080F191F5D
:10773000B801882777FD8095982FD70112962C9154
:107740001297332727FD3095432F532F0E94D76B75
:10775000F701008110E00150104027812695277025
:10776000213071F0F801EE0FFF1FEE0FFF1F2230E6
:1077700069F5E55FF84F608371838283938334C03A
:1077800024E630E040E050E00E944B6CE22EC32E35
:10779000DA01000F111F000F111F055F184FF801CC
:1077A00020813181428153816E2D7C2DCD010E943B
:1077B000D76B20E034E040E050E00E944B6CD801F1
:1077C0002D933D934D935C9313970EC0E55FF84F57
:1077D0002081318142815381260F371F481F591F55
:1077E0002083318342835383B985BF5FB98708946F
:1077F000411C511CE4E0F0E06E0E7F1E22E030E000
:10780000220E331EB03209F049CD0E94830E8C0146
:10781000ED84E0FE05C0882319F48EE10E94D06B50
:10782000E1FE0BC0C80190708034910519F08834D6
:10783000910519F48FE10E94D06BE2FE0DC010702B
:107840000038110531F00838110519F0003911051B
:1078500019F480E20E94D06BB8EF4B2EB4E05B2E9F
:107860003F8D28A1832F922F9A8789872224332442
:10787000598A488AAB85BC85ED90FD900D911C918D
:10788000C801B70124E630E040E050E00E944B6CB4
:10789000EB85FC852083318342835383A889B98992
:1078A0002D933D93B98BA88BEE85FF85E35AFE4F50
:1078B00080819181EE85FF85E55AFE4F2081BAE0F7
:1078C0002B0260011124E8EEF3E0CE0EDF1EEE8500
:1078D000FF85E65AFE4F20812B0250011124A8E1BA
:1078E0004A2EACEF5A2EA40CB51C96014C2D232F1A
:1078F0008C159D0514F4482F292F842E922E8A145E
:107900009B040CF44501E114F1040105110569F132
:107910009401442737FD4095542F1E141F04100670
:10792000110654F4B601882777FD8095982F621BC5
:10793000730B840B950B0DC0C501AA2797FDA0956D
:10794000BA2F29013A01481A590A6A0A7B0AC30167
:10795000B201A80197010E94D76B20EA36E841E006
:1079600050E00E944B6C79018A01C4010E94AE185C
:107970003C01882477FC8094982C6E0C7F1C801E20
:10798000911EC6010E94AE188C01C5010E94AE185E
:10799000222717FD2095322F0615170528053905D2
:1079A00014F438014901AA2797FDA095BA2F840144
:1079B0007301681679068A069B0614F47C018D0112
:1079C000EE85FF85E45AFE4F8081882341F01095B3
:1079D0000095F094E094E11CF11C011D111DF2EAE8
:1079E000CF2EF1E0DF2EC20CD31CF601E358FD4F81
:1079F0008081882389F060E040E00E94561088234F
:107A000059F0F601E258FD4F80810E946E0E7C0114
:107A10000027F7FC0095102FF894A985BA85ED9200
:107A2000FD92BA87A9877894EB85FC853496FC870C
:107A3000EB87E2E04E2E512C240C351C2E853F8521
:107A40002B5F3F4F3F872E8730E22316310409F02A
:107A500011CF04C08F7009F09AC9C3C9A2960FB69E
:107A6000F894DEBF0FBECDBFCF91DF911F910F9174
:107A7000FF90EF90DF90CF90BF90AF909F908F904E
:107A80007F906F905F904F903F902F900895EF926E
:107A9000FF920F931F93DF93CF93CDB7DEB7C05400
:107AA000D0400FB6F894DEBF0FBECDBF8E010F5F82
:107AB0001F4FC80163E00E94E43381E2E82EF12CFD
:107AC000EC0EFD1EC70161E00E94E433EEEFF2E030
:107AD000418152816081D8012D913C91D7018D91D6
:107AE0009C911197662329F0B901681B790BCB0192
:107AF00002C0821B930B840F951F73E0883E97078B
:107B00002CF4ACEF89319A0724F005C088EE93E09D
:107B100002C088E19CEF9283818335960E5F1F4FF0
:107B200062E070E0E60EF71E73E0EE34F70781F6D0
:107B30008091860190E08170907022E030E0281BF7
:107B4000390B80E090E02817390721F0FC01EC5751
:107B5000FC4F1082019684309105A9F786E00E94BF
:107B60009C5581E00E94D06BC05CDF4F0FB6F8944B
:107B7000DEBF0FBECDBFCF91DF911F910F91FF9060
:107B8000EF9008952F923F924F925F926F927F9263
:107B90008F929F92AF92BF92CF92DF92EF92FF921D
:107BA0000F931F93DF93CF930F92CDB7DEB7009162
:107BB0008401102F1F700073813809F480C082384F
:107BC00090F4833209F447C0843230F48032E1F01B
:107BD000823209F086C04EC0813609F465C0803813
:107BE00009F07FC01BC0843811F1853838F4823821
:107BF00009F454C0833809F074C04AC0853811F1C3
:107C00008F3B09F06EC061C0153009F06AC08091E9
:107C1000A00491E089278093A00455C081E080935F
:107C20001B050E94B8140E94F71480E808C081E088
:107C300080931B0582EA9FE20E94F71484E80E9469
:107C400025604FC081E080931B0586EF98E40E9479
:107C5000F71485E8F4CF1F5F163008F010E0812F8D
:107C6000802B8093840181E00E949C5583E10E94D7
:107C7000D06B37C0112311F0115001C015E0812FD6
:107C8000802B8093840181E00E949C5584E1EFCF9A
:107C90008FEF98E10E94E71483E8D1CF8AE999E158
:107CA0000E94E71482E8CBCF80914106823021F414
:107CB00083E08093410607C0153099F402C00E940A
:107CC0000D2F0E941C1587E1D2CF81E00E94256014
:107CD00083E00E94256082E00E94256081E080931D
:107CE00031088091B60160E040E00E945610882380
:107CF00031F080913108882311F40E94473D809132
:107D0000B60160E040E00E945610809331080023E5
:107D100009F0B4C09091080180917101981710F496
:107D200096E001C094E0F2EAEF2EF1E0FF2E0AE0C7
:107D3000D7014D917D01802F60E024E099830E945E
:107D4000B85A055F9981083799F7492F406884E24E
:107D500060E10E94260F84E268E146E50E94775BBD
:107D600080914106882399F0823011F406E001C029
:107D700004E040914206509143068EE560E1202FD9
:107D80000E94A70E83E368E140E00E94CB0F84E2EB
:107D900060E146EF57E02091B40100E00E94A55B4E
:107DA0008091B3018F7031F089E360E142EF57E0D9
:107DB0000E94E95BEEE0EE2EE1E0FE2E70E0C72EC1
:107DC00071E0D72E662477246FE1962EF70101919A
:107DD0007F01D601ED91FD916D01808187FD8D5F61
:107DE00085958595843E0CF484EEA82E8D3114F093
:107DF0005CE1A52E862D81508230F8F4802F64E05E
:107E000046E30E946B5C2091860130E026253725F1
:107E100020FD04C08091B3018F7061F4802F8150E8
:107E20006EE143E00E946B5C802F8F5F6EE143E068
:107E30000E946B5C692D6A1914C0802F8B516BE313
:107E400046E30E94675C802E8A94882D6AE343E0B3
:107E50000E94675C882D6CE343E00E94675C0A0D1A
:107E60006BE3802F47E00E94CD180894611C711CC1
:107E7000B4E06B16710409F0A9CF27C080E060E080
:107E800042EA51E02AE001E10E947B5B9091080107
:107E900080917101981710F442E001C040E084E540
:107EA00060E00E94260F80914106882371F08230A5
:107EB00011F402E001C000E04091420650914306F7
:107EC0008FE660E0202F0E94A70E123008F085C0D8
:107ED0004EE1E42E45E0F42E00E039E1A32EB12C72
:107EE0002BE1922E90E2692E712C80E8482E512CC5
:107EF000F701219031907F01113011F1802F8370B3
:107F0000899DC02C1124D02ED694D694DD0CDD0C86
:107F1000DD0CF8E2DF0EC101B3010E94166C9B017B
:107F2000C101B2010E94166CAB01421B530B420D02
:107F3000531D8C2D8F5D6D2D20E20E945C5E48C02C
:107F4000043018F4B2E2CB2E02C0AEE5CA2E802F68
:107F50008370D82EDD0CDD0CD80E26E2D20EC101C6
:107F600037FE04C088279927821993098A9DA001AA
:107F70008B9D500D9A9D500D112440505E4F452F02
:107F8000550F550B45954595842E4A3114F0E9E17E
:107F90008E2E8C2D89516D2D43E325E50E94395C91
:107FA0006D2D62508C2D45E00E946B5C1214130401
:107FB00014F4C39401C0C8186D2D6F5F8C2D482D2B
:107FC0000E94675C6D2D61508C2D482D0E94675C6E
:107FD0000F5F083009F08CCF8AC0153008F07DC0E3
:107FE0000E94641F123061F0812F880F810F880F6B
:107FF0008950912F9150192F110F190F110F02C095
:1080000080E016E0C82E992787FD90952C01440C3E
:10801000551C480E591E60E2D62EEE24FF2452E075
:10802000852E912C880E991E3C011AC00E94C80F03
:108030005C018C2D60E040E00E945610082FA501E5
:10804000440D551D8AE06D2D23E00E947B5B089452
:10805000E11CF11C83E090E0480E591E98E0D90E17
:10806000C394C701860D971D88169906FCF6812FCB
:10807000992787FD90952C01440C551C480E591EDC
:1080800030E2D32EEE24FF2422E0822E912C880EA3
:10809000991E3C011AC00E94C80F5C01812F60E04C
:1080A00040E00E945610082FA501440D551D85E69D
:1080B0006D2D23E00E947B5B0894E11CF11CA3E082
:1080C000B0E04A0E5B1EB8E0DB0E1F5FC701860DF5
:1080D000971D88169906FCF60AC04091A20450919B
:1080E000A3048CE368E224E004E00E94A70E0F9052
:1080F000CF91DF911F910F91FF90EF90DF90CF9084
:10810000BF90AF909F908F907F906F905F904F90B7
:108110003F902F900895909118051816B4F4282FC9
:10812000332727FD3095291B3109462F50E0421790
:10813000530714F4982F07C04650504024173507B2
:108140002CF4982F9A5F961B01C090E0909318052D
:10815000892F0895AF92CF92DF92EF92FF920F9303
:108160001F93DF93CF930F92CDB7DEB7182F8EE713
:108170009BE00E94F8188BE898E0612F42E022ED26
:1081800037E00AE079E8E72E7BE0F72ECC2456E0D2
:10819000A52E0E946C1AF0908B088F2D67E00E942C
:1081A0008B4088E063E77BE00E94E15B31E08F2D4C
:1081B000813009F030E08091B80182958695877012
:1081C00090E0AC01440F551F480F591F440F551F35
:1081D0004C5A544F84E568E026E0032F39830E940F
:1081E0007B5B3981332399F06091B8016295669584
:1081F0006770812F40E024E00E949A148295880FD6
:10820000807E9091B8019F71982B9093B80180E186
:1082100069E47BE00E94E15B01E0EF2DE23009F0D0
:1082200000E084E560E14091B901202F0E942C0F0D
:10823000002349F0812F6091B90140E024E20E94BF
:108240009A148093B90188E16EE37BE00E94E15BC0
:108250004091BA01FF2DF33011F421E401C020E474
:1082600084E568E150E00E945C5E8F2D833049F424
:10827000812F6091BA0140E024E60E949A14809315
:10828000BA010091B80106950695017080E260E39D
:108290007BE00E94E15BCF2CDD24C7FCD09421E081
:1082A000E4E0CE16D10409F020E084E560E2402F3E
:1082B0000E943A1AFF2DF43079F4812F602F40E0AC
:1082C00021E00E949A148170880F880F9091B80164
:1082D0009B7F982B9093B8010091B8010695069565
:1082E0000695017088E262E27BE00E94E15B21E09A
:1082F00085E0C816D10409F020E084E568E2402F4B
:108300000E943A1AEF2DE53081F4812F602F40E072
:1083100021E00E949A148170880F880F880F909135
:10832000B801977F982B9093B8010091B8010295FE
:10833000017080E364E17BE00E94E15B21E0F6E014
:10834000CF16D10409F020E084E560E3402F0E94BD
:108350003A1A8F2D863079F4812F602F40E021E08A
:108360000E949A1481708295807F9091B8019F7EBF
:10837000982B9093B8010F90CF91DF911F910F919F
:10838000FF90EF90DF90CF90AF900895AF92BF92A3
:10839000CF92DF92EF92FF920F931F93DF93CF93D1
:1083A0000F92CDB7DEB7D82E80EE9CE00E94F81871
:1083B0008DE898E06D2D41E022ED37E00AE0A6EE71
:1083C000EA2EACE0FA2EFBE0CF2EE0E1AE2E0E94CA
:1083D0006C1A10918D08F0908E08812F67E00E9432
:1083E0008B40982F20916F0130E02F5F3F4F442743
:1083F00037FD4095542F8AE260E001E172E0E72EFC
:1084000099830E94265D99812D2D253451F02634C3
:1084100018F4243401F511C03D2D343671F0353691
:10842000D1F41130C1F4FF20B1F0809119058823F7
:1084300091F080918E0881500CC0113061F44F2D65
:10844000493048F480911905882329F080918E08DD
:108450008F5F80938E08992309F088C088E06BEDC8
:108460007CE00E94E15B113031F481E090E02091EA
:108470001905222311F080E090E0082F00618CE3C1
:1084800068E042EA51E02AE00E947B5B8091190596
:10849000882359F480911C0587FF07C081E08093F1
:1084A000190510921C0510928E08809119058823D9
:1084B00081F020911C05332727FD30958F2D90E00A
:1084C0008217930734F41092190510921C0510922C
:1084D0008E08113009F058C480911905882309F4D9
:1084E00053C480918E0890911C05891B80938E083F
:1084F00087FF02C010928E0880918E088A301CF08F
:1085000089E080938E0810921C05AF2CBB24F501E6
:10851000EE55FE4F80810E94392C682F20919A04DD
:1085200030919B042115310549F47D2D723631F0CF
:10853000733621F0723411F0733431F48D2D40E034
:1085400021E40E949A14682F862F0E94492C482FFC
:10855000F501EE55FE4F80838F2D880F8F0D880F0C
:10856000845C68E021E00E94B85A0EC4923008F0A2
:1085700079C0B8E0EB2E8E2D65ED7CE00E94E15BCA
:108580004091AF015091B001123099F4FF2039F4BD
:1085900080911905882309F0FAC321E0F9C38F2DD2
:1085A000813039F480911905882329F020E002E018
:1085B00004C020E0EDC320E001E087E46E2D0E94BE
:1085C000A70E123009F04BC080911905882339F4A9
:1085D00080919A0490919B04009709F440C0809187
:1085E000AF019091B0016CE370E00E94026C082F23
:1085F000FF2021F09F2D913091F515C08D2D40E089
:108600002BE30E949A142CE3482F4203900111247B
:10861000802F992787FD9095280F391F3093B0013F
:108620002093AF011CC00E5F8D2D602F41E02EE323
:108630000E949A14081B602F772767FD7095209180
:10864000AF013091B001261B370B3093B00120935E
:10865000AF0137FF04C01092B0011092AF010E2D90
:10866000085F03C0923019F508E0802F6DEC7CE0C4
:108670000E94E15B91E0133009F090E08CE3602F01
:10868000492F99830E94CB0F9981992349F08D2D11
:108690006091AD0147EC29E30E949A148093AD01EB
:1086A000A8E0EA2EE00E6E2D693328F073C39330F4
:1086B00069F5F8E0EF2E8E2D66EC7CE00E94E15B20
:1086C00091E0143009F090E02091AE0121708CE32C
:1086D0006E2D40EB5CE0092F99830E94A55B998188
:1086E000992379F06091AE0161708D2D40E021E019
:1086F0000E949A1481709091AE019E7F982B909366
:10870000AE010E2D085F093320F044C3943031F5DB
:1087100008E0E090B3017FE0E722802F69EA7CE087
:108720000E94E15B21E0153009F020E08CE3602F2E
:108730004E2D0E942B1A153069F48D2D6E2D40E0C0
:1087400021E00E949A148F709091B301907F982B32
:108750009093B301085F093320F01CC3953059F59D
:1087600008E0E090B301E294EFE0EE22802F62EAAD
:108770007CE00E94E15B21E0163009F020E08CE310
:10878000602F4E2D0E942B1A163071F48D2D6E2DF8
:1087900040E021E00E949A148295807F9091B3017D
:1087A0009F70982B9093B30178E0E72EE00E8E2D0A
:1087B000893328F0EFC2963031F568E0E62E8E2D31
:1087C00069E97CE00E94E15B91E0173009F090E0FC
:1087D0008CE36E2D49E75CE02091B401092F998369
:1087E0000E94A55B9981992349F08D2D6091B40178
:1087F00040E024E00E949A148093B4010E2D085F9B
:10880000093320F0C7C2973029F508E0802F61E7CF
:108810007CE00E94E15B91E0183009F090E086E393
:10882000602F4091B601292F99830E94780F99817A
:10883000992349F08D2D6091B6014AEE26E10E9400
:108840009A148093B60158E0E52EE00E9E2D9933E0
:1088500030F0A0C2983009F053C048E0E42E8E2DCD
:1088600068E67CE00E94E15B9CE3AA24BB24A501AE
:10887000405A534FFA1411F4193061F02091B701A6
:1088800030E00A2C02C0359527950A94E2F7022FB2
:10889000017001C002E0892F6E2D21E099830E94B2
:1088A0007B5B0894A11CB11C99819A5F9636F9F6FE
:1088B000193001F5ED2DE03631F080919A04909158
:1088C0009B040097B9F08D2D0E9425601092190528
:1088D00081E090E00F2C02C0880F991F0A94E2F704
:1088E0002091B70128272093B70182E00E949C5570
:1088F0000E943856F8E0EF0E2E2D293330F04AC290
:10890000993009F0E2C038E0E32E8E2D6AE57CE074
:108910000E94E15B4091B10186E0489FA0011124D3
:108920004F5B534F1A3041F4FF2031F48091190509
:10893000882321F002E003C000E001C001E084E2EE
:108940006E2D26E00E947B5B8091B101882321F08F
:10895000833009F046C009C086E66E2D4CE35CE02A
:1089600020E00E94BA5B9CE308C082E76E2D49E3D9
:108970005CE020E00E94BA5B98E42091B2012E5F97
:108980001A3049F43F2D313031F480911905882394
:1089900021F002E003C000E001C001E0892F6E2D4C
:1089A0004BE15CE099830E94A55B9981892F865DEC
:1089B0004091B50192E34902A0011124445D5E4F4C
:1089C0001A3049F46F2D623031F4909119059923D2
:1089D00021F022E003C020E001C021E06E2D0E94C2
:1089E0005C5E8091B101813001F582E46E2D44E13D
:1089F0005CE020E00E94BA5B4091B201552747FD40
:108A000050954F5F5F4F1A3049F47F2D713031F42C
:108A100080911905882321F022E003C020E001C0E5
:108A200021E08EE76E2D0E945C5E1A3009F046C090
:108A300080911905882331F480919A0490919B04C8
:108A40000097E1F10091B1018F2D813071F08130FB
:108A500018F0823069F51FC08D2D602F40E023E0B3
:108A60000E949A148093B10123C0002311F00330B7
:108A700031F48D2D6091B2014EEF24E007C001303A
:108A8000B9F48D2D6091B20140E02CE70E949A1458
:108A90008093B2010DC0002311F0033049F48D2DF5
:108AA0006091B5014CEF2AE00E949A148093B501C1
:108AB0008091B101801711F01092B20128E0F22EDE
:108AC000FE0C9F2D993330F065C19A3009F07CC0BF
:108AD00098E0F92E8091B101882311F0833019F5C7
:108AE0008F2D65E07CE00E94E15B4091BB0185E059
:108AF0004802A00111244F515F4F1B3011F421E2B5
:108B000001C020E28EE46F2D0E945C5E1B3009F0F4
:108B100055C08D2D6091BB014CEE24E10E949A144A
:108B20008093BB014BC08130B9F401E01B3009F0E8
:108B300000E080E06F2D4FEE5BE0202F0E94BA5BDB
:108B40000023E1F1ED2DE038C9F581E08093670E57
:108B500080E00E94D06B32C08F2D66EE7BE00E94D9
:108B6000E15B8091B20187FD03C083301CF403C038
:108B700080E001C082E08093B20149E08402A0015C
:108B800011244653544F1B3031F48091190588232A
:108B900021F002E003C000E001C001E08CE36F2D92
:108BA00029E00E947B5B1B3049F48D2D6091B2015E
:108BB00040E022E00E949A148093B201F8E0FF0E98
:108BC0002F2D293328F0E6C09B30A9F588E0F82E38
:108BD0008F2D60EC7BE00E94E15B31E01C3009F0FE
:108BE00030E08091B801817090E0AC01440F551FD6
:108BF000480F591F4754544F8CE36F2D23E0032F28
:108C000039830E947B5B3981332379F06091B8010D
:108C100061708D2D40E021E00E949A148170909146
:108C2000B8019E7F982B9093B80138E0F30E4F2D3A
:108C3000493328F0AFC09C3051F5B8E0FB2E0091CD
:108C4000B801069501708F2D6FEA7BE00E94E15B11
:108C500021E01D3009F020E08CE36F2D402F0E94B1
:108C60002B1A1D3071F48D2D602F40E021E00E9401
:108C70009A148170880F9091B8019D7F982B9093E2
:108C8000B80168E0F60E7F2D793328F083C09D305F
:108C900051F5A8E0FA2E0091AE01069501708F2DD6
:108CA00067EA7BE00E94E15B21E01E3009F020E0F2
:108CB0008CE36F2D402F0E942B1A1E3071F48D2DE6
:108CC000602F40E021E00E949A148170880F9091FB
:108CD000AE019D7F982B9093AE0188E0F80E9F2DFA
:108CE000993328F057C09E3059F5F8E0FF2E0091D7
:108CF000AE010695069501708F2D6EE97BE00E940E
:108D0000E15B21E01F3009F020E08CE36F2D402F64
:108D10000E942B1A1F3079F48D2D602F40E021E046
:108D20000E949A148170880F880F9091AE019B7FEA
:108D3000982B9093AE016F2D685F693320F02AC0A5
:108D40009F3041F568E080911A05882319F421E0ED
:108D5000103109F020E080E04AE85BE00E94BA5B55
:108D60001031C1F4ED2DE038A9F41092190589E114
:108D700080931A0580E80E9425601092350680E2F3
:108D80009FE20E94F71406C0E0E1EE2EF4CB22E051
:108D900000E013CC0F90CF91DF911F910F91FF90C6
:108DA000EF90DF90CF90BF90AF9008958F929F92F9
:108DB000AF92BF92CF92DF92EF92FF920F931F93E9
:108DC000CF93DF93B82E8CE39FE00E94F81883EADC
:108DD00098E06B2D47E022ED37E00AE05CE4E52EF9
:108DE0005FE0F52ECC24C3941CE0A12E0E946C1AE7
:108DF0008090A3088A94D090A408882D66E00E94F1
:108E00008B40C82E18E0992487FC90948C2D8C30D0
:108E100009F43CC1EC2CFF248E149F0439F480919A
:108E20001905882329F0B2E0AB2E04C0AA2402C0A1
:108E3000AA24A39480E0612F49E35FE022E000E0F0
:108E40000E947B5BEC2DE93010F048E301C041E368
:108E50004C0D8CE0612F0E94775BF701EE0FFF1F36
:108E6000EE0DFF1DE650FC4F4081F7E04F9FA00143
:108E700011244A52514FDD2011F000E001C00A2DAB
:108E800088E1612F27E00E947B5BC701880F991F53
:108E90008E0D9F1D8E559E4FFC01E85AFD4F20817F
:108EA000253008F4E4C0FC01EA5AFD4F283008F4EC
:108EB000E7C040818D2D8130D1F53BC020E001C05D
:108EC0002A2D88E4612F0E942C0FF701EE0FFF1F5F
:108ED000EE0DFF1DE750FC4F4081552747FD509593
:108EE000ED2DE23011F020E001C02A2D88E7612F3E
:108EF0000E945C5E00E035C020E001C02A2D88E4BD
:108F0000612F0E94780FF701EE0FFF1FEE0DFF1D7E
:108F1000E750FC4F4081FD2DF23011F020E001C000
:108F20002A2D80E6612F0E94780F01E01AC020E010
:108F300001C02A2D88E4612F0E942C0FF701EE0F4B
:108F4000FF1FEE0DFF1DE750FC4F40818D2D82303D
:108F500011F020E001C02A2D86E6612F0E942C0F1F
:108F600002E080911905882339F480919A04909148
:108F70009B04009709F475C0AA2009F472C0ED2D76
:108F8000E130B1F1E13020F0E23009F06AC042C0D6
:108F9000E701CC0FDD1FCE0DDF1DC650DC4F8B2D42
:108FA000688140E02DE00E949A148883202F30E0F1
:108FB000853028F0883030F481E090E005C080E012
:108FC00090E002C082E090E02817390709F449C018
:108FD000C701880F991F8E0D9F1D8E559E4FFC0156
:108FE000EA5AFD4F1082895A9D4FFC01108239C008
:108FF000013041F0E701CC0FDD1FCE0DDF1DC85061
:10900000DC4F28C0E701CC0FDD1FCE0DDF1DC8509F
:10901000DC4F17C0013071F0E701CC0FDD1F0230CB
:10902000A9F0CE0DDF1DC750DC4F8B2D688143E8C2
:109030002DE714C0E701CC0FDD1FCE0DDF1DC7509B
:10904000DC4F8B2D68814AEE26E108C0CE0DDF1D76
:10905000C750DC4F8B2D688140E024E20E949A14B7
:109060008883C394185F103409F0D0CE0FC08A5A99
:109070009D4FFC014081FD2DF13009F01FCF20CF25
:1090800040818D2D813009F037CF38CFDF91CF91DE
:109090001F910F91FF90EF90DF90CF90BF90AF9016
:1090A0009F908F9008956F927F928F929F92AF9230
:1090B000BF92CF92DF92EF92FF920F931F93CF93C5
:1090C000DF93982E8EE49FE00E94F81885EA98E0DE
:1090D000692D48E022ED37E00AE0AEE5EA2EAFE088
:1090E000FA2ECC24C394F0E1AF2E0E946C1A60904B
:1090F000A5086A948090A608862D66E00E948B40A1
:10910000E82EE8E0FE2E772467FC70948E2D8031E7
:1091100009F45DC0AE2CBB24E39480E06F2D4E2D8E
:1091200020E00E94580FDD24E501CC0FDD1FC05E5A
:10913000DB4F8501000F111F015E1B4F6A147B047A
:1091400071F48D1461F480911905882359F480918C
:109150009A0490919B04009739F421E001C020E02B
:10916000CC2405C022E001C021E0CC24C394DD2042
:1091700091F48EE16F2DF80140810E94780FCC2090
:10918000D9F0892DF80160814AEE26E10E949A14F7
:10919000F801808311C04881552747FD509580E62E
:1091A0006F2D0E945C5ECC2039F0892D688143E8E8
:1091B0002DE70E949A148883D394FD2DF33009F093
:1091C000BDCF88E0F80EEF2DE03409F09FCFDF919E
:1091D000CF911F910F91FF90EF90DF90CF90BF90B4
:1091E000AF909F908F907F906F9008958F929F92F5
:1091F000AF92BF92CF92DF92EF92FF920F931F93A5
:10920000DF93CF9300D0CDB7DEB7182F80919101B7
:10921000813019F048E1F42E02C03AE1F32E2BEF31
:10922000B22EBF0C87E19AE00E94F81882E498E021
:10923000612F40E026EE37E006E0EF2C0E94E71DAC
:10924000E0904208C09043088E2D67E00E948B405A
:10925000D82E8F2D90E04D2D50E09C0127503040AE
:109260004217530751F42E2D30E004972817390781
:1092700014F48FEF01C081E0D80E113629F11236B7
:1092800078F4143409F448C0153420F4123408F486
:109290006AC063C0153419F1103609F064C009C002
:1092A000143608F45AC01436B9F1153609F05BC00B
:1092B00016C0EE2009F457C081E090911905911174
:1092C00080E0809319054FC080911905882309F427
:1092D0004AC01092190581E60E94256044C02E2DD7
:1092E000213059F4CC2049F080911905882329F0C8
:1092F000809143088150809343082E2D30E08B2DC0
:10930000992787FD90952817390769F5CC2059F1E1
:109310008091430881501EC03E2D313061F48C2D68
:10932000893048F480911905882329F080914308F9
:109330008F5F809343082E2D30E08B2D992787FD7A
:1093400090952817390779F49C2D973060F4809117
:1093500043088F5F8093430806C0809119058823D6
:1093600011F410924308DD2009F089C088E06CE018
:109370007AE00E94E15BEE2DE13031F481E090E093
:1093800020911905222311F080E090E0082F006160
:1093900082E468E043E951E02AE00E947B5B80912F
:1093A0001905882359F480911C0587FF07C081E0C7
:1093B0008093190510921C0510924308809119059D
:1093C000882381F020911C05332727FD30958C2DB3
:1093D00090E08217930734F41092190510921C053F
:1093E00010924308FE2DF13009F078C480911905E0
:1093F000882309F473C48091430890911C05891B4C
:109400008093430887FF02C010924308809143086D
:109410008A301CF089E08093430810921C05AC2C24
:10942000BB24F501ED56FE4F80810E94392C682F38
:1094300020919A0430919B042115310541F4123694
:1094400031F0133621F0123411F0133431F4812F3E
:1094500040E021E40E94A914682F862F0E94492C25
:10946000482FF501ED56FE4F80838C2D880F8C0D13
:10947000880F8E5B68E021E00E94B85A2FC42D2D22
:10948000223090F598E0F92EB0908501B694B6940C
:10949000B69437E0B3228F2D65E07AE00E94E15B5D
:1094A00091E08E2D823009F090E08CE56F2D49ED32
:1094B00059E02B2D092F9A830E94A55B9A8199234D
:1094C00081F0812F6B2D40E026E00E94A914877067
:1094D000880F880F880F90918501977C982B909327
:1094E000850198E0F90E05C0ED2DE23041F588E0E8
:1094F000F82EB09091018F2D6EEC79E00E94E15B27
:1095000091E0FE2DF33009F090E08CE56F2D40ECFA
:1095100059E02B2D092F9A830E94A55B9A819923EC
:1095200041F0812F6B2D40E021E00E94A91480932F
:10953000910128E0F20E3F2D393318F0D2C308E034
:10954000F02E80919101813039F58D2D843030F5E8
:109550008F2D62EB79E00E94E15B40918F019E2D9F
:10956000943011F421E401C020E486E66F2D50E030
:109570000E945C5EEE2DE43049F4812F60918F01F2
:1095800041E024E60E94A91480938F01F8E0FF0EC9
:109590002F2D293318F0A5C304E001C005E0809108
:1095A00091018150823028F5D01610F58F2D62EA96
:1095B00079E00E94E15B40919001E01611F421E412
:1095C00001C020E486E66F2D50E00E945C5EE0164C
:1095D00049F4812F6091900140E025E00E94A91498
:1095E0008093900138E0F30E8F2D893308F079C312
:1095F0000F5FD01620F58F2D69E979E00E94E15BBD
:1096000040917001E01611F421E401C020E486E6E7
:109610006F2D50E00E945C5EE01659F4812F60913E
:1096200070014AE02DE20E94A914809370010E940B
:10963000BC5E98E0F90EEF2DE93308F052C3B02E6E
:10964000B394DB1408F58F2D69E879E00E94E15BA3
:1096500040917101EB1411F421E401C020E486E68D
:109660006F2D0E94120FEB1449F4812F609171014C
:1096700048E228E70E94A91480937101F8E0FF0EE8
:109680002F2D293308F02DC3B394DB1460F58F2DF3
:1096900068E779E00E94E15B40918701552747FD2B
:1096A0005095465F5F4FEB1411F421E401C020E4B4
:1096B00086E66F2D0E945C5E8091A30D6F2D4DE6B6
:1096C0000E94775BEB1449F4812F6091870146EF8C
:1096D0002EE60E94A9148093870138E0F30E8F2DA7
:1096E000893308F0FEC2B394DB1420F58F2D6DE6AC
:1096F00079E00E94E15B91E0EB1090E086E66F2D4F
:109700004FE559E020918901092F9A830E94A55BBA
:109710009A81992349F0812F6091890140E022E0EC
:109720000E94A9148093890198E0F90EEF2DE93386
:1097300008F0D7C2B394DB14C8F48091880181701B
:1097400021E0EB1020E06F2D4EE459E0012F0E9444
:10975000532C8170909188019E7F982B9093880163
:10976000F8E0FF0E2F2D293308F0BBC2B394DB14B1
:10977000D8F4809188018695817021E0EB1020E07B
:109780006F2D42E459E0012F0E94532C8170880F05
:10979000909188019D7F982B9093880138E0F30E7B
:1097A0008F2D893308F09DC2B394DB14E8F48091C7
:1097B000880186958695817021E0EB1020E06F2D61
:1097C00043E359E0012F0E94532C8170880F880FCA
:1097D000909188019B7F982B9093880198E0F90ED7
:1097E000EF2DE93308F07DC2B394DB14F8F48091D7
:1097F0008801869586958695817021E0EB1020E0A2
:109800006F2D45E259E0012F0E94532C8170880F83
:10981000880F880F90918801977F982B90938801EB
:10982000F8E0FF0E2F2D293308F05BC2B394DB1450
:1098300000F58F2D68E179E00E94E15B01E0EB101B
:1098400000E080E66F2D40917301202F0E94780F79
:10985000002349F0812F609173014AEE26E10E94B6
:10986000A9148093730138E0F30E8F2D893308F02B
:1098700038C2B39400E0DB1408F047C0002319F4A9
:1098800068E079E002C068EF78E08F2D0E94E15B2C
:10989000002319F4A0908A0102C0A0909201AA208E
:1098A000A9F09A2DE5E09E9FA0011124EB1411F47C
:1098B00021E401C020E486E66F2D0E945C5E809169
:1098C000A30D6F2D43E70E94775B09C021E0EB10E9
:1098D00020E086E66F2D40EF54E00E94BA5BEB1467
:1098E00039F4812F6A2D40E028E70E94A914A82EA0
:1098F000002319F4A0928A0102C0A0929201F8E01C
:10990000FF0E2F2D293308F0ECC1B3940F5F023006
:1099100009F0B1CFDB14F8F48091880182958F7043
:109920008095817021E0EB1020E06F2D4AEE58E029
:10993000012F0E94532C809581708295807F909199
:1099400088019F7E982B9093880138E0F30E8F2D2D
:10995000893308F0C6C1B394DB14F8F480918E010A
:1099600082958F708095817021E0EB1020E06F2D43
:109970004EED58E0012F0E94532C80958170829506
:10998000807F90918E019F7E982B90938E0198E01E
:10999000F90EEF2DE93308F0A4C1B394DB14D8F429
:1099A000809185018095817021E0EB1020E06F2D82
:1099B0004DEC58E0012F0E94532C809581709091BE
:1099C00085019E7F982B90938501F8E0FF0E2F2D47
:1099D000293308F086C1B394DB14E8F48091850143
:1099E00086958095817021E0EB1020E06F2D4EEB85
:1099F00058E0012F0E94532C80958170880F909120
:109A000085019D7F982B9093850138E0F30E8F2D73
:109A1000893308F066C1B394DB1408F086C08F2D3B
:109A200063EB78E00E94E15B92E488249924A4012E
:109A30004A58574FE0919D01F0E0082C02C0F5957F
:109A4000E7950A94E2F7E170F070892F6F2D21E01D
:109A50000E2F9A830E947B5B0894811C911C9A8133
:109A60009A5F923721F7EB1409F059C080914308AF
:109A700090911C05891B8093430887FF02C01092B8
:109A80004308809143088A301CF089E080934308A2
:109A900010921C058C2D880F8C0D880F4C2D50E0DA
:109AA0004A58574F8E5B6F2D21E002E00E947B5B8E
:109AB000103631F080919A0490919B04009779F1CF
:109AC000812F0E9425601092190581E090E002C06C
:109AD000880F991FCA94E2F790919D01982790935F
:109AE0009D01803151F0803271F0883099F493FFFC
:109AF00002C09F7C0DC098600BC094FF02C0977D90
:109B000007C0906105C095FF02C0977E01C09062BA
:109B100090939D0181E00E949C550E94385698E0E8
:109B2000F90EEF2DE93308F0DCC0B394DB14F8F440
:109B300080918501869586958095817021E0EB1056
:109B400020E06F2D44EA58E0012F0E94532C8095AD
:109B50008170880F880F909185019B7F982B90933F
:109B60008501F8E0FF0E2F2D293308F0BAC0B39419
:109B7000DB1400F590918501991F9927991F81E0C9
:109B8000891B21E0EB1020E06F2D46E958E0012F02
:109B90000E94532C80958795882787959091850101
:109BA0009F77982B9093850138E0F30E8F2D8933A2
:109BB00008F097C0B394DB1408F580918801829572
:109BC000869587708095817021E0EB1020E06F2DE5
:109BD0004CE858E0012F0E94532C809581708295AB
:109BE000880F807E909188019F7D982B90938801AB
:109BF00098E0F90EEF2DE93308F073C0B394DB144D
:109C000018F5809188018295869586958370809558
:109C1000817021E0EB1020E06F2D44E858E0012F27
:109C20000E94532C809581708295880F880F807CCC
:109C3000909188019F7B982B90938801F8E0FF0E0C
:109C40002F2D293308F04DC0B394DB1408F049C020
:109C500086E06F2D4FE758E00E94E95B3F2D3833D7
:109C600090F434E290E0832F6F2D47E857E0292FDE
:109C700000E039839A830E94595A9A819F5F398103
:109C8000385E943081F788E0F80E9F2D993348F5BF
:109C9000DD24D394EB10DD24409186014F5C82E1FA
:109CA0006F2D2D2D0E94B85A94E200E00F5F892F8E
:109CB0006F2D402F20E09A830E942C0F9A81985E8E
:109CC0000430A1F7DD2069F0812F6091860140E02A
:109CD00023E00E94A9148093860103C0B0E1FB2E0B
:109CE000D3CB0F900F90CF91DF911F910F91FF90E9
:109CF000EF90DF90CF90BF90AF909F908F9008959E
:109D00008F929F92AF92BF92CF92DF92EF92FF928B
:109D10000F931F93DF93CF930F92CDB7DEB7C82E6B
:109D200087E89FE00E94F81887EA98E06C2D49E0E8
:109D300022ED37E00AE0FAE0EF2E0E94E71D1091D5
:109D4000A7081150812F66E00E948B40D82E2C2D41
:109D5000203899F480E80E94256089E180931A05F3
:109D6000193019F40E94E46005C0183018F4812FEE
:109D70000E94566181E00E94D06BE8E0FE2EA12E89
:109D8000BB24A7FCB0943D2D383021F48F2D8933AE
:109D900090F180C08D2C992494012F5F3F4F442770
:109DA00037FD4095542FA814B90411F401E101C006
:109DB00000E182E16F2D72E0E72E0E94265DF40142
:109DC000EE0FFF1FEB5FF54E85919491AC018091F2
:109DD0001A05882321F421E0A814B90409F020E031
:109DE00088E16F2D0E94BA5BE8E0FE0ED394FF2D50
:109DF000F03449F64FC080911A05882321F4DD2400
:109E0000D394183009F0DD2486E06F2D49E75FE038
:109E10000E94E95B9AE556E0A52EB12CE0918B01FA
:109E2000F0E0E852FB4F449150E00A2C02C05595F7
:109E300047950A94E2F7437050704C58504F892F61
:109E40006F2D21E00D2D99830E947B5B2EEF3FEF5C
:109E5000A20EB31E99819A5F923701F7DD2049F077
:109E60008C2D60918B0140E027E10E94A914809322
:109E70008B016F2D685F693368F480911A05882320
:109E800019F421E0193009F020E086E040E65FE0B7
:109E90000E94BA5B0F90CF91DF911F910F91FF90BD
:109EA000EF90DF90CF90BF90AF909F908F900895EC
:109EB0004F925F926F927F928F929F92BF92CF92BA
:109EC000DF92EF92FF920F931F93DF93CF9300D017
:109ED000CDB7DEB7182F85EC9FE00E94F8188BEB0A
:109EE00098E0612F46E022ED37E00AE050E1E52EF0
:109EF0000E94E71D6090BB086A94862D66E00E9470
:109F00008B40103611F0143641F467FC06C06092A5
:109F1000A0088AE891E30E94F714CC24DD24EE2403
:109F2000E39418E0F12E772467FC709430911805C3
:109F30003C0DBB24B394383028F4BB248E2D8830DC
:109F400028F074C09E2D973008F070C0032F10E0E9
:109F500091E06016710609F090E0DD2019F0DD2433
:109F6000D39401C0D92E80E06F2D42EC5FE0292F01
:109F70003A8399830E94BA5B3A819981393010F40F
:109F800082E101C087E1A8014F5F5F4F6F2D292F4C
:109F90000E945C5EBB2079F0085010402801B3E0BD
:109FA000440C551CBA95E1F7400E511EE0EBF3E06E
:109FB0004E0E5F1E0BC02801440C551C440C551C52
:109FC000400E511E88E893E0480E591E42010AE2F5
:109FD000F40141914F01552747FD5095802F6F2D7A
:109FE00020E00E945C5E0B5E033991F7F8E0FF0E03
:109FF000E394BB20B1F085E090E0480E591E0AE2E0
:10A00000F20141912F01552747FD5095802F6F2D6B
:10A0100020E00E945C5E0B5E0E3791F7F8E0FF0EC9
:10A02000E394C3948C2D873009F080CFDD2029F490
:10A03000809118058F5F809318050F900F90CF9136
:10A04000DF911F910F91FF90EF90DF90CF90BF9025
:10A050009F908F907F906F905F904F900895BF92E8
:10A06000CF92DF92EF92FF920F931F93CF93DF93E4
:10A07000F82E81EA98E06F2D4DE00E94581F8091E4
:10A080009908882319F08AEC9EE002C080EC9EE0DB
:10A090000E94F818182F80919A080E948B0EEC01EC
:10A0A000812F8A5F60E0488120E00E94580FC090B5
:10A0B000A1088C2D66E00E948B4018E0EE24DD2480
:10A0C000C7FCD094209118052E0D822F90E0BB2460
:10A0D000B394C816D90609F0BB24263009F4F3C09E
:10A0E000273090F4223009F457C0233030F4222373
:10A0F00009F1213009F0DAC134C0243009F495C0E7
:10A10000253008F0B3C069C02A3009F45DC12B3096
:10A1100038F4283009F419C1293008F036C1EAC0F2
:10A120002C3009F48EC12C3008F46CC12D3009F0AC
:10A13000BDC1A4C18CE0612F49EB5EE00E94E95BE8
:10A1400084E5612F49812B2D0E942C0FBB2009F43F
:10A15000ADC18F2D698141E024E20E949A14898368
:10A16000A5C18CE0612F42EB5EE00E94E95B4A8171
:10A17000552747FD50952B2D206484E5612F0E94C3
:10A180005C5EBB2009F492C18F2D6A8143E82DE704
:10A190000E949A148A838AC18F8186FF03C048EA8D
:10A1A0005EE002C041EA5EE08CE0612F0E94E95B64
:10A1B0004885552747FD50952B2D206484E5612F58
:10A1C0000E945C5EBB2009F471C18F2D688543E855
:10A1D0002DE70E949A14888769C10F810295069520
:10A1E000069501708CE0612F46E95EE00E94E95B14
:10A1F000002319F044EF54E002C040EF54E084E53E
:10A20000612F2B2D0E94BA5BBB2009F44FC18F2D0B
:10A21000602F40E021E00E949A1481708295880F9F
:10A22000880F807C9F819F7B8DC08CE0612F41E9EE
:10A230005EE00E94E95B8F8180FF03C044EF54E041
:10A2400002C040EF54E084E5612F2B2D0E94BA5BE1
:10A25000BB2009F42BC16F8161708F2D40E021E09C
:10A260000E949A1481709F819E7F6CC08CE0612F48
:10A270004AE85EE020E00E94BA5B4C8183E0489FA0
:10A28000A00111244651504F84E5612F23E00B2D8E
:10A290000E947B5BBB2009F409C18F2D6C8140E0DB
:10A2A00026E10E949A148C83873008F4FFC09F2D0A
:10A2B000903609F0FBC087508093A0088AE891E3AC
:10A2C0000E94F714F3C08CE0612F43E85EE00E9427
:10A2D000E95B8EE4612F4B812B2D0E94780FBB2010
:10A2E00009F4E4C08F2D6B814AEE26E10E949A1496
:10A2F0008B83DCC08CE0612F4BE75EE00E94E95B62
:10A300000F810295037049F02B2D206484E5612FA5
:10A31000402F50E00E945C5E07C084E5612F40EF53
:10A3200054E02B2D0E94BA5BBB2009F4BFC08F2DD7
:10A33000602F40E023E00E949A1483708295807F12
:10A340009F819F7C982B9F83B1C08CE0612F44E755
:10A350005EE00E94E95B2F812695277084E5612FDE
:10A360004AE55EE00B2D0E94A55BBB2009F49EC070
:10A370006F81669567708F2D40E022E00E949A14ED
:10A380008770880F9F81917FDDCF8CE0612F4FE434
:10A390005EE00E94E95B4D8142954F7080E6612F3F
:10A3A00050E02B2D0E945C5EBB2009F47FC06D81C4
:10A3B00062956F708F2D40E02FE00E949A14829575
:10A3C000807F9D819F701BC08CE0612F46E45EE022
:10A3D0000E94E95B4D814F7080E6612F50E02B2D8C
:10A3E0000E945C5EBB2009F461C06D816F708F2D8F
:10A3F00040E02FE00E949A148F709D81907F982BEF
:10A400009D8354C08CE0612F4BE35EE00E94E95BCA
:10A410004E8142954F7080E6612F50E02B2D0E94B7
:10A420005C5EBB2009F442C06E8162956F708F2D17
:10A4300040E02FE00E949A148295807F9E819F7059
:10A440001AC08CE0612F42E35EE00E94E95B4E811E
:10A450004F7080E6612F50E02B2D0E945C5EBB2088
:10A4600029F16E816F708F2D40E02FE00E949A14C9
:10A470008F709E81907F982B9E8318C08CE0612FF7
:10A4800040E25EE02B2D0E94BA5BBB2079F08F2D5D
:10A49000803861F40E94256080919A080E941621FC
:10A4A00081E00E94D06B80E00E94C214E394185FA8
:10A4B0009E2D973009F006CEDF91CF911F910F911D
:10A4C000FF90EF90DF90CF90BF9008955F926F92D2
:10A4D0007F928F929F92AF92BF92CF92DF92EF9234
:10A4E000FF920F931F93CF93DF93D82E89EA9FE0BB
:10A4F0000E94F81889EB98E06D2D45E022ED37E0D9
:10A500000AE050EBE52E5FE0F52E11E1C12EB1E13E
:10A51000AB2E0E946C1AF090B908FA94A090BA0879
:10A520008F2D66E00E948B40C82E2D2D203809F516
:10A530008F2D8031F0F4EF2DFF27E7FDF095EC191A
:10A54000F109EE0FFF1FE25EFA4FC081D1810E9438
:10A550009B0EFC01AA2069F48281882319F0D09512
:10A56000C195DF4FD483C38382E00E949C550E9433
:10A57000385618E0552453946F2C772467FC709458
:10A580002C2D203109F4DFC08C2D0E949B0EEC0194
:10A590004A812B813C81442319F0309521953F4F0E
:10A5A0008C2C9924F401EE0FFF1FE25EFA4F80819C
:10A5B0009181821B930B8333910524F0F401E755BD
:10A5C000F74F08C02FEF8E3C92072CF4F401E755AB
:10A5D000F74F45254083C39480E0612F4C2D20E048
:10A5E0000E94580FF401E755F74F8081882311F03E
:10A5F0004FE701C04EE78BE4612F20E00E94B85A7C
:10A60000EE246814790471F4AE1461F48091190594
:10A61000882359F480919A0490919B04009739F40F
:10A6200001E001C000E0BB2405C002E001C001E080
:10A63000BB24B3948E2D823009F43FC0833009F4DB
:10A640005DC08130C1F04B815C81202F206280E3AE
:10A65000612F0E945C5EBB2009F46BC06B817C8122
:10A660008D2D48E15CEF28EE33E002E00E94D61326
:10A670009C838B835EC048814456552747FD509587
:10A6800088E4612F202F0E945C5EBB2009F451C03A
:10A690006881645668838091B80181FF04C08D2D64
:10A6A00043E82DE703C08D2D4CE924E60E949A145F
:10A6B000888388818C5988833CC049814C595527AF
:10A6C00047FD509586E6612F202F0E945C5EBB20DF
:10A6D00081F169816C5969838091B80181FF04C05F
:10A6E0008D2D43E82DE703C08D2D4CE924E60E9413
:10A6F0009A1489838981845689831BC08A8190E05A
:10A70000AC01440F551F480F591F4E55504F8CE652
:10A71000612F23E00E947B5BBB2059F08D2D6A8165
:10A7200040E021E00E949A1491E0882309F490E02F
:10A730009A83E3942E2D243009F063CF185F1034F0
:10A7400009F01ECF1FC001E08F2D803109F000E01D
:10A7500080911A05882311F020E001C0202F82E1AA
:10A76000612F41E95FE00E94BA5B002359F02D2D73
:10A77000203841F489E180931A0580E80E94256021
:10A780000E94473DDF91CF911F910F91FF90EF9075
:10A79000DF90CF90BF90AF909F908F907F906F9001
:10A7A0005F900895F8942091D10D3091D20D789456
:10A7B000C9010895CF93DF93C2E4D1E080E6FE01A2
:10A7C00011928A95E9F78AE08093420189E18093AA
:10A7D00070018AE58093710181E080938601219662
:10A7E000FE0120E032E080E891E0219331939587EB
:10A7F0008487938F828F41E0E135F407B1F783E9D5
:10A8000091E06CE870E14AE050E00E946C6C80E0FE
:10A8100090E029913991820F931FE1E0CB35DE075B
:10A82000C1F790936E0180936D01DF91CF910895F0
:10A830001F93CF93DF9384EC98E060E00E94F85779
:10A8400062E471E080E6FB0111928A95E9F784ECFD
:10A8500098E040E650E00E948458182FC3E9D1E008
:10A8600088810E94392C0E94492C8993F1E0CD39CE
:10A87000DF07B1F7809142018A3028F480917F048C
:10A88000816080937F048AE0809342011D3468F0E8
:10A89000E3E4F1E020E030E081919191280F391F4D
:10A8A00081E0EB35F807C1F702C020E030E081E03D
:10A8B00040916D0150916E014217530709F080E0FD
:10A8C000DF91CF911F9108951F93182FE2EAF1E0D5
:10A8D00025EA32E0DF01C9011D920197E9F7CF01B6
:10A8E00061E870E14AE050E00E946C6C812F90E0DA
:10A8F00001966AE070E00E94166C605D6093A701AB
:10A90000805D8093A80180E00E9456611F910895A8
:10A91000CF92DF92EF92FF920F931F93DF93CF932B
:10A920000F92CDB7DEB76B01803160F5682F6F5F96
:10A9300084EC98E049830E94F8574981042F10E085
:10A94000C60160E270E050E00E948D6C84EC98E0FB
:10A95000B6014AE050E00E9484588A30910591F493
:10A9600084EC98E00E94EA57F601E00FF11F2AE01C
:10A9700030E006C0B9010E94026C805D8293CB0179
:10A980000097C1F70F90CF91DF911F910F91FF902A
:10A99000EF90DF90CF9008958F5F0E947B570895CE
:10A9A0001F93CF93DF93182F803150F5682F6F5F7F
:10A9B00084EC98E00E94F85762EA71E025EA32E000
:10A9C000FB01C90111920197E9F784EC98E045EA8F
:10A9D00052E00E9484588F3F910509F018F4812FAE
:10A9E0000E946454C2EAD1E088810E94392C0E94FE
:10A9F000492C899391E0CC3AD907B1F70E941C15F4
:10AA0000DF91CF911F9108950F931F93DF93CF9301
:10AA1000CDB7DEB760970FB6F894DEBF0FBECDBFDF
:10AA2000682F6F5F062F0AC0102F1F5F812F688B62
:10AA30000E947B576889882329F0012F0031A0F3F9
:10AA4000003139F184EC98E00E94F857602F6F5F75
:10AA50008DEC98E042E028E532E00E946A598E01D0
:10AA60000F5F1F4F06C08DEC98E0B8010E94E558BB
:10AA7000A89584EC98E0B8014FE050E00E9413588C
:10AA8000482F882381F78DEC98E00E94935981E04C
:10AA900001C080E060960FB6F894DEBF0FBECDBF58
:10AAA000CF91DF911F910F910895EF920F931F9314
:10AAB0000E946657882341F00E94D15687FD04C04A
:10AAC0000E941854882381F581E790E161E00E949B
:10AAD000A5128FE590E10E948C120E9440570E94BF
:10AAE000DA5384EC98E060E041E022E431E000E6F3
:10AAF00010E078ECE72E0E94C2598036910529F0CB
:10AB000080E590E160E00E94A51280E00E9464541C
:10AB100084EC98E061E042E022EA31E005EA12E0EC
:10AB200058ECE52E0E94C25980916F010E94D054CA
:10AB30001F910F91EF900895882359F09091E008AC
:10AB4000982B9093E0080E94830E9093E2088093E4
:10AB5000E1080895EF920F931F93CF93DF93109125
:10AB6000E008112309F47EC0882309F076C00E9412
:10AB7000830E2091E1083091E208AC01421B530B97
:10AB80004436510508F46EC068C081E08093DF0848
:10AB9000812F90E0EC01C470D07012FF03C023E05D
:10ABA0002093DF081092E00880FF1CC086ED98E03B
:10ABB00061E141E022E431E000E610E0F4E1EF2E53
:10ABC0000E94C2598036910511F480E020C0809126
:10ABD000DC08823021F48091E008816029C080E4A3
:10ABE00090E135C081FF36C086ED98E061E142E03A
:10ABF00022EA31E005EA12E0E4E1EE2E0E94C259B9
:10AC000052E0853A950739F480916F018F5F61E1D9
:10AC10000E9489571FC08091DC088230A1F4809186
:10AC2000E008982F92609093E008209719F08660D2
:10AC30008093E0080E94830E845690409093E2082F
:10AC40008093E10807C0209729F480E390E160E059
:10AC50000E94A5121092DF0805C08091DF088823AA
:10AC600009F493CFDF91CF911F910F91EF90089549
:10AC70000AC081E00E94AA558091650E833019F4C4
:10AC8000A8951092650E8091E008882391F70895A9
:10AC9000DF93CF930F92CDB7DEB7682F70E084E0DB
:10ACA000660F771F8A95E1F7CE01019641E050E0EB
:10ACB0000E94946C89810F90CF91DF910895DF936A
:10ACC000CF930F92CDB7DEB76983682F70E094E021
:10ACD000660F771F9A95E1F7CE01019641E050E0AB
:10ACE0000E94F95E0F90CF91DF91089583EE98E076
:10ACF00060E070E040E450E00E94F95E089585EE67
:10AD000098E062E070E041E050E00E94F95E089552
:10AD10000F931F93182F082F04C0802F0E944856AE
:10AD2000082F802F0E9448568823B9F7802F609102
:10AD3000E5080E945F561093E5080E947F561F9118
:10AD40000F9108951F931091E508112359F0812F59
:10AD50000E9448568093E5080E947F56812F60E04C
:10AD60000E945F56812F1F910895F8942091D10D74
:10AD70003091D20D7894C9010895EF92FF92CF934C
:10AD8000DF938091E508C0E0D0E003C02F960E94D9
:10AD900048568823D9F7CE01DF91CF91FF90EF90ED
:10ADA0000895CF92DF92EF92FF920F931F93CF936C
:10ADB000DF9380E8E3E2F9E0DF011D928A95E9F78D
:10ADC00007EE18E0C0E0D0E08C2FC43139F4D09009
:10ADD000E50835EEE32E38E0F32E0BC07E01EE0CD5
:10ADE000FF1CEC0EFD1E27EE38E0E20EF31ED8012C
:10ADF000DC9090E0C82EC3941DC08D2D84508C37FC
:10AE000038F4ED2DF0E0ED5DF64F8081882361F0A0
:10AE1000992329F0892F60E00E945F560DC0F70149
:10AE200010820E94765608C0C0828D2D0E9448561E
:10AE30009D2DD82EDD2009F721960D5F1F4FC531BE
:10AE4000D10511F604E0E02FF0E0ED5DF64F8081D2
:10AE5000882349F4802F6091E5080E945F56009393
:10AE6000E5080E947F560F5F003869F780E0DF91A8
:10AE7000CF911F910F91FF90EF90DF90CF900895A9
:10AE80001F9380E4E3EEF8E0DF01982F1D929A957E
:10AE9000E9F794E09093E3088093E40880E18093DD
:10AEA000E60884E001C0812F182F1F5F612F0E94E8
:10AEB0005F561038C1F78FE760E00E945F5684E06C
:10AEC0008093E5080E9476561F91089583EE98E0DE
:10AED00060E070E040E450E00E94946C8091E308F0
:10AEE000843039F481E09091E408903419F080E0E6
:10AEF000089580E0089590E0FC01EE0FFF1FE80F39
:10AF0000F91FED51F74F81E09481992309F480E016
:10AF10000895DF93CF9300D00F92CDB7DEB790E0C6
:10AF2000FC01EE0FFF1FE80FF91FDE011196E9513A
:10AF3000F74F23E001900D922150E1F770E0DC0122
:10AF4000AA0FBB1FA80FB91FFB01EE0FFF1FE60FD3
:10AF5000F71FA951B74FE951F74F83E001900D92C8
:10AF60008150E1F7FB01EE0FFF1FE60FF71FE951DC
:10AF7000F74FDE01119683E00D9001928150E1F7C9
:10AF80000E9476560F900F900F90CF91DF91089509
:10AF9000DF93CF930F92CDB7DEB790E09C01220FE5
:10AFA000331F280F391FF901ED51F74F84812951C3
:10AFB000374F93E0D9011D929A95E9F789830E9452
:10AFC00076568981882311F00E9488560F90CF9180
:10AFD000DF910895FC01808190E0FC01EE0FFF1FDE
:10AFE000E80FF91FE851F74F918180819F70089514
:10AFF000FC0160831282118270E0CB01880F991FDF
:10B00000860F971FDC01AD51B74F14962C91149702
:10B0100023831482158216828751974FFC01808109
:10B0200082958F7008958F929F92AF92BF92CF9228
:10B03000DF92EF92FF920F931F93DF93CF930F92C4
:10B04000CDB7DEB78C015B01FC01808190E0FC0193
:10B05000EE0FFF1FE80FF91FE851F74F80812181A4
:10B06000922F9F70F80121813281821B930BE42E75
:10B07000F52E8E159F0508F47C0167014E0108949A
:10B08000811C911C25C0F8016381662321F1848114
:10B090008F5F848370E0B4E0660F771FBA95E1F7A5
:10B0A000680F711DC40141E050E00E94946C8981D9
:10B0B000F50181935F01F80184818F3030F01482B3
:10B0C00083810E944856F80183830894C108D108FF
:10B0D000C114D104C1F6F801818192818E0D9F1DAA
:10B0E0008C199D09928381838E2D8C190F90CF919D
:10B0F000DF911F910F91FF90EF90DF90CF90BF9065
:10B10000AF909F908F9008958F929F92AF92BF9231
:10B11000DF92EF92FF920F931F93CF93DF938C01F7
:10B120005B017A01C0E0D0E045E0842E912C880ECE
:10B13000991E3BC0F801858190E08F779070009751
:10B1400041F4C801B40141E050E00E94135881303D
:10B1500079F5F80145813FE7D32ED4222D2D30E03B
:10B16000C7018C1B9D0B8217930710F4DE2CDC1A91
:10B17000B5016C0F7D1F47FF08C0CB0160E070E098
:10B180004D2D50E00E948D6C0AC0C8014D2D50E03D
:10B190000E9413588D1519F0C80FD11D09C0CD0D8F
:10B1A000D11DF80185818D198583CE15DF0510F23B
:10B1B000CE01DF91CF911F910F91FF90EF90DF9023
:10B1C000BF90AF909F908F9008959F92AF92BF9243
:10B1D000CF92DF92EF92FF920F931F93CF93DF9363
:10B1E000EC018B01C42E8B81882389F489819A819B
:10B1F000009769F4E880FF240E94A2568B83F70130
:10B20000EE0FFF1FEE0DFF1DED51F74F8483DC2C79
:10B210006FE0962E44C0EF80F8840E94830EE81AF7
:10B22000F90AF7FE02C082E004C08B81882319F47A
:10B2300081E08E8337C09C819F3080F01C820E9409
:10B240004856882339F4EB800E94A256682F8E2D31
:10B250000E945F568B810E9448568B838B81882386
:10B2600039F36C81992D961BED2C9D1508F4E92E70
:10B27000AE2CBB2470E06F5F7F4F90E054E0880FEE
:10B28000991F5A95E1F7680F791FC801A5010E941F
:10B29000F95E0A0D1B1D8C818E0D8C83DE18DD205E
:10B2A00009F0B9CF2C2D30E02D19310989819A810F
:10B2B000820F931F9A8389838C2D8D19DF91CF91F3
:10B2C0001F910F91FF90EF90DF90CF90BF90AF90C4
:10B2D0009F9008950F931F93CF93DF93EC01890103
:10B2E00068831A82198270E0CB01880F991F860F3C
:10B2F000971FFC01ED51F74F24812B831C821D8287
:10B300001E82FC01E851F74F10824295407F418335
:10B310000E94830E080F191F18870F83DF91CF91AA
:10B320001F910F9108951F93CF93DF93EC018881B4
:10B3300090E0FC01EE0FFF1FE80FF91FE851F74FF7
:10B34000898180839A819F708181807F892B81830D
:10B350008B81882389F00E944856182F882361F03A
:10B360008B8160E00E945F560E947656112331F077
:10B37000812F0E94885602C010E0F6CFDF91CF9156
:10B380001F9108954F925F926F927F929F92AF921A
:10B39000BF92CF92DF92EF92FF920F931F93DF93B2
:10B3A000CF930F92CDB7DEB75C01290168012E2D36
:10B3B00030E00E946A591982720100E010E081E0D9
:10B3C0003E010894611C711CF70191917F01992342
:10B3D00041F4882349F49081992349F49924939462
:10B3E0001EC0882371F403C09924939401C099244A
:10B3F00099819F3718F40C151D0561F5882379F0A4
:10B4000001C099248981882321F180688983C5013D
:10B41000B30141E00E94E5588130D1F025C0898117
:10B420008823B9F0C501B30141E00E94E55881309D
:10B43000D9F44981B801641B7109640D751DC501FA
:10B440000E94E5589981891719F0981B99830CC0BF
:10B450001982892D99819F5F99830F5F1F4FC016B5
:10B46000D10608F0B1CF05C089818F776801C81A6D
:10B47000D108C5010E949359C6010F90CF91DF9169
:10B480001F910F91FF90EF90DF90CF90BF90AF9002
:10B490009F907F906F905F904F90089580E094E030
:10B4A000E3EAF9E0DF019C011D9221503040E1F711
:10B4B00008950F931F93CF93DF93DA011196FA014A
:10B4C0004491ED012196FD01A491B0E0179613E09F
:10B4D000B595A7951A95E1F71A2FDE011196FE0191
:10B4E0009491929FE0011124AC0FBD1F00FD08C094
:10B4F00001FF08C09091D30D51E096FD04C002C039
:10B5000051E001C050E066956695669570E09B013C
:10B510003695322F22273795279590E0280F391F2F
:10B52000610F711D7695762F662777956795680F61
:10B53000791F042F10E014C0E901CD55D64F80E0EB
:10B5400090E008C0FD01E80FF91FE4915111E0956A
:10B55000E99301968417B0F3A00FB11F20583F4F15
:10B560002617370749F7DF91CF911F910F91089563
:10B57000FF920F931F93CF93DF93942F46313CF4A8
:10B58000440F490F440F22FFABC0440FA9C0482FFE
:10B590004A5F092F112707FD109520FD09C021FFE3
:10B5A0000AC03091D30DFF24F39436FD05C003C0CB
:10B5B000FF24F39401C0FF2466956695669570E0BC
:10B5C0007695762F662777956795680F711DEB0145
:10B5D000CD55D64F22FF4FC09E3209F04A5FC801B9
:10B5E000809760E170E00E94166C80EA90E0689FAE
:10B5F0009001699F300D789F300D1124C801880F8C
:10B60000991F53E0000F111F5A95E1F7800F911F0A
:10B61000280F391F235C3E4E85E0882369F0F9012D
:10B620009491E056FF4F54912F5F3F4FF901649181
:10B63000E056FF4F749104C060E050E090E070E08D
:10B64000FF2021F09095609550957095DE01AF57E1
:10B65000BF4FFDE0A33ABF0740F498836983FE0122
:10B66000E058FF4F50837C93229681508F3FC1F169
:10B670002F5F3F4FD2CF23FF0DC0FF2011F08FEF80
:10B6800001C080E06D55764FFB01808321964F5FAE
:10B6900091E001C090E09801220F331F220F331F69
:10B6A000200F311F2650304F85E0F9012F5F3F4FAB
:10B6B000E491992311F0843039F0FDE0C33ADF07BB
:10B6C00018F4F110E095E993815079F75DE0C33A01
:10B6D000D50730F4FF2011F08FEF01C080E08883A0
:10B6E000842FDF91CF911F910F91FF90089520E05B
:10B6F0000E94B85A0895CF92DF92EF92FF920F9373
:10B700001F93CF93DF93162FF22EF0E1EF2EE0225E
:10B71000C42EE6016E01D52EE6010CC0EE2011F01C
:10B72000488102C0FE014491612F202F0E94B85A27
:10B73000FA942196FF2091F7DF91CF911F910F91FD
:10B74000FF90EF90DF90CF9008950F93FA019491BE
:10B750004F5F5F4F929FF00111244E0F5F1F292F03
:10B760000E947B5B0F9108950F9300E00E947B5B2A
:10B770000F910895CF92DF92FF920F931F93CF9373
:10B78000DF93162F022FA0E1FA2EF222C42EE6013B
:10B790006E01D52EE601FF2011F0488102C0FE01A6
:10B7A00044912196442329F0612F202F0E94B85AFA
:10B7B000F2CFDF91CF911F910F91FF90DF90CF904B
:10B7C0000895982FAB0180E0692F20E00E94BA5BBA
:10B7D000089520E00E94BA5B0895EF92FF920F93C4
:10B7E0001F93DF93CF930F92CDB7DEB7182F062F9D
:10B7F0007A01982F9C5E95504E2D4F704A301CF068
:10B80000495C28E002C0405D20E0892F602F9983C9
:10B810000E94B85A9981911731F0B4E0F694E794F8
:10B82000BA95E1F7E8CF0F90CF91DF911F910F917B
:10B83000FF90EF900895E62FE695E695E695F0E007
:10B84000F695FE2FEE27F795E795E80FF11DED55DC
:10B85000F64F8DE0E33AF80758F4677081E090E026
:10B8600002C0880F991F6A95E2F72081282720835C
:10B87000089547FF02C0840F4195E62FE695E695AF
:10B88000E695F0E0F695FE2FEE27F795E795E80FA1
:10B89000F11DED55F64F6770A1E0B0E001C0AA0FB1
:10B8A0006A95EAF711C08DE0E33AF80778F4822F41
:10B8B00090E09C013595279580FF04C080818A2700
:10B8C0008083206841503196442369F708952FEF13
:10B8D0000E94395C08950F931F93CF93DF93C82F75
:10B8E000D0E0E62FE695E695E695F0E0F695FE2F9A
:10B8F000EE27F795E795EC0FFD1FED55F64F062F58
:10B9000010E0242F332727FD3095200F311FC90168
:10B9100068E070E00E94166C7695762F6627779522
:10B9200067956C0F7D1F6D55764F0770107081E025
:10B9300090E002C0880F991F0A95E2F781959081E7
:10B94000892708C0E058FF4F8DE0E33AF807D0F4AC
:10B95000808180958083E617F707A0F38DE0E33AB6
:10B96000F80780F4C90168E070E00E94166C21E0DD
:10B9700030E002C0220F331F8A95E2F721958081C3
:10B9800082278083DF91CF911F910F910895EF92CD
:10B99000FF920F931F93F82E162F042FE22E422FA3
:10B9A0000E946B5C023038F08F2D8150800F612F28
:10B9B0004E2D0E946B5CF3940250612F61506E0D0E
:10B9C0008F2D402F0E94675C8F2D612F402F0E948A
:10B9D000675C1F910F91FF90EF900895DF92EF92B7
:10B9E000FF920F931F93F82E162FE22E053608F0C4
:10B9F00004E6602F70E0242F30E022503040629F38
:10BA0000C001639F900D729F900D112464E670E059
:10BA10000E94166C062F8F2D612F2E2D0E94C75C61
:10BA2000002371F0D12EDA94DE0C1F5FF39406C070
:10BA30008F2D612F402F0E94675C1F5F1D15C0F383
:10BA40001F910F91FF90EF90DF9008952F923F92FA
:10BA50004F925F926F927F928F929F92AF92BF921E
:10BA6000CF92DF92EF92FF920F931F93DF93CF93CA
:10BA700000D00F92CDB7DEB7182F662E59016A019C
:10BA8000F02E802F05FF04C004FF04C002E003C0B5
:10BA900000E001C001E0E7FE04C0E1942224239409
:10BAA00001C02224D7FE0BC0D094C094B094A094BF
:10BAB000A11CB11CC11CD11C4424439401C04424CA
:10BAC00082FF06C09CE09093A30D3AE0932E05C040
:10BAD00096E09093A30D25E0922E86FF2FC0411093
:10BAE000190D28EEA21623E0B20620E0C20620E0DF
:10BAF000D20614F0190D06C034E6A316B104C10431
:10BB0000D10414F0190D06C08AE0A816B104C104CE
:10BB1000D1040CF0190D002391F0023039F4E4E661
:10BB2000AE16B104C104D10454F4190DFAE0AF16F5
:10BB3000B104C104D1041CF4190D01C0191B80917A
:10BB4000A30D810F8093A30D023011F420EFF20EAC
:10BB50005524539492E0792E88242E2D332727FDE7
:10BB60003095862D8A5F89833B832A8370C0C60106
:10BB7000B5012AE030E040E050E00E944B6CE62E38
:10BB800080E3382E3E0C812F662D432D2F2D0E94F1
:10BB9000B85A0515D9F5F2FE23C08E2D8150833099
:10BBA00008F47394C601B5012AE030E040E050E0AB
:10BBB0000E944B6CCA01B9012AE030E040E050E03D
:10BBC0000E944B6C623011F06430C1F4E32DE43319
:10BBD00019F4812E839413C0812E8A9473940FC01C
:10BBE0001250812F8F5FF0FE05C0662D47E00E9446
:10BBF0006B5C05C069810E941B5C01C0812EFAE06C
:10BC0000AF16B104C104D1040CF000E0C601B501C7
:10BC10002AE030E040E050E00E944B6C59016A019C
:10BC2000211531054105510581F4002331F0023021
:10BC300059F4252D223040F408C0F4FE10C0222013
:10BC400021F430EFF30E01C000E019195394852D53
:10BC500090E0EA81FB81E817F9070CF088CF882093
:10BC600061F0662D645F882D472D0E94675C662D0C
:10BC7000635F882D472D0E94675C442039F0812F37
:10BC80008919662D4DE22F2D0E94B85A0F900F9002
:10BC90000F90CF91DF911F910F91FF90EF90DF9068
:10BCA000CF90BF90AF909F908F907F906F905F905C
:10BCB0004F903F902F900895EF920F93022FFA012B
:10BCC0009F01442737FD4095542F75E0E72E0E94D1
:10BCD000265D0F91EF90089520E00E945C5E08952C
:10BCE000A998AB98AC988BBBAD9AAD98AB9AA99A32
:10BCF000089520E030E006C045E04A95F1F70000E5
:10BD00002F5F3F4F28173907BCF30895AA9885E0A5
:10BD10008A95F1F7000085E08A95F1F70000AA9A6C
:10BD20008CED95E00E94795E82EE0E94705E8EEA54
:10BD30000E94705E81EA0E94705E86EA0E94705ED8
:10BD400084EA0E94705E82EA0E94705E80EC0E942B
:10BD5000705E8FE20E94705E85E20E94705E81E8F4
:10BD60000E94705E82E20E94705E8FEA0E94705EA6
:10BD700082E28093700108951F93182F81E80E943A
:10BD8000705E812F0E94705E1F9108951F93CF9364
:10BD9000DF9310E0C3EAD9E084E00E94705E80E1A6
:10BDA0000E94705E812F806B0E94705EA998AB9A92
:10BDB000AC98FE0180E290819BBBAD9AAD989181D9
:10BDC0009BBBAD9AAD9892819BBBAD9AAD98938188
:10BDD0009BBB3496AD9AAD98815069F7C058DF4F40
:10BDE000AB9AA99A1F5F1830B9F6DF91CF911F91D6
:10BDF0000895BF92CF92DF92EF92FF920F931F931D
:10BE0000CF93DF93EA01E82EF92E062F172F21C0DA
:10BE1000F701B1907F0168010894C11CD11C04C0D6
:10BE2000009739F00E94E3178091DF0890E082705C
:10BE30009070E199F5CF1FBB0EBBE09A8DB3B81699
:10BE400031F0BDBA8FB7F894E29AE19A8FBF21978B
:10BE500086012097E9F6DF91CF911F910F91FF9016
:10BE6000EF90DF90CF90BF9008958093D40D089508
:10BE70008091D40D1092D40D0895FC018081982FEB
:10BE8000990F9E70807F892B8083662321F09160BB
:10BE9000807F892B808381818F5F81839281992329
:10BEA00091F020812F7079F4933659F0242F20627D
:10BEB0002093D40D903111F4803118F080818F7C63
:10BEC0008083118212828281883009F443C08930D4
:10BED00058F4813009F446C08130A0F08230D1F1AD
:10BEE000843009F052C036C08F3549F1803620F4D5
:10BEF000803109F04AC02EC0813689F0823609F0BF
:10BF000044C03DC08081982F9F709F30F1F591E62D
:10BF1000928391819131E0F08F7C808319C04066DB
:10BF20004093D40D9081892F82958F708F5F83709D
:10BF30008295807F9F7C982B90838FE508C08181BC
:10BF4000883111F4406818C08832F9F480E18283A6
:10BF5000118208959181903328F090E0959587950E
:10BF600082831182828190E00197218130E08223D7
:10BF70009323009751F440644093D40D0895818138
:10BF8000803418F088E08283118208958E30910504
:10BF90006CF4FC01EE0FFF1FE80FF91FE955F24F9B
:10BFA00090819F7081E09F30E9F53FC0823129F197
:10BFB000833160F48F30C9F0803118F48E3091F500
:10BFC00029C0803161F0813169F512C0843151F0AE
:10BFD0008431C8F08531D9F0863121F51EC091B188
:10BFE00094701DC091B192701AC09091630013C0FB
:10BFF000909163009095987012C08091630083FFC8
:10C0000013C091B102C091B19095907408C091B1E4
:10C01000907105C091B1917002C091B1907281E0B0
:10C02000992319F480E0089580E008958F708E3090
:10C0300058F490E0FC01EE0FFF1FE80FF91FE955DF
:10C04000F24F82E68283118208958F708E3068F4F9
:10C0500090E0FC01EE0FFF1FE80FF91FE955F24FCA
:10C0600083E6828380818F7C808308950F931F9362
:10C07000CF93DF938091D10D9091D20D0196909343
:10C08000D20D8093D10D8091D30D8F5F8093D30D0E
:10C0900006B3009540E050E010E001C0AE01EA01B7
:10C0A0002196CA01880F991F840F951FB8010C2E85
:10C0B00002C0759567950A94E2F7617070708955B2
:10C0C000924F50E00E943D5FC630D10539F700B372
:10C0D0000095C0E0D0E0FE01E350F64EE4919E01F1
:10C0E0002A5F3F4FC901880F991F820F931F8955FF
:10C0F000924FE02361E009F460E09E012A5F422F45
:10C1000050E00E943D5F2196C830D10521F7DF91B4
:10C11000CF911F910F910895FF920F931F93CF938B
:10C12000DF93F82EECEBF1E080E090E0582F9C01DB
:10C130004081F41638F0442329F001963A96813272
:10C140009105A1F75032B9F1E901CC0FDD1FC9010A
:10C15000A3E0880F991FAA95E1F7C80FD91F8E0198
:10C1600004541E4FA9014F5F5F4FCA01880F991FEA
:10C17000E3E0440F551FEA95E1F7840F951F2095E2
:10C180003095205E3F4FA901440F551F63E0220FF9
:10C19000331F6A95E1F7420F531F84549E4FB80135
:10C1A0000E947B6C8AE0D8011D928A95E9F7CE55F2
:10C1B000DE4FFA8E02C00CEB11E0C801DF91CF9187
:10C1C0001F910F91FF90089580E491E0ECEBF1E076
:10C1D000DF019C011D9221503040E1F70895E8E80D
:10C1E000F3E088E2DF011D928A95E9F7B89688E4CA
:10C1F000DF011D928A95E9F70895282F30E08830F5
:10C20000C0F4462F572FDA01F901EE0FFF1FEE0F92
:10C21000FF1FE20FF31FE857FC4F95E0899FC00115
:10C22000112483579C4F2D912193E817F907D9F7D3
:10C230000895462F572FDA0128503040F90193E036
:10C24000EE0FFF1F9A95E1F7E20FF31FE055FC4F49
:10C2500099E0899FC00111248F589C4F2D91219303
:10C26000E817F907D9F7089590E00197FC01EE0F60
:10C27000FF1FE80FF91FEE55FE4FDF01A85ABD4F13
:10C280006C93DF01AA5ABD4F4C93E95AFD4F2083AE
:10C290000895E0918601F0E0EE0FFF1FEE0FFF1F03
:10C2A000E80FF11DE950FB4F849108958F929F9202
:10C2B000AF92BF92CF92DF92EF92FF920F931F93B4
:10C2C000DF93CF93CDB7DEB76D970FB6F894DEBF8F
:10C2D0000FBECDBFF82EDE011596E6E2F1E085E057
:10C2E00001900D928150E1F7DE011A96E1E2F1E052
:10C2F00085E001900D928150E1F7DE011F96ECE19F
:10C30000F1E085E001900D928150E1F7DE01549655
:10C31000E7E1F1E085E001900D928150E1F7DE0167
:10C320005996E2E1F1E085E001900D928150E1F74C
:10C3300019821A821B821C82E0918B01F0E0E85284
:10C34000FB4F26E030E011E0E491CE2EDD24BE016B
:10C350006F5F7F4F0FC04F5F5F4FA417B50711F49A
:10C36000FC01108344305105B1F71F5F225030406B
:10C37000153081F040E050E0C601022E02C09595D4
:10C3800087950A94E2F783709070DC011196860F0E
:10C39000971FE1CFFF2041F50E94E46089810E9450
:10C3A0008C608C0181E00E944961F801818374E610
:10C3B000F72EF2828A810E948C608C0182E00E94BA
:10C3C0004961F8018183F2828B810E948C608C012B
:10C3D00083E00E944961F8018183F2828C810E948E
:10C3E0008C608C0184E07EC0FF2DF13071F48B8174
:10C3F0000E948C60FC0188E081838CE98283F38257
:10C400008781817F84608783D7C18F2D8230E9F552
:10C410008B810E948C60FC0108E001836CE9F62EA0
:10C42000F28285E183838781817F846087838EE0C8
:10C430000E948C60FC0182E2818314E612838EE00C
:10C440000E948C60FC010183F28284E183838781F6
:10C45000817F846087838EE00E948C60FC01018371
:10C46000128381E083838781817F8460878383E077
:10C470000E944961482F8BE062E02DE90E943461FF
:10C480008CE061E042E220E095C1EF2DE33081F5E0
:10C490000E94E460E9808E2D0E948C608C0181E016
:10C4A0000E944961F801818354E6F52EF2828E2DB7
:10C4B0000E948C608C0182E00E944961F8018183B6
:10C4C0008CE98283EA808E2D0E948C608C0181E051
:10C4D0000E944961F8018183F2828E2D0E948C6056
:10C4E0008C0182E00E944961F8018183F28264C17B
:10C4F000FF2DF43081F50E94E460EA808E2D0E94C9
:10C500008C608C0182E00E944961F801818344E6DD
:10C51000F42EF2828E2D0E948C608C0184E00E94A9
:10C520004961F8018183F282EC808E2D0E948C603B
:10C530008C0182E00E944961F8018183F2828E2D94
:10C540000E948C608C0184E00E944961F801818323
:10C550008CE9828331C1FF2DF53009F0D0C00E94F3
:10C56000E4600E94EF6081E00E948C60FC013AE090
:10C57000C32EC18224E6B22EB28282E00E948C6079
:10C58000FC019BE0D92ED182B28283E00E948C60B4
:10C59000FC018CE0E82EE182B28284E00E948C6093
:10C5A0008C0181E00E944961F8018183B28285E0BB
:10C5B0000E948C608C0183E00E944961F8018183B4
:10C5C000B28204E0A02EA38287E084838781816009
:10C5D000878385E00E948C608C0183E00E94496122
:10C5E000F8018183B282F38218E0812E84828781F0
:10C5F0008160878385E00E948C608C0183E00E94CB
:10C600004961F8018183B282B6E0BB2EB382A9E012
:10C610009A2E948287818160878385E00E948C6056
:10C62000FC0181828CE9828381E083838781817F21
:10C630008460878386E00E948C60FC0191828EE199
:10C64000828388EF83838BE00E948C608C0183E07F
:10C650000E944961F801818376E4972E9282A38239
:10C66000C4828781816087838BE00E948C608C010B
:10C6700083E00E944961F80181839282F382D4822F
:10C680008781816087838BE00E948C608C0183E0CE
:10C690000E944961F80181839282B382E48287819A
:10C6A000816087838091B8018F7180628093B80127
:10C6B0008FE18093B90180E0BE016B5F7F4F0E94E4
:10C6C000FD6081E0BE01665F7F4F0E94FD6082E0F9
:10C6D000BE01615F7F4F0E94FD6083E0BE016C5E22
:10C6E0007F4F0E94FD608E01075E1F4F84E0B801FE
:10C6F0000E94FD6085E0B8010E94FD605DC0FF2DD5
:10C70000F630B1F486E00E948C60FC01F18282E395
:10C71000828388EF838314E6108786E00E948C6012
:10C72000FC01F1828EEC828388E08383108744C011
:10C730008F2D873009F040C08FE00E948C60FC0193
:10C7400084E2818384E6828388E8868380E10E9494
:10C750008C60FC0189E081830EE602838AE083839A
:10C7600080E10E948C60FC0118E0118382E98283E1
:10C770008BE083838781817F8460878380E10E944F
:10C780008C60FC01118302838CE083838781817F2D
:10C790008460878381E06BE043E224E20E9434619D
:10C7A00082E061E043E229E60E94346183E062E0D6
:10C7B00043E227E90E94346182E00E949C550E9476
:10C7C00038566D960FB6F894DEBF0FBECDBFCF9131
:10C7D000DF911F910F91FF90EF90DF90CF90BF906E
:10C7E000AF909F908F9008956F927F928F929F92BB
:10C7F000AF92BF92CF92DF92EF92FF920F931F936F
:10C80000CF93DF938091B80181FF03C060E075E0B2
:10C8100002C060E074E09091B50184E69802C00126
:10C820001124885A9D4FE091BB01FF27E7FDF09549
:10C8300048EE53E0E49F9001E59F300DF49F300DEA
:10C84000112428533045AA24BB24A81AB90A281B4E
:10C85000390BFEE1EF2EF5E0FF2E4091B201440FBF
:10C86000485F50E0440F551F440F551F4B52524F25
:10C87000E5EDFDE0CC24DD24C61AD70AA8E5B2E038
:10C88000A81BB90B1CC0E701699079907E014B0190
:10C89000661677060CF4430184018C149D040CF495
:10C8A0008601005A164FE501C01BD10B2C0F3D1F0E
:10C8B0000A0F1B1F11830083938382833496E4172E
:10C8C000F50709F7318320839383828315821482CD
:10C8D000DF91CF911F910F91FF90EF90DF90CF905C
:10C8E000BF90AF909F908F907F906F900895E09150
:10C8F0002B01F0912C018193F0932C01E0932B01FB
:10C900000895FF920F931F93CF93DF93B9E0FB2E0F
:10C9100090E120E0C82FD0E08E0101701070201748
:10C9200011F4905F07C0892F90E001970E9477640F
:10C93000202F90E1FA9431F0D595C795AE0140686B
:10C94000842FE8CF892F90E00F960E947764DF91C3
:10C95000CF911F910F91FF9008951F93CF93DF9375
:10C96000182F25ED3DE030932C0120932B01809171
:10C970003101877471F08091B201882319F0813000
:10C9800029F402C080E803C080E901C088E98093EF
:10C9900031018091310187FF0BC086E190E00E9458
:10C9A000C65F882329F4809131018F77809331010C
:10C9B0008091310187FD5AC085E160E040E00E942E
:10C9C0005610882309F452C080913101806280930F
:10C9D000310180916F018F5F80933201E3E3F1E0D9
:10C9E000AEE1B5E080E01CC02D913D9135952795D5
:10C9F00020503E4F37FD05C093E02F3F390724F408
:10CA000005C020E030E002C02FEF33E0932F937099
:10CA1000482F440F440F942B908321838F5F3296CD
:10CA2000811711F7C1E3D1E089910E94816481E00F
:10CA3000CF33D807C9F780912B0190912C01019732
:10CA400090932C0180932B018FEF90E00E947764EC
:10CA500080E090E00E94776485ED9DE09093300146
:10CA600080932F01DF91CF911F9108958091310123
:10CA70008F7DADCF1F920F920FB60F9211242F937F
:10CA80008F939F93EF93FF9388B391E0892788BB9F
:10CA9000E0912F01F09130012191F0933001E0936A
:10CAA0002F01822F90E097BD86BD293C08F0C09AE7
:10CAB0008091650E81608093650EFF91EF919F914B
:10CAC0008F912F910F900FBE0F901F9018951F926E
:10CAD0000F920FB60F9211242F933F938F939F9332
:10CAE000EF93FF9388B391E0892788BBE0912B01F6
:10CAF000F0912C01208130E020FD04C088B599B56B
:10CB0000809603C088B599B5409699BD88BDC90186
:10CB100095958795009791F4CF01019690932C01FC
:10CB200080932B018181882351F48091780090912A
:10CB300079008053984F99BD88BD01C08083809152
:10CB4000650E81608093650EFF91EF919F918F91AB
:10CB50003F912F910F900FBE0F901F901895EDE70A
:10CB6000F0E08081857E808317981F9AAAE8B0E064
:10CB70001C9210928B0082E88C938081806280836B
:10CB80000895EDE7F0E080818F7D8083179AAAE811
:10CB9000B0E01C9210928B008AE08C9380818861B7
:10CBA000808308951F920F920FB60F9211248F93D6
:10CBB0009F93AF93BF93EF93FF938091710E882360
:10CBC00021F01F9A1092710E04C01F9881E080938B
:10CBD000710EA0912D01B0912E01FD0181919191D5
:10CBE0009093870080938600F0932E01E0932D01AF
:10CBF0008091680E9091690E9093850080938400D7
:10CC000012968D919C911397009759F48DE19EE0B7
:10CC100090932E0180932D018091B80181708093B3
:10CC2000710E8091650E81608093650EFF91EF918A
:10CC3000BF91AF919F918F910F900FBE0F901F905A
:10CC40001895AF92BF92CF92DF92EF92FF920F931F
:10CC50001F93CF93DF938091B80181FF03C040E021
:10CC600055E002C040E054E0F090B201FF0C80E1DA
:10CC7000F80E2091B50184E6280290011124285A6B
:10CC80003D4FE091BB01FF27E7FDF09568EE73E0B3
:10CC9000E69FC001E79F900DF69F900D11248853E9
:10CCA0009045CC24DD24C21AD30A821B930B68EF73
:10CCB000E62EEF0CEDE1FEE000271127041B150B1B
:10CCC00068E572E0621B730B21C0AE2DB0E0AA0FC5
:10CCD000BB1FA25EBA4FAC901196BC90D5014A170B
:10CCE0005B070CF4DA01A017B1070CF4D801A05AC5
:10CCF000B64FE601CA1BDB0B8C0F9D1F31832083CF
:10CD0000A60FB71FB383A2833496E394EF14E8F21F
:10CD10003183208393838283885E93409093690E4E
:10CD20008093680E15821482DF91CF911F910F912D
:10CD3000FF90EF90DF90CF90BF90AF9008951F923B
:10CD40000F920FB60F9211242F933F934F935F933F
:10CD50006F937F938F939F93AF93BF93EF93FF93C3
:10CD600078940E942166FF91EF91BF91AF919F91BE
:10CD70008F917F916F915F914F913F912F910F9084
:10CD80000FBE0F901F90189520916E0E30916F0E70
:10CD900090E0822793279070880F991F8759954EAE
:10CDA000FC0145915491232F332742275327509359
:10CDB0006F0E40936E0E089590916A0E969596951B
:10CDC000982B90936A0E80916B0E8F5F80936B0E01
:10CDD000843068F0E0916C0EF0916D0E9193F093B9
:10CDE0006D0EE0936C0E10926A0E10926B0E089509
:10CDF00003C080E00E94DC6680916B0E8823C9F737
:10CE0000E0916C0EF0916D0E10820895882339F038
:10CE10008091700E8F5F8093700E80E803C0109237
:10CE2000700E80EC0E94DC668091700E8530B8F741
:10CE300008950F931F93182F0E94C46608E0812F56
:10CE400080780E940667110F0150C9F71F910F915A
:10CE5000089580EC0E94DC6680E80E94DC6680E831
:10CE60000E94DC6680E80E94DC6680E80E94DC6646
:10CE700080E80E94DC6680E80E94DC6680EC0E940C
:10CE8000DC660895CF92DF92EF92FF920F931F938B
:10CE9000CF93DF9385ED9DE090932C0180932B0140
:10CEA00090936D0E80936C0E10926F0E10926E0E1A
:10CEB00010926A0E10926B0E1092700E0E942967EB
:10CEC0008091B2010E9419678091670E0E941967D4
:10CED00080E00E9419671092670ECEE1D5E014E061
:10CEE000C12ED12C28813981C901880F991F820F49
:10CEF000931FB6010E94166C8B010653174F2A81AF
:10CF00003B81C901880F991F820F931FB6010E94B0
:10CF1000166C7B018AEC98E0E80EF91E802F0E94C7
:10CF20001967912F9F708E2D8295807F892B0E948B
:10CF30001967C701F4E096958795FA95E1F70E9485
:10CF40001967249695E0CE32D90761F600916F0EED
:10CF500080916E0E0E941967802F0E9419670E94AF
:10CF600029670E94F8668091780090917900805C32
:10CF700093469093790080937800C09ADF91CF9187
:10CF80001F910F91FF90EF90DF90CF9008958091C7
:10CF9000B1019091660E981709F494C08093660EC3
:10CFA0008130F9F0813030F08230F1F1833009F0D6
:10CFB00089C05EC00E94AF651EBC80E49CE99BBD39
:10CFC0008ABD1DBC1CBC87B7837C87BF8CE386BF32
:10CFD0008FE380937C0087B7806187BF1FBC8AE0A6
:10CFE00021C00E94AF651EBC1DBC1CBC80E797E140
:10CFF00099BD88BD80EA9FE0909379008093780086
:10D0000087B7837C87BF8CE386BF8FE380937C00E8
:10D0100087B7886087BF80917D00816080937D00A5
:10D020001FBC82E08EBD4EC00E94AF651EBC88EC66
:10D0300090E090937900809378008CE291E09DBD20
:10D040008CBD80EE9BEA97BD86BD87B7837C87BF8A
:10D050008CE386BF8FE380937C0087B7806287BFB5
:10D0600080917D00816080937D001FBC8AE1DACFD2
:10D070001EBC80E49CE99BBD8ABD1DBC1CBC87B75F
:10D08000837C87BF80917D008E7F80937D008CE3C1
:10D0900086BF8FE380937C0087B7806187BF1FBC0A
:10D0A0008AE08EBD0E94216680E593EC9093870014
:10D0B0008093860088E893E19093850080938400B4
:10D0C0000E94C1658091B101813051F0813028F01A
:10D0D000823051F0833079F40CC00E94F4630895DB
:10D0E00078940E9442670895789486E00E94AD6427
:10D0F00008950E94F46308951F920F920FB60F9245
:10D1000011242F933F934F935F936F937F938F934C
:10D110009F93AF93BF93EF93FF938091B1018230C0
:10D12000C1F480E492EA97BD86BD80917800909129
:10D1300079008F3F910538F488E598E9909379005C
:10D140008093780008C088EC90E0909379008093F9
:10D1500078000E94C767FF91EF91BF91AF919F91B7
:10D160008F917F916F915F914F913F912F910F9090
:10D170000FBE0F901F9018951F920F920FB60F922F
:10D1800011242F933F934F935F936F937F938F93CC
:10D190009F93AF93BF93EF93FF938CB59DB5209171
:10D1A000720E222321F0C09A1092720E04C0C09811
:10D1B00021E02093720EA0913F01B0914001FD014A
:10D1C000219131913BBD2ABDF0934001E0933F0195
:10D1D0002091BF063091C0062817390720F490939C
:10D1E000C0068093BF0620910C0130910D0182177B
:10D1F000930720F490930D0180930C0112968D916A
:10D200009C9113970097D9F485ED9DE09093400190
:10D2100080933F018091B801809581708093720E58
:10D2200087B78F7E87BF0E94C7678091B10188232F
:10D2300011F0833021F487B7806187BF78948091A3
:10D24000650E81608093650EFF91EF91BF91AF9164
:10D250009F918F917F916F915F914F913F912F910E
:10D260000F900FBE0F901F901895909185019873A5
:10D27000903121F463E00E94F66B0895983111F427
:10D2800086950895983211F4880F0895903319F413
:10D29000982F990F890F0895FC01A5E6B0E08C91B5
:10D2A0008B7F8C93148215821082118216A617A68A
:10D2B00008950E944C69089521E0FC01848188232F
:10D2C00009F420E0822F0895FC0181819081891B5F
:10D2D000877098E0981B81E0933008F480E008950F
:10D2E000FC0184818823F9F08150848382819381B9
:10D2F000890F828386A5882309F44CC087A5982FBF
:10D30000915097A7882331F08091650084608093C5
:10D3100065000895809165008B7F80936500809102
:10D32000900187A708951B98809165008B7F80935B
:10D3300065008581882319F0815085830895808157
:10D340009181891739F190E0DF01A80FB91F169676
:10D350002C911697228356962C91569724831E96CD
:10D360002C911E9723835E962C915E972583D096F1
:10D370002C91D09726A717A696962C919697322F88
:10D38000315096963C939697222321F4019687700C
:10D390009070808308958F929F92AF92BF92CF92A8
:10D3A000EF92FF920F931F93DF93CF9300D0CDB7EF
:10D3B000DEB74C01122F4A8369830E9464694A8157
:10D3C0006981882331F180918501887311F1F4011D
:10D3D000A180BB24C501019697E0F92EF822808137
:10D3E000F816B9F0662329F080918F01865F860FC9
:10D3F00001C080E0A80CB91CF5018683842F0E942F
:10D400003569F501868B168FE0AA06A3C686F4015E
:10D41000F1820F900F90CF91DF911F910F91FF90AC
:10D42000EF90CF90BF90AF909F908F900895AF9264
:10D43000BF92CF92EF920F93DF93CF9300D00F92D2
:10D44000CDB7DEB75C012B834A8369830E94646990
:10D450002B814A816981882329F180918501887314
:10D4600009F1662329F080918F01865F860F01C044
:10D4700080E0F5018283842F2B834A8369830E9495
:10D480003569F50184832B812583E6A617A6C3821F
:10D49000808181834A816981002321F00150C50187
:10D4A0000E94CB690F900F900F90CF91DF910F9159
:10D4B000EF90CF90BF90AF900895CF92EF920F93DF
:10D4C000CF93DF93EC0180918501869586958695B3
:10D4D000877028819981291709F05CC1E62FF0E057
:10D4E000E132F10508F056C1EA5BFF4FEE0FFF1F76
:10D4F0000590F491E02D0994CE0166E44AE0DEC087
:10D50000CE0166E444E1DAC0CE0166E44EE1D6C065
:10D51000CE0164E64AE022E002E0EE24E39452E029
:10D52000C52E36C1CE016FE545E022E00AE0EE24CB
:10D53000E394CC240E94CB69CE016FE545E02AE05C
:10D5400001E00E94CB69CE016FE545E022E00AE0F0
:10D550001FC1CE0160E54AE023E002E0EE24CC24C6
:10D56000CA940E94CB69CE016CE34AE023E0CC244C
:10D57000C3940E94CB69CE0166E44AE021E000E05A
:10D5800032E0E32E96C0CE0166E445E021E001E002
:10D59000EE24E394CC240E94CB69CE0162E34FE0F9
:10D5A00022E00E94CB69CE0160E54FE022E0F0C0AE
:10D5B000CE016EE645E021E002E0EE24E394CC24C7
:10D5C0000E94CB69CE016CE745E021E02AC0CE0184
:10D5D00062E345E025E000E0EE24CC240E94CB6924
:10D5E000CE016AE545E025E00E94CB69CE016EE6FA
:10D5F00043E024E002E0CCC0CE0160E545E02AE053
:10D6000003E0EE24E394CC240E94CB69CE0160E5D4
:10D6100045E024E101E00E94CB69CE0160E545E0F0
:10D620002AE003E0B5C0CE016AE044E125E002E073
:10D63000EE24E394CC24C394ABC0CE0162E344E077
:10D640002AE002E0EE24E394CC240E94CB69CE01D0
:10D6500066E448E024E101E00E94CB69CE0162E388
:10D6600048E02AE002E00E94CB69CE0166E444E093
:10D6700024E101E08DC0CE0168E745E02AE00AE040
:10D6800016C0CE0168E745E022E30AC0CE0160E0A3
:10D6900044E12AE001E00BC0CE0160E044E12AE071
:10D6A00002E005C0CE0160E044E12AE003E0EE24A0
:10D6B000E394CC246DC0CE0166E448E221E000E0B2
:10D6C00048C0813009F466C0CE016BE405C08130EA
:10D6D00009F460C0CE0161E44AE021E000E041C00D
:10D6E000CE01642F46E0F9CFCE0166E44AE022E0A5
:10D6F000E6CF813009F44EC0CE0166E44AE022E074
:10D70000EDCFCE0168E7E8CFCE0168E74AE021E03F
:10D710001FC0CE016AE74AE021E00FC0CE016CE7EE
:10D720004AE021E004C0CE0168E74FE023E003E0D7
:10D7300010C0CE0168E74FE023E002E00AC0CE014E
:10D7400068E74FE023E004C0CE0166E444E129E14C
:10D7500001E0EE24E39406C0CE0166E44AE022E054
:10D7600002E0EE24CC240E94176A14C0CE016CE3C0
:10D7700044E123E002E0EE24CC24C3940E94CB6970
:10D78000CE0160E544E123E0EE24E394CC24CA9486
:10D790000E94CB69DF91CF910F91EF90CF900895C8
:10D7A000682F87E494E046E40E945D6A0895629FD2
:10D7B000D001739FF001829FE00DF11D649FE00D89
:10D7C000F11D929FF00D839FF00D749FF00D659FEA
:10D7D000F00D9927729FB00DE11DF91F639FB00DE9
:10D7E000E11DF91FBD01CF0111240895991B79E0B6
:10D7F00004C0991F961708F0961B881F7A95C9F7E1
:10D8000080950895AA1BBB1B51E107C0AA1FBB1F2F
:10D81000A617B70710F0A61BB70B881F991F5A95BC
:10D82000A9F780959095BC01CD01089597FB092E2D
:10D8300007260AD077FD04D0E5DF06D000201AF4D1
:10D84000709561957F4F0895F6F7909581959F4F5C
:10D850000895A1E21A2EAA1BBB1BFD010DC0AA1F31
:10D86000BB1FEE1FFF1FA217B307E407F50720F049
:10D87000A21BB30BE40BF50B661F771F881F991FC4
:10D880001A9469F760957095809590959B01AC010D
:10D89000BD01CF01089597FB092E05260ED057FD37
:10D8A00004D0D7DF0AD0001C38F45095409530954D
:10D8B00021953F4F4F4F5F4F0895F6F79095809514
:10D8C000709561957F4F8F4F9F4F0895EE0FFF1F0B
:10D8D0000590F491E02D0994FB01DC01415050408A
:10D8E00048F005900D920020C9F701C01D924150EB
:10D8F0005040E0F708956817790768F4FB01DC01F0
:10D90000E40FF51FA40FB51F02C002900E92415004
:10D910005040D8F708950C94A46CDC0101C06D93BD
:10D9200041505040E0F70895DC01CB01FC01E19942
:10D93000FECF06C0FFBBEEBBE09A31960DB20D9252
:10D9400041505040B8F70895FB01DC0102C001903E
:0ED950000D9241505040D8F70895F894FFCF43
:10D95E0084038503860387034AF0004DFF072204E4
:10D96E007C5E9CCE003264E2F1003264645A505AFE
:10D97E006450463C46649CEC1E465AD50D1D0ED591
:10D98E000DFF0000AA05FF09FF0DFF135414AAD5C1
:02D99E000D007A
:00000001FF
